
IBM(R) Linker for OS/2(R), Version 5.0 
Copyright (C) IBM Corporation 1988, 2003.
Copyright (C) Microsoft Corp. 1988, 1989.
All rights reserved.

Current option settings:
	PDD	CODE:RX	DATA:RWS
	Alignfile:0x00000010	ALIGNAddr:0x00010000	NOBASe
	NOBRowse	NODBgpack	NODEbug:none	NODEFaultlibrarysearch
	EXEPACK:2	NOEXTdictionary	NOFIxed	FReeformat	NOIGnorecase
	Linenumbers	NOLOgo	MAP:bin\Release.ACP\uniaud32.map
	OCache:0x1d1d2000	OLDcpp	NOOPTFunc	PACKCode:0xffffffff
	PACKData:0xffffffff	PMTYPE:VIO	SEGMENTS:256 	NOSEGOrder
	NOSTRictwarnings	NONOSTRictwarnings	NOSTUB	NOVERBose
	VERSION:00.00


ILink : warning LNK4019: device driver can not have a stack

 UNIAUD32

 Start         Length     Name                   Class
 0001:00000000 000000483H DATA16                 DATA16 16-bit
	at offset 00000000 00483H bytes from F:\src\os2\uniaud32t\drv32\bin\Release.ACP\startup.obj (startup.asm)

 0002:00000000 0000006DBH CODE16                 CODE 16-bit
	at offset 00000000 006DBH bytes from F:\src\os2\uniaud32t\drv32\bin\Release.ACP\startup.obj (startup.asm)

 0003:00000000 000000000H FIRSTCODE32            CODE 32-bit

 0003:00000000 00008822CH CODE32                 CODE 32-bit
	at offset 00000000 004C1H bytes from F:\src\os2\uniaud32t\drv32\bin\Release.ACP\startup.obj (startup.asm)
	at offset 000004C1 000E9H bytes from F:\src\os2\uniaud32t\drv32\bin\Release.ACP\strategy.obj (F:\src\os2\uniaud32t\drv32\strategy.c)
	at offset 000005AA 00106H bytes from F:\src\os2\uniaud32t\drv32\bin\Release.ACP\read.obj (F:\src\os2\uniaud32t\drv32\read.cpp)
	at offset 000006B0 00EF4H bytes from F:\src\os2\uniaud32t\drv32\bin\Release.ACP\init.obj (F:\src\os2\uniaud32t\drv32\init.c)
	at offset 000015A4 01F6BH bytes from F:\src\os2\uniaud32t\drv32\bin\Release.ACP\parse.obj (F:\src\os2\uniaud32t\drv32\parse.c)
	at offset 00003510 0004EH bytes from F:\src\os2\uniaud32t\drv32\bin\Release.ACP\devhlp.obj (devhlp.asm)
	at offset 0000355E 00872H bytes from F:\src\os2\uniaud32t\drv32\bin\Release.ACP\idc.obj (F:\src\os2\uniaud32t\drv32\idc.c)
	at offset 00003DD0 00740H bytes from F:\src\os2\uniaud32t\drv32\bin\Release.ACP\dispatch.obj (F:\src\os2\uniaud32t\drv32\dispatch.c)
	at offset 00004510 00768H bytes from F:\src\os2\uniaud32t\drv32\bin\Release.ACP\rmhelp.obj (F:\src\os2\uniaud32t\drv32\rmhelp.cpp)
	at offset 00004C78 000F4H bytes from F:\src\os2\uniaud32t\drv32\bin\Release.ACP\irq.obj (F:\src\os2\uniaud32t\drv32\irq.cpp)
	at offset 00004D6C 0002DH bytes from F:\src\os2\uniaud32t\drv32\bin\Release.ACP\util.obj (F:\src\os2\uniaud32t\drv32\util.cpp)
	at offset 00004D99 004E6H bytes from F:\src\os2\uniaud32t\lib\Release.ACP\linuxlib.lib (vsprintf.c)
	at offset 0000527F 000FBH bytes from F:\src\os2\uniaud32t\lib\Release.ACP\linuxlib.lib (timer.c)
	at offset 0000537A 0004CH bytes from F:\src\os2\uniaud32t\lib\Release.ACP\linuxlib.lib (strncmp.c)
	at offset 000053C6 00039H bytes from F:\src\os2\uniaud32t\lib\Release.ACP\linuxlib.lib (task.c)
	at offset 000053FF 003EDH bytes from F:\src\os2\uniaud32t\lib\Release.ACP\linuxlib.lib (misc.c)
	at offset 000057EC 00362H bytes from F:\src\os2\uniaud32t\lib\Release.ACP\linuxlib.lib (ossidc.cpp)
	at offset 00005B4E 00643H bytes from F:\src\os2\uniaud32t\lib\Release.ACP\linuxlib.lib (soundmidi.c)
	at offset 00006191 01010H bytes from F:\src\os2\uniaud32t\lib\Release.ACP\linuxlib.lib (soundmixer.c)
	at offset 000071A1 0180EH bytes from F:\src\os2\uniaud32t\lib\Release.ACP\linuxlib.lib (sound.c)
	at offset 000089AF 0055CH bytes from F:\src\os2\uniaud32t\lib\Release.ACP\linuxlib.lib (debug.c)
	at offset 00008F0B 00CB7H bytes from F:\src\os2\uniaud32t\lib\Release.ACP\linuxlib.lib (memory.cpp)
	at offset 00009BC2 0103AH bytes from F:\src\os2\uniaud32t\lib\Release.ACP\linuxlib.lib (ioctl.c)
	at offset 0000ABFC 002B0H bytes from F:\src\os2\uniaud32t\lib\Release.ACP\linuxlib.lib (irq.c)
	at offset 0000AEAC 01B08H bytes from F:\src\os2\uniaud32t\lib\Release.ACP\linuxlib.lib (pci.c)
	at offset 0000C9B4 00560H bytes from F:\src\os2\uniaud32t\lib\Release.ACP\linuxlib.lib (malloc.cpp)
	at offset 0000CF14 00025H bytes from F:\src\os2\uniaud32t\lib\Release.ACP\linuxlib.lib (strncpy.c)
	at offset 0000CF39 00010H bytes from F:\src\os2\uniaud32t\lib\Release.ACP\linuxlib.lib (waitqueue.c)
	at offset 0000CF49 00023H bytes from F:\src\os2\uniaud32t\lib\Release.ACP\linuxlib.lib (spinlock.c)
	at offset 0000CF6C 008EAH bytes from F:\src\os2\uniaud32t\lib\Release.ACP\core.lib (hwdep.c)
	at offset 0000D856 024B5H bytes from F:\src\os2\uniaud32t\lib\Release.ACP\core.lib (timer.c)
	at offset 0000FD0B 01D02H bytes from F:\src\os2\uniaud32t\lib\Release.ACP\core.lib (rawmidi.c)
	at offset 00011A0D 002EEH bytes from F:\src\os2\uniaud32t\lib\Release.ACP\core.lib (pcm_misc.c)
	at offset 00011CFB 0276EH bytes from F:\src\os2\uniaud32t\lib\Release.ACP\core.lib (pcm_lib.c)
	at offset 00014469 00C24H bytes from F:\src\os2\uniaud32t\lib\Release.ACP\core.lib (pcm.c)
	at offset 0001508D 003F9H bytes from F:\src\os2\uniaud32t\lib\Release.ACP\core.lib (sound.c)
	at offset 00015486 00C78H bytes from F:\src\os2\uniaud32t\lib\Release.ACP\core.lib (info.c)
	at offset 000160FE 00323H bytes from F:\src\os2\uniaud32t\lib\Release.ACP\core.lib (pcm_memory.c)
	at offset 00016421 00227H bytes from F:\src\os2\uniaud32t\lib\Release.ACP\core.lib (pcm_timer.c)
	at offset 00016648 037D6H bytes from F:\src\os2\uniaud32t\lib\Release.ACP\core.lib (pcm_native.c)
	at offset 00019E1E 0020CH bytes from F:\src\os2\uniaud32t\lib\Release.ACP\core.lib (info_oss.c)
	at offset 0001A02A 00324H bytes from F:\src\os2\uniaud32t\lib\Release.ACP\core.lib (sound_oss.c)
	at offset 0001A34E 00279H bytes from F:\src\os2\uniaud32t\lib\Release.ACP\core.lib (device.c)
	at offset 0001A5C7 01B3BH bytes from F:\src\os2\uniaud32t\lib\Release.ACP\core.lib (control.c)
	at offset 0001C102 003A2H bytes from F:\src\os2\uniaud32t\lib\Release.ACP\core.lib (memalloc.c)
	at offset 0001C4A4 00C56H bytes from F:\src\os2\uniaud32t\lib\Release.ACP\core.lib (init.c)
	at offset 0001D0FA 001A1H bytes from F:\src\os2\uniaud32t\lib\Release.ACP\core.lib (sgbuf.c)
	at offset 0001D29B 00E4CH bytes from F:\src\os2\uniaud32t\lib\Release.ACP\pci.lib (bt87x.c)
	at offset 0001E0E7 00B2CH bytes from F:\src\os2\uniaud32t\lib\Release.ACP\pci.lib (als4000.c)
	at offset 0001EC13 03090H bytes from F:\src\os2\uniaud32t\lib\Release.ACP\pci.lib (cmipci.c)
	at offset 00021CA3 01700H bytes from F:\src\os2\uniaud32t\lib\Release.ACP\pci.lib (atiixp.c)
	at offset 000233A3 013E1H bytes from F:\src\os2\uniaud32t\lib\Release.ACP\pci.lib (fm801.c)
	at offset 00024784 024F8H bytes from F:\src\os2\uniaud32t\lib\Release.ACP\pci.lib (via82xx.c)
	at offset 00026C7C 01F46H bytes from F:\src\os2\uniaud32t\lib\Release.ACP\pci.lib (maestro3.c)
	at offset 00028BC2 02A10H bytes from F:\src\os2\uniaud32t\lib\Release.ACP\pci.lib (intel8x0.c)
	at offset 0002B5D2 02CCCH bytes from F:\src\os2\uniaud32t\lib\Release.ACP\pci.lib (es1968.c)
	at offset 0002E29E 01B02H bytes from F:\src\os2\uniaud32t\lib\Release.ACP\pci.lib (es1938.c)
	at offset 0002FDA0 01A5EH bytes from F:\src\os2\uniaud32t\lib\Release.ACP\pci.lib (cs4281.c)
	at offset 000317FE 01EA7H bytes from F:\src\os2\uniaud32t\lib\Release.ACP\pci.lib (ens1371.c)
	at offset 000336A5 00234H bytes from F:\src\os2\uniaud32t\lib\Release.ACP\pci.lib (pci_iomap_compat.c)
	at offset 000338D9 0197BH bytes from F:\src\os2\uniaud32t\lib\Release.ACP\ca0106.lib (ca0106_main.c)
	at offset 00035254 0050BH bytes from F:\src\os2\uniaud32t\lib\Release.ACP\ca0106.lib (ca_midi.c)
	at offset 0003575F 00B8FH bytes from F:\src\os2\uniaud32t\lib\Release.ACP\ca0106.lib (ca0106_mixer.c)
	at offset 000362EE 008F1H bytes from F:\src\os2\uniaud32t\lib\Release.ACP\ca0106.lib (ca0106_proc.c)
	at offset 00036BDF 02D74H bytes from F:\src\os2\uniaud32t\lib\Release.ACP\hda.lib (patch_via.c)
	at offset 00039953 010D5H bytes from F:\src\os2\uniaud32t\lib\Release.ACP\hda.lib (patch_conexant.c)
	at offset 0003AA28 001D6H bytes from F:\src\os2\uniaud32t\lib\Release.ACP\hda.lib (patch_atihdmi.c)
	at offset 0003ABFE 04A1CH bytes from F:\src\os2\uniaud32t\lib\Release.ACP\hda.lib (patch_sigmatel.c)
	at offset 0003F61A 022D2H bytes from F:\src\os2\uniaud32t\lib\Release.ACP\hda.lib (patch_analog.c)
	at offset 000418EC 0070DH bytes from F:\src\os2\uniaud32t\lib\Release.ACP\hda.lib (patch_cmedia.c)
	at offset 00041FF9 072BCH bytes from F:\src\os2\uniaud32t\lib\Release.ACP\hda.lib (patch_realtek.c)
	at offset 000492B5 02475H bytes from F:\src\os2\uniaud32t\lib\Release.ACP\hda.lib (hda_intel.c)
	at offset 0004B72A 03CCDH bytes from F:\src\os2\uniaud32t\lib\Release.ACP\hda.lib (hda_codec.c)
	at offset 0004F3F7 00270H bytes from F:\src\os2\uniaud32t\lib\Release.ACP\hda.lib (hda_hwdep.c)
	at offset 0004F667 01299H bytes from F:\src\os2\uniaud32t\lib\Release.ACP\hda.lib (hda_generic.c)
	at offset 00050900 010D4H bytes from F:\src\os2\uniaud32t\lib\Release.ACP\hda.lib (hda_proc.c)
	at offset 000519D4 0004BH bytes from F:\src\os2\uniaud32t\lib\Release.ACP\sequencer.lib (seq.c)
	at offset 00051A1F 00699H bytes from F:\src\os2\uniaud32t\lib\Release.ACP\sequencer.lib (seq_device.c)
	at offset 000520B8 000A1H bytes from F:\src\os2\uniaud32t\lib\Release.ACP\sequencer.lib (seq_info.c)
	at offset 00052159 00212H bytes from F:\src\os2\uniaud32t\lib\Release.ACP\sequencer.lib (seq_system.c)
	at offset 0005236B 00B72H bytes from F:\src\os2\uniaud32t\lib\Release.ACP\sequencer.lib (seq_queue.c)
	at offset 00052EDD 0077CH bytes from F:\src\os2\uniaud32t\lib\Release.ACP\sequencer.lib (seq_memory.c)
	at offset 00053659 024F9H bytes from F:\src\os2\uniaud32t\lib\Release.ACP\sequencer.lib (seq_clientmgr.c)
	at offset 00055B52 00BDCH bytes from F:\src\os2\uniaud32t\lib\Release.ACP\sequencer.lib (seq_ports.c)
	at offset 0005672E 00765H bytes from F:\src\os2\uniaud32t\lib\Release.ACP\sequencer.lib (seq_timer.c)
	at offset 00056E93 004DEH bytes from F:\src\os2\uniaud32t\lib\Release.ACP\sequencer.lib (seq_prioq.c)
	at offset 00057371 00319H bytes from F:\src\os2\uniaud32t\lib\Release.ACP\sequencer.lib (seq_fifo.c)
	at offset 0005768A 003D5H bytes from F:\src\os2\uniaud32t\lib\Release.ACP\opl3.lib (opl3_seq.c)
	at offset 00057A5F 0090DH bytes from F:\src\os2\uniaud32t\lib\Release.ACP\opl3.lib (opl3_lib.c)
	at offset 0005836C 0029CH bytes from F:\src\os2\uniaud32t\lib\Release.ACP\opl3.lib (opl3_drums.c)
	at offset 00058608 00BECH bytes from F:\src\os2\uniaud32t\lib\Release.ACP\opl3.lib (opl3_midi.c)
	at offset 000591F4 00820H bytes from F:\src\os2\uniaud32t\lib\Release.ACP\opl3.lib (opl3_synth.c)
	at offset 00059A14 008B7H bytes from F:\src\os2\uniaud32t\lib\Release.ACP\mpu401.lib (mpu401_uart.c)
	at offset 0005A2CB 001E3H bytes from F:\src\os2\uniaud32t\lib\Release.ACP\cs46xx.lib (cs46xx.c)
	at offset 0005A4AE 02659H bytes from F:\src\os2\uniaud32t\lib\Release.ACP\cs46xx.lib (cs46xx_lib.c)
	at offset 0005CB07 0057BH bytes from F:\src\os2\uniaud32t\lib\Release.ACP\cs5535audio.lib (cs5535audio.c)
	at offset 0005D082 001A2H bytes from F:\src\os2\uniaud32t\lib\Release.ACP\cs5535audio.lib (cs5535audio_pm.c)
	at offset 0005D224 00518H bytes from F:\src\os2\uniaud32t\lib\Release.ACP\cs5535audio.lib (cs5535audio_pcm.c)
	at offset 0005D73C 004DFH bytes from F:\src\os2\uniaud32t\lib\Release.ACP\emu10k1.lib (emu10k1.c)
	at offset 0005DC1B 00BF5H bytes from F:\src\os2\uniaud32t\lib\Release.ACP\emu10k1.lib (p16v.c)
	at offset 0005E810 00149H bytes from F:\src\os2\uniaud32t\lib\Release.ACP\emu10k1.lib (timer.c)
	at offset 0005E959 075B4H bytes from F:\src\os2\uniaud32t\lib\Release.ACP\emu10k1.lib (emufx.c)
	at offset 00065F0D 01E71H bytes from F:\src\os2\uniaud32t\lib\Release.ACP\emu10k1.lib (emumixer.c)
	at offset 00067D7E 027E7H bytes from F:\src\os2\uniaud32t\lib\Release.ACP\emu10k1.lib (emupcm.c)
	at offset 0006A565 006ADH bytes from F:\src\os2\uniaud32t\lib\Release.ACP\emu10k1.lib (emumpu401.c)
	at offset 0006AC12 01E56H bytes from F:\src\os2\uniaud32t\lib\Release.ACP\emu10k1.lib (emu10k1_main.c)
	at offset 0006CA68 00B3CH bytes from F:\src\os2\uniaud32t\lib\Release.ACP\emu10k1.lib (emuproc.c)
	at offset 0006D5A4 00A33H bytes from F:\src\os2\uniaud32t\lib\Release.ACP\emu10k1.lib (io.c)
	at offset 0006DFD7 0025FH bytes from F:\src\os2\uniaud32t\lib\Release.ACP\emu10k1.lib (voice.c)
	at offset 0006E236 0081AH bytes from F:\src\os2\uniaud32t\lib\Release.ACP\emu10k1.lib (memory.c)
	at offset 0006EA50 0041DH bytes from F:\src\os2\uniaud32t\lib\Release.ACP\emu10k1.lib (irq.c)
	at offset 0006EE6D 0066EH bytes from F:\src\os2\uniaud32t\lib\Release.ACP\ymfpci.lib (ymfpci.c)
	at offset 0006F4DB 02D18H bytes from F:\src\os2\uniaud32t\lib\Release.ACP\ymfpci.lib (ymfpci_main.c)
	at offset 000721F3 02117H bytes from F:\src\os2\uniaud32t\lib\Release.ACP\ali5451.lib (ali5451.c)
	at offset 0007430A 002E5H bytes from F:\src\os2\uniaud32t\lib\Release.ACP\trident.lib (trident.c)
	at offset 000745EF 03936H bytes from F:\src\os2\uniaud32t\lib\Release.ACP\trident.lib (trident_main.c)
	at offset 00077F25 00300H bytes from F:\src\os2\uniaud32t\lib\Release.ACP\trident.lib (trident_memory.c)
	at offset 00078225 0156BH bytes from F:\src\os2\uniaud32t\lib\Release.ACP\nm256.lib (nm256.c)
	at offset 00079790 00CB6H bytes from F:\src\os2\uniaud32t\lib\Release.ACP\sb.lib (sb_mixer.c)
	at offset 0007A446 003D4H bytes from F:\src\os2\uniaud32t\lib\Release.ACP\sb.lib (sb_common.c)
	at offset 0007A81A 037F4H bytes from F:\src\os2\uniaud32t\lib\Release.ACP\core_oss.lib (pcm_oss.c)
	at offset 0007E020 00140H bytes from F:\acpi\lib\acpidrv.lib (acpi)
	at offset 0007E160 002BCH bytes from F:\acpi\lib\acpidrv.lib (FindAddress)
	at offset 0007E41C 00007H bytes from F:\src\os2\uniaud32t\lib\Release.ACP\linuxlib.lib (semaphore.c)
	at offset 0007E423 00574H bytes from F:\src\os2\uniaud32t\lib\Release.ACP\core.lib (vmaster.c)
	at offset 0007E997 00055H bytes from F:\src\os2\uniaud32t\lib\Release.ACP\core.lib (misc.c)
	at offset 0007E9EC 000DFH bytes from F:\src\os2\uniaud32t\lib\Release.ACP\core.lib (memory.c)
	at offset 0007EACB 00CCBH bytes from F:\src\os2\uniaud32t\lib\Release.ACP\ac97.lib (ac97_pcm.c)
	at offset 0007F796 06DACH bytes from F:\src\os2\uniaud32t\lib\Release.ACP\ac97.lib (ac97_codec.c)
	at offset 00086542 0103DH bytes from F:\src\os2\uniaud32t\lib\Release.ACP\ac97.lib (ac97_proc.c)
	at offset 0008757F 00B03H bytes from F:\src\os2\uniaud32t\lib\Release.ACP\sequencer.lib (seq_midi_emul.c)
	at offset 00088082 001AAH bytes from F:\src\os2\uniaud32t\lib\Release.ACP\synth.lib (util_mem.c)

 0003:00088230 0000029B8H _TEXT                  CODE 32-bit
	at offset 00000000 0004FH bytes from E:\watcom\lib386\os2\clib3r.lib (i8s)
	at offset 00000050 0001CH bytes from E:\watcom\lib386\os2\clib3r.lib (i8m)
	at offset 00000070 000ADH bytes from E:\watcom\lib386\os2\clib3r.lib (strstr.c)
	at offset 00000120 00041H bytes from E:\watcom\lib386\os2\clib3r.lib (strlcpy.c)
	at offset 00000170 00091H bytes from E:\watcom\lib386\os2\clib3r.lib (sscanf.c)
	at offset 00000210 000C7H bytes from E:\watcom\lib386\os2\clib3r.lib (snprintf.c)
	at offset 000002E0 00018H bytes from E:\watcom\lib386\os2\clib3r.lib (memset.c)
	at offset 00000300 00053H bytes from E:\watcom\lib386\os2\clib3r.lib (memmove.c)
	at offset 00000360 00101H bytes from E:\watcom\lib386\os2\clib3r.lib (istable.c)
	at offset 00000470 000A3H bytes from E:\watcom\lib386\os2\clib3r.lib (__stos)
	at offset 00000520 00DCBH bytes from E:\watcom\lib386\os2\clib3r.lib (scnf.c)
	at offset 000012F0 00CE4H bytes from E:\watcom\lib386\os2\clib3r.lib (prtf.c)
	at offset 00001FD4 0004CH bytes from E:\watcom\lib386\os2\clib3r.lib (fdfs386)
	at offset 00002020 00020H bytes from E:\watcom\lib386\os2\clib3r.lib (strupr.c)
	at offset 00002040 00008H bytes from E:\watcom\lib386\os2\clib3r.lib (bits.c)
	at offset 00002050 00042H bytes from E:\watcom\lib386\os2\clib3r.lib (noefgfmt.c)
	at offset 000020A0 0002EH bytes from E:\watcom\lib386\os2\clib3r.lib (wctomb.c)
	at offset 000020D0 000BCH bytes from E:\watcom\lib386\os2\clib3r.lib (mbtowc.c)
	at offset 00002190 00017H bytes from E:\watcom\lib386\os2\clib3r.lib (mbislead.c)
	at offset 000021B0 00074H bytes from E:\watcom\lib386\os2\clib3r.lib (ltoa.c)
	at offset 00002230 00099H bytes from E:\watcom\lib386\os2\clib3r.lib (lltoa.c)
	at offset 000022D0 00074H bytes from E:\watcom\lib386\os2\clib3r.lib (itoa.c)
	at offset 00002350 0000EH bytes from E:\watcom\lib386\os2\clib3r.lib (tolower.c)
	at offset 00002360 00070H bytes from E:\watcom\lib386\os2\clib3r.lib (xmsgo32.c)
	at offset 000023D0 00132H bytes from E:\watcom\lib386\os2\clib3r.lib (mbinit.c)
	at offset 00002502 00128H bytes from E:\watcom\lib386\os2\clib3r.lib (maino32.c)
	at offset 00002630 00026H bytes from E:\watcom\lib386\os2\clib3r.lib (enterdb.c)
	at offset 00002660 000B3H bytes from E:\watcom\lib386\os2\clib3r.lib (initrtns.c)
	at offset 00002713 00001H bytes from E:\watcom\lib386\os2\clib3r.lib (crwdata)
	at offset 00002720 0000BH bytes from E:\watcom\lib386\os2\clib3r.lib (cinit.c)
	at offset 00002730 0023DH bytes from E:\watcom\lib386\os2\clib3r.lib (strtol.c)
	at offset 0000296D 0004BH bytes from E:\watcom\lib386\os2\clib3r.lib (seterrno.c)

 0003:0008ABE8 000000000H LASTCODE32             CODE 32-bit

 0004:00000000 000000007H BEGTEXT                CODE 32-bit
	at offset 00000000 00007H bytes from E:\watcom\lib386\os2\clib3r.lib (segdefns)

 0005:00000000 000000030H BSS32                  BSS 32-bit
	at offset 00000000 00004H bytes from F:\src\os2\uniaud32t\drv32\bin\Release.ACP\begin.obj (begin.asm)
	at offset 00000004 0002CH bytes from F:\acpi\lib\acpidrv.lib (acpi)

 0005:00000030 000001728H _BSS                   BSS 32-bit
	at offset 00000000 00008H bytes from F:\src\os2\uniaud32t\drv32\bin\Release.ACP\strategy.obj (F:\src\os2\uniaud32t\drv32\strategy.c)
	at offset 00000008 0000CH bytes from F:\src\os2\uniaud32t\drv32\bin\Release.ACP\read.obj (F:\src\os2\uniaud32t\drv32\read.cpp)
	at offset 00000014 00008H bytes from F:\src\os2\uniaud32t\drv32\bin\Release.ACP\parse.obj (F:\src\os2\uniaud32t\drv32\parse.c)
	at offset 0000001C 00006H bytes from F:\src\os2\uniaud32t\drv32\bin\Release.ACP\idc.obj (F:\src\os2\uniaud32t\drv32\idc.c)
	at offset 00000024 0005CH bytes from F:\src\os2\uniaud32t\drv32\bin\Release.ACP\rmhelp.obj (F:\src\os2\uniaud32t\drv32\rmhelp.cpp)
	at offset 00000080 00028H bytes from F:\src\os2\uniaud32t\lib\Release.ACP\linuxlib.lib (ossidc.cpp)
	at offset 000000A8 00028H bytes from F:\src\os2\uniaud32t\lib\Release.ACP\linuxlib.lib (debug.c)
	at offset 000000D0 00008H bytes from F:\src\os2\uniaud32t\lib\Release.ACP\linuxlib.lib (memory.cpp)
	at offset 000000D8 00440H bytes from F:\src\os2\uniaud32t\lib\Release.ACP\linuxlib.lib (pci.c)
	at offset 00000518 0002CH bytes from F:\src\os2\uniaud32t\lib\Release.ACP\linuxlib.lib (malloc.cpp)
	at offset 00000544 00004H bytes from F:\src\os2\uniaud32t\lib\Release.ACP\core.lib (hwdep.c)
	at offset 00000548 00004H bytes from F:\src\os2\uniaud32t\lib\Release.ACP\core.lib (timer.c)
	at offset 0000054C 00020H bytes from F:\src\os2\uniaud32t\lib\Release.ACP\core.lib (rawmidi.c)
	at offset 0000056C 00104H bytes from F:\src\os2\uniaud32t\lib\Release.ACP\core.lib (pcm.c)
	at offset 00000670 0040CH bytes from F:\src\os2\uniaud32t\lib\Release.ACP\core.lib (sound.c)
	at offset 00000A7C 00010H bytes from F:\src\os2\uniaud32t\lib\Release.ACP\core.lib (info.c)
	at offset 00000A8C 000C4H bytes from F:\src\os2\uniaud32t\lib\Release.ACP\core.lib (info_oss.c)
	at offset 00000B50 00204H bytes from F:\src\os2\uniaud32t\lib\Release.ACP\core.lib (sound_oss.c)
	at offset 00000D54 00004H bytes from F:\src\os2\uniaud32t\lib\Release.ACP\core.lib (memalloc.c)
	at offset 00000D58 0004CH bytes from F:\src\os2\uniaud32t\lib\Release.ACP\core.lib (init.c)
	at offset 00000DA4 00028H bytes from F:\src\os2\uniaud32t\lib\Release.ACP\pci.lib (bt87x.c)
	at offset 00000DCC 00004H bytes from F:\src\os2\uniaud32t\lib\Release.ACP\pci.lib (als4000.c)
	at offset 00000DD0 00024H bytes from F:\src\os2\uniaud32t\lib\Release.ACP\pci.lib (cmipci.c)
	at offset 00000DF4 00008H bytes from F:\src\os2\uniaud32t\lib\Release.ACP\pci.lib (atiixp.c)
	at offset 00000DFC 00024H bytes from F:\src\os2\uniaud32t\lib\Release.ACP\pci.lib (fm801.c)
	at offset 00000E20 00014H bytes from F:\src\os2\uniaud32t\lib\Release.ACP\pci.lib (via82xx.c)
	at offset 00000E34 00004H bytes from F:\src\os2\uniaud32t\lib\Release.ACP\pci.lib (maestro3.c)
	at offset 00000E38 00018H bytes from F:\src\os2\uniaud32t\lib\Release.ACP\pci.lib (intel8x0.c)
	at offset 00000E50 00024H bytes from F:\src\os2\uniaud32t\lib\Release.ACP\pci.lib (es1968.c)
	at offset 00000E74 00004H bytes from F:\src\os2\uniaud32t\lib\Release.ACP\pci.lib (es1938.c)
	at offset 00000E78 00024H bytes from F:\src\os2\uniaud32t\lib\Release.ACP\pci.lib (cs4281.c)
	at offset 00000E9C 00044H bytes from F:\src\os2\uniaud32t\lib\Release.ACP\pci.lib (ens1371.c)
	at offset 00000EE0 00024H bytes from F:\src\os2\uniaud32t\lib\Release.ACP\ca0106.lib (ca0106_main.c)
	at offset 00000F04 00008H bytes from F:\src\os2\uniaud32t\lib\Release.ACP\hda.lib (patch_sigmatel.c)
	at offset 00000F0C 0006CH bytes from F:\src\os2\uniaud32t\lib\Release.ACP\hda.lib (hda_intel.c)
	at offset 00000F78 00008H bytes from F:\src\os2\uniaud32t\lib\Release.ACP\sequencer.lib (seq_device.c)
	at offset 00000F80 0000CH bytes from F:\src\os2\uniaud32t\lib\Release.ACP\sequencer.lib (seq_info.c)
	at offset 00000F8C 00024H bytes from F:\src\os2\uniaud32t\lib\Release.ACP\sequencer.lib (seq_queue.c)
	at offset 00000FB0 003C8H bytes from F:\src\os2\uniaud32t\lib\Release.ACP\sequencer.lib (seq_clientmgr.c)
	at offset 00001378 00044H bytes from F:\src\os2\uniaud32t\lib\Release.ACP\cs46xx.lib (cs46xx.c)
	at offset 000013BC 00008H bytes from F:\src\os2\uniaud32t\lib\Release.ACP\cs5535audio.lib (cs5535audio.c)
	at offset 000013C4 00084H bytes from F:\src\os2\uniaud32t\lib\Release.ACP\emu10k1.lib (emu10k1.c)
	at offset 00001448 00064H bytes from F:\src\os2\uniaud32t\lib\Release.ACP\ymfpci.lib (ymfpci.c)
	at offset 000014AC 00008H bytes from F:\src\os2\uniaud32t\lib\Release.ACP\ali5451.lib (ali5451.c)
	at offset 000014B4 00004H bytes from F:\src\os2\uniaud32t\lib\Release.ACP\trident.lib (trident.c)
	at offset 000014B8 0001CH bytes from F:\src\os2\uniaud32t\lib\Release.ACP\nm256.lib (nm256.c)
	at offset 000014D4 00020H bytes from F:\src\os2\uniaud32t\lib\Release.ACP\core_oss.lib (pcm_oss.c)
	at offset 000014F4 00101H bytes from E:\watcom\lib386\os2\clib3r.lib (mbislead.c)
	at offset 000015F8 00004H bytes from E:\watcom\lib386\os2\clib3r.lib (mbisdbcs.c)
	at offset 000015FC 00106H bytes from E:\watcom\lib386\os2\clib3r.lib (maino32.c)
	at offset 00001704 00004H bytes from E:\watcom\lib386\os2\clib3r.lib (cinit.c)
	at offset 00001708 00020H bytes from F:\src\os2\uniaud32t\lib\Release.ACP\ac97.lib (ac97_codec.c)

 0005:00001758 000000000H C_COMMON               DATA 32-bit

 0005:00001758 000000010H c_common               DATA 32-bit
	at offset 00000000 00010H bytes from F:\acpi\lib\acpidrv.lib (acpi)

 0005:00001768 000000098H DATA32                 DATA 32-bit
	at offset 00000000 0008AH bytes from F:\src\os2\uniaud32t\drv32\bin\Release.ACP\startup.obj (startup.asm)
	at offset 0000008C 0000CH bytes from F:\src\os2\uniaud32t\drv32\bin\Release.ACP\devhlp.obj (devhlp.asm)

 0005:00001800 00005E334H _DATA                  DATA 32-bit
	at offset 00000000 00080H bytes from F:\src\os2\uniaud32t\drv32\bin\Release.ACP\strategy.obj (F:\src\os2\uniaud32t\drv32\strategy.c)
	at offset 00000080 00018H bytes from F:\src\os2\uniaud32t\drv32\bin\Release.ACP\parse.obj (F:\src\os2\uniaud32t\drv32\parse.c)
	at offset 00000098 00004H bytes from F:\src\os2\uniaud32t\drv32\bin\Release.ACP\rmhelp.obj (F:\src\os2\uniaud32t\drv32\rmhelp.cpp)
	at offset 0000009C 00020H bytes from F:\src\os2\uniaud32t\drv32\bin\Release.ACP\irq.obj (F:\src\os2\uniaud32t\drv32\irq.cpp)
	at offset 000000BC 0000CH bytes from F:\src\os2\uniaud32t\lib\Release.ACP\linuxlib.lib (timer.c)
	at offset 000000C8 00028H bytes from F:\src\os2\uniaud32t\lib\Release.ACP\linuxlib.lib (task.c)
	at offset 000000F0 00414H bytes from F:\src\os2\uniaud32t\lib\Release.ACP\linuxlib.lib (misc.c)
	at offset 00000504 00108H bytes from F:\src\os2\uniaud32t\lib\Release.ACP\linuxlib.lib (ossidc.cpp)
	at offset 0000060C 00004H bytes from F:\src\os2\uniaud32t\lib\Release.ACP\linuxlib.lib (soundmidi.c)
	at offset 00000610 001F1H bytes from F:\src\os2\uniaud32t\lib\Release.ACP\linuxlib.lib (soundmixer.c)
	at offset 00000804 061D8H bytes from F:\src\os2\uniaud32t\lib\Release.ACP\linuxlib.lib (sound.c)
	at offset 000069DC 00013H bytes from F:\src\os2\uniaud32t\lib\Release.ACP\linuxlib.lib (debug.c)
	at offset 000069F0 0202CH bytes from F:\src\os2\uniaud32t\lib\Release.ACP\linuxlib.lib (ioctl.c)
	at offset 00008A1C 00880H bytes from F:\src\os2\uniaud32t\lib\Release.ACP\linuxlib.lib (irq.c)
	at offset 0000929C 03F44H bytes from F:\src\os2\uniaud32t\lib\Release.ACP\linuxlib.lib (pci.c)
	at offset 0000D1E0 00004H bytes from F:\src\os2\uniaud32t\lib\Release.ACP\linuxlib.lib (malloc.cpp)
	at offset 0000D1E4 00068H bytes from F:\src\os2\uniaud32t\lib\Release.ACP\core.lib (hwdep.c)
	at offset 0000D24C 000ACH bytes from F:\src\os2\uniaud32t\lib\Release.ACP\core.lib (timer.c)
	at offset 0000D2F8 00090H bytes from F:\src\os2\uniaud32t\lib\Release.ACP\core.lib (rawmidi.c)
	at offset 0000D388 00210H bytes from F:\src\os2\uniaud32t\lib\Release.ACP\core.lib (pcm_misc.c)
	at offset 0000D598 000A0H bytes from F:\src\os2\uniaud32t\lib\Release.ACP\core.lib (pcm_lib.c)
	at offset 0000D638 00030H bytes from F:\src\os2\uniaud32t\lib\Release.ACP\core.lib (pcm.c)
	at offset 0000D668 0005CH bytes from F:\src\os2\uniaud32t\lib\Release.ACP\core.lib (sound.c)
	at offset 0000D6C4 00048H bytes from F:\src\os2\uniaud32t\lib\Release.ACP\core.lib (info.c)
	at offset 0000D70C 00008H bytes from F:\src\os2\uniaud32t\lib\Release.ACP\core.lib (pcm_memory.c)
	at offset 0000D714 00030H bytes from F:\src\os2\uniaud32t\lib\Release.ACP\core.lib (pcm_timer.c)
	at offset 0000D744 00144H bytes from F:\src\os2\uniaud32t\lib\Release.ACP\core.lib (pcm_native.c)
	at offset 0000D888 0000CH bytes from F:\src\os2\uniaud32t\lib\Release.ACP\core.lib (info_oss.c)
	at offset 0000D894 0000CH bytes from F:\src\os2\uniaud32t\lib\Release.ACP\core.lib (sound_oss.c)
	at offset 0000D8A0 00060H bytes from F:\src\os2\uniaud32t\lib\Release.ACP\core.lib (control.c)
	at offset 0000D900 0001CH bytes from F:\src\os2\uniaud32t\lib\Release.ACP\core.lib (memalloc.c)
	at offset 0000D91C 00058H bytes from F:\src\os2\uniaud32t\lib\Release.ACP\core.lib (init.c)
	at offset 0000D974 00408H bytes from F:\src\os2\uniaud32t\lib\Release.ACP\pci.lib (bt87x.c)
	at offset 0000DD7C 0019CH bytes from F:\src\os2\uniaud32t\lib\Release.ACP\pci.lib (als4000.c)
	at offset 0000DF18 00E61H bytes from F:\src\os2\uniaud32t\lib\Release.ACP\pci.lib (cmipci.c)
	at offset 0000ED7C 003A0H bytes from F:\src\os2\uniaud32t\lib\Release.ACP\pci.lib (atiixp.c)
	at offset 0000F11C 004C0H bytes from F:\src\os2\uniaud32t\lib\Release.ACP\pci.lib (fm801.c)
	at offset 0000F5DC 00614H bytes from F:\src\os2\uniaud32t\lib\Release.ACP\pci.lib (via82xx.c)
	at offset 0000FBF0 00624H bytes from F:\src\os2\uniaud32t\lib\Release.ACP\pci.lib (maestro3.c)
	at offset 00010214 00F74H bytes from F:\src\os2\uniaud32t\lib\Release.ACP\pci.lib (intel8x0.c)
	at offset 00011188 002B4H bytes from F:\src\os2\uniaud32t\lib\Release.ACP\pci.lib (es1968.c)
	at offset 0001143C 00899H bytes from F:\src\os2\uniaud32t\lib\Release.ACP\pci.lib (es1938.c)
	at offset 00011CD8 002D0H bytes from F:\src\os2\uniaud32t\lib\Release.ACP\pci.lib (cs4281.c)
	at offset 00011FA8 0047CH bytes from F:\src\os2\uniaud32t\lib\Release.ACP\pci.lib (ens1371.c)
	at offset 00012424 004ECH bytes from F:\src\os2\uniaud32t\lib\Release.ACP\ca0106.lib (ca0106_main.c)
	at offset 00012910 00020H bytes from F:\src\os2\uniaud32t\lib\Release.ACP\ca0106.lib (ca_midi.c)
	at offset 00012930 00634H bytes from F:\src\os2\uniaud32t\lib\Release.ACP\ca0106.lib (ca0106_mixer.c)
	at offset 00012F64 00058H bytes from F:\src\os2\uniaud32t\lib\Release.ACP\ca0106.lib (ca0106_proc.c)
	at offset 00012FBC 01668H bytes from F:\src\os2\uniaud32t\lib\Release.ACP\hda.lib (patch_via.c)
	at offset 00014624 01E20H bytes from F:\src\os2\uniaud32t\lib\Release.ACP\hda.lib (patch_conexant.c)
	at offset 00016444 0015CH bytes from F:\src\os2\uniaud32t\lib\Release.ACP\hda.lib (patch_atihdmi.c)
	at offset 000165A0 02E96H bytes from F:\src\os2\uniaud32t\lib\Release.ACP\hda.lib (patch_sigmatel.c)
	at offset 00019438 07510H bytes from F:\src\os2\uniaud32t\lib\Release.ACP\hda.lib (patch_analog.c)
	at offset 00020948 00790H bytes from F:\src\os2\uniaud32t\lib\Release.ACP\hda.lib (patch_cmedia.c)
	at offset 000210D8 1CB2DH bytes from F:\src\os2\uniaud32t\lib\Release.ACP\hda.lib (patch_realtek.c)
	at offset 0003DC08 0062CH bytes from F:\src\os2\uniaud32t\lib\Release.ACP\hda.lib (hda_intel.c)
	at offset 0003E234 00447H bytes from F:\src\os2\uniaud32t\lib\Release.ACP\hda.lib (hda_codec.c)
	at offset 0003E67C 0008CH bytes from F:\src\os2\uniaud32t\lib\Release.ACP\hda.lib (hda_generic.c)
	at offset 0003E708 000E0H bytes from F:\src\os2\uniaud32t\lib\Release.ACP\hda.lib (hda_proc.c)
	at offset 0003E7E8 0005CH bytes from F:\src\os2\uniaud32t\lib\Release.ACP\sequencer.lib (seq.c)
	at offset 0003E844 00028H bytes from F:\src\os2\uniaud32t\lib\Release.ACP\sequencer.lib (seq_device.c)
	at offset 0003E86C 00008H bytes from F:\src\os2\uniaud32t\lib\Release.ACP\sequencer.lib (seq_system.c)
	at offset 0003E874 00004H bytes from F:\src\os2\uniaud32t\lib\Release.ACP\sequencer.lib (seq_queue.c)
	at offset 0003E878 00140H bytes from F:\src\os2\uniaud32t\lib\Release.ACP\sequencer.lib (seq_clientmgr.c)
	at offset 0003E9B8 00030H bytes from F:\src\os2\uniaud32t\lib\Release.ACP\opl3.lib (opl3_seq.c)
	at offset 0003E9E8 00074H bytes from F:\src\os2\uniaud32t\lib\Release.ACP\opl3.lib (opl3_lib.c)
	at offset 0003EA5C 000A7H bytes from F:\src\os2\uniaud32t\lib\Release.ACP\opl3.lib (opl3_drums.c)
	at offset 0003EB04 000E8H bytes from F:\src\os2\uniaud32t\lib\Release.ACP\opl3.lib (opl3_midi.c)
	at offset 0003EBEC 00024H bytes from F:\src\os2\uniaud32t\lib\Release.ACP\opl3.lib (opl3_synth.c)
	at offset 0003EC10 00028H bytes from F:\src\os2\uniaud32t\lib\Release.ACP\mpu401.lib (mpu401_uart.c)
	at offset 0003EC38 0011CH bytes from F:\src\os2\uniaud32t\lib\Release.ACP\cs46xx.lib (cs46xx.c)
	at offset 0003ED54 0DBC8H bytes from F:\src\os2\uniaud32t\lib\Release.ACP\cs46xx.lib (cs46xx_lib.c)
	at offset 0004C91C 00118H bytes from F:\src\os2\uniaud32t\lib\Release.ACP\cs5535audio.lib (cs5535audio.c)
	at offset 0004CA34 00110H bytes from F:\src\os2\uniaud32t\lib\Release.ACP\cs5535audio.lib (cs5535audio_pcm.c)
	at offset 0004CB44 0015CH bytes from F:\src\os2\uniaud32t\lib\Release.ACP\emu10k1.lib (emu10k1.c)
	at offset 0004CCA0 002E8H bytes from F:\src\os2\uniaud32t\lib\Release.ACP\emu10k1.lib (p16v.c)
	at offset 0004CF88 00030H bytes from F:\src\os2\uniaud32t\lib\Release.ACP\emu10k1.lib (timer.c)
	at offset 0004CFB8 001C0H bytes from F:\src\os2\uniaud32t\lib\Release.ACP\emu10k1.lib (emufx.c)
	at offset 0004D178 0169CH bytes from F:\src\os2\uniaud32t\lib\Release.ACP\emu10k1.lib (emumixer.c)
	at offset 0004E814 00334H bytes from F:\src\os2\uniaud32t\lib\Release.ACP\emu10k1.lib (emupcm.c)
	at offset 0004EB48 00020H bytes from F:\src\os2\uniaud32t\lib\Release.ACP\emu10k1.lib (emumpu401.c)
	at offset 0004EB68 00894H bytes from F:\src\os2\uniaud32t\lib\Release.ACP\emu10k1.lib (emu10k1_main.c)
	at offset 0004F3FC 00270H bytes from F:\src\os2\uniaud32t\lib\Release.ACP\emu10k1.lib (emuproc.c)
	at offset 0004F66C 00280H bytes from F:\src\os2\uniaud32t\lib\Release.ACP\emu10k1.lib (io.c)
	at offset 0004F8EC 00150H bytes from F:\src\os2\uniaud32t\lib\Release.ACP\ymfpci.lib (ymfpci.c)
	at offset 0004FA3C 006D8H bytes from F:\src\os2\uniaud32t\lib\Release.ACP\ymfpci.lib (ymfpci_main.c)
	at offset 00050114 002E8H bytes from F:\src\os2\uniaud32t\lib\Release.ACP\ali5451.lib (ali5451.c)
	at offset 000503FC 0013CH bytes from F:\src\os2\uniaud32t\lib\Release.ACP\trident.lib (trident.c)
	at offset 00050538 004ECH bytes from F:\src\os2\uniaud32t\lib\Release.ACP\trident.lib (trident_main.c)
	at offset 00050A24 0C808H bytes from F:\src\os2\uniaud32t\lib\Release.ACP\nm256.lib (nm256.c)
	at offset 0005D22C 005B0H bytes from F:\src\os2\uniaud32t\lib\Release.ACP\sb.lib (sb_mixer.c)
	at offset 0005D7DC 00014H bytes from F:\src\os2\uniaud32t\lib\Release.ACP\sb.lib (sb_common.c)
	at offset 0005D7F0 00080H bytes from F:\src\os2\uniaud32t\lib\Release.ACP\core_oss.lib (pcm_oss.c)
	at offset 0005D870 00008H bytes from E:\watcom\lib386\os2\clib3r.lib (noefgfmt.c)
	at offset 0005D878 00004H bytes from E:\watcom\lib386\os2\clib3r.lib (mbinit.c)
	at offset 0005D87C 00040H bytes from E:\watcom\lib386\os2\clib3r.lib (maino32.c)
	at offset 0005D8BC 00001H bytes from E:\watcom\lib386\os2\clib3r.lib (enterdb.c)
	at offset 0005D8C0 0004AH bytes from E:\watcom\lib386\os2\clib3r.lib (crwdata)
	at offset 0005D90C 00004H bytes from E:\watcom\lib386\os2\clib3r.lib (amblksiz.c)
	at offset 0005D910 00051H bytes from F:\src\os2\uniaud32t\lib\Release.ACP\ac97.lib (ac97_pcm.c)
	at offset 0005D964 00812H bytes from F:\src\os2\uniaud32t\lib\Release.ACP\ac97.lib (ac97_codec.c)
	at offset 0005E178 00110H bytes from F:\src\os2\uniaud32t\lib\Release.ACP\ac97.lib (ac97_proc.c)
	at offset 0005E288 00018H bytes from F:\src\os2\uniaud32t\lib\Release.ACP\sequencer.lib (seq_midi_emul.c)
	at offset 0005E2A0 00008H bytes from F:\src\os2\uniaud32t\lib\Release.ACP\synth.lib (util_mem.c)
	at offset 0005E2A8 0008CH bytes from E:\watcom\lib386\os2\clib3r.lib (strtol.c)

 0005:0005FB34 000012255H CONST                  DATA 32-bit
	at offset 00000000 00013H bytes from F:\src\os2\uniaud32t\drv32\bin\Release.ACP\strategy.obj (F:\src\os2\uniaud32t\drv32\strategy.c)
	at offset 00000013 00034H bytes from F:\src\os2\uniaud32t\drv32\bin\Release.ACP\init.obj (F:\src\os2\uniaud32t\drv32\init.c)
	at offset 00000047 00073H bytes from F:\src\os2\uniaud32t\drv32\bin\Release.ACP\parse.obj (F:\src\os2\uniaud32t\drv32\parse.c)
	at offset 000000BA 00012H bytes from F:\src\os2\uniaud32t\drv32\bin\Release.ACP\idc.obj (F:\src\os2\uniaud32t\drv32\idc.c)
	at offset 000000CC 00096H bytes from F:\src\os2\uniaud32t\drv32\bin\Release.ACP\dispatch.obj (F:\src\os2\uniaud32t\drv32\dispatch.c)
	at offset 00000162 0006AH bytes from F:\src\os2\uniaud32t\drv32\bin\Release.ACP\rmhelp.obj (F:\src\os2\uniaud32t\drv32\rmhelp.cpp)
	at offset 000001CC 00081H bytes from F:\src\os2\uniaud32t\drv32\bin\Release.ACP\irq.obj (F:\src\os2\uniaud32t\drv32\irq.cpp)
	at offset 00000250 00029H bytes from F:\src\os2\uniaud32t\lib\Release.ACP\linuxlib.lib (vsprintf.c)
	at offset 0000027C 00054H bytes from F:\src\os2\uniaud32t\lib\Release.ACP\linuxlib.lib (misc.c)
	at offset 000002D0 0005AH bytes from F:\src\os2\uniaud32t\lib\Release.ACP\linuxlib.lib (ossidc.cpp)
	at offset 0000032C 000BBH bytes from F:\src\os2\uniaud32t\lib\Release.ACP\linuxlib.lib (soundmidi.c)
	at offset 000003E8 0022FH bytes from F:\src\os2\uniaud32t\lib\Release.ACP\linuxlib.lib (soundmixer.c)
	at offset 00000618 0057FH bytes from F:\src\os2\uniaud32t\lib\Release.ACP\linuxlib.lib (sound.c)
	at offset 00000B98 0002EH bytes from F:\src\os2\uniaud32t\lib\Release.ACP\linuxlib.lib (debug.c)
	at offset 00000BC8 00098H bytes from F:\src\os2\uniaud32t\lib\Release.ACP\linuxlib.lib (ioctl.c)
	at offset 00000C60 0007BH bytes from F:\src\os2\uniaud32t\lib\Release.ACP\linuxlib.lib (irq.c)
	at offset 00000CDC 001C8H bytes from F:\src\os2\uniaud32t\lib\Release.ACP\linuxlib.lib (pci.c)
	at offset 00000EA4 000A1H bytes from F:\src\os2\uniaud32t\lib\Release.ACP\linuxlib.lib (malloc.cpp)
	at offset 00000F48 000E9H bytes from F:\src\os2\uniaud32t\lib\Release.ACP\core.lib (hwdep.c)
	at offset 00001034 00146H bytes from F:\src\os2\uniaud32t\lib\Release.ACP\core.lib (timer.c)
	at offset 0000117C 002DEH bytes from F:\src\os2\uniaud32t\lib\Release.ACP\core.lib (rawmidi.c)
	at offset 0000145C 00089H bytes from F:\src\os2\uniaud32t\lib\Release.ACP\core.lib (pcm_lib.c)
	at offset 000014E8 000CCH bytes from F:\src\os2\uniaud32t\lib\Release.ACP\core.lib (pcm.c)
	at offset 000015B4 000DEH bytes from F:\src\os2\uniaud32t\lib\Release.ACP\core.lib (sound.c)
	at offset 00001694 000B4H bytes from F:\src\os2\uniaud32t\lib\Release.ACP\core.lib (info.c)
	at offset 00001748 0006AH bytes from F:\src\os2\uniaud32t\lib\Release.ACP\core.lib (pcm_timer.c)
	at offset 000017B4 000A4H bytes from F:\src\os2\uniaud32t\lib\Release.ACP\core.lib (pcm_native.c)
	at offset 00001858 000F2H bytes from F:\src\os2\uniaud32t\lib\Release.ACP\core.lib (info_oss.c)
	at offset 0000194C 00068H bytes from F:\src\os2\uniaud32t\lib\Release.ACP\core.lib (sound_oss.c)
	at offset 000019B4 000BDH bytes from F:\src\os2\uniaud32t\lib\Release.ACP\core.lib (device.c)
	at offset 00001A74 000D9H bytes from F:\src\os2\uniaud32t\lib\Release.ACP\core.lib (control.c)
	at offset 00001B50 0005BH bytes from F:\src\os2\uniaud32t\lib\Release.ACP\core.lib (memalloc.c)
	at offset 00001BAC 0022FH bytes from F:\src\os2\uniaud32t\lib\Release.ACP\core.lib (init.c)
	at offset 00001DDC 00311H bytes from F:\src\os2\uniaud32t\lib\Release.ACP\pci.lib (bt87x.c)
	at offset 000020F0 00103H bytes from F:\src\os2\uniaud32t\lib\Release.ACP\pci.lib (als4000.c)
	at offset 000021F4 0055FH bytes from F:\src\os2\uniaud32t\lib\Release.ACP\pci.lib (cmipci.c)
	at offset 00002754 00228H bytes from F:\src\os2\uniaud32t\lib\Release.ACP\pci.lib (atiixp.c)
	at offset 0000297C 00260H bytes from F:\src\os2\uniaud32t\lib\Release.ACP\pci.lib (fm801.c)
	at offset 00002BDC 00473H bytes from F:\src\os2\uniaud32t\lib\Release.ACP\pci.lib (via82xx.c)
	at offset 00003050 001EAH bytes from F:\src\os2\uniaud32t\lib\Release.ACP\pci.lib (maestro3.c)
	at offset 0000323C 00A49H bytes from F:\src\os2\uniaud32t\lib\Release.ACP\pci.lib (intel8x0.c)
	at offset 00003C88 002FBH bytes from F:\src\os2\uniaud32t\lib\Release.ACP\pci.lib (es1968.c)
	at offset 00003F84 00428H bytes from F:\src\os2\uniaud32t\lib\Release.ACP\pci.lib (es1938.c)
	at offset 000043AC 002CBH bytes from F:\src\os2\uniaud32t\lib\Release.ACP\pci.lib (cs4281.c)
	at offset 00004678 00266H bytes from F:\src\os2\uniaud32t\lib\Release.ACP\pci.lib (ens1371.c)
	at offset 000048E0 002D4H bytes from F:\src\os2\uniaud32t\lib\Release.ACP\ca0106.lib (ca0106_main.c)
	at offset 00004BB4 00045H bytes from F:\src\os2\uniaud32t\lib\Release.ACP\ca0106.lib (ca_midi.c)
	at offset 00004BFC 00689H bytes from F:\src\os2\uniaud32t\lib\Release.ACP\ca0106.lib (ca0106_mixer.c)
	at offset 00005288 003CCH bytes from F:\src\os2\uniaud32t\lib\Release.ACP\ca0106.lib (ca0106_proc.c)
	at offset 00005654 003A0H bytes from F:\src\os2\uniaud32t\lib\Release.ACP\hda.lib (patch_via.c)
	at offset 000059F4 00438H bytes from F:\src\os2\uniaud32t\lib\Release.ACP\hda.lib (patch_conexant.c)
	at offset 00005E2C 00048H bytes from F:\src\os2\uniaud32t\lib\Release.ACP\hda.lib (patch_atihdmi.c)
	at offset 00005E74 00BB2H bytes from F:\src\os2\uniaud32t\lib\Release.ACP\hda.lib (patch_sigmatel.c)
	at offset 00006A28 0088FH bytes from F:\src\os2\uniaud32t\lib\Release.ACP\hda.lib (patch_analog.c)
	at offset 000072B8 0016AH bytes from F:\src\os2\uniaud32t\lib\Release.ACP\hda.lib (patch_cmedia.c)
	at offset 00007424 010F2H bytes from F:\src\os2\uniaud32t\lib\Release.ACP\hda.lib (patch_realtek.c)
	at offset 00008518 0071CH bytes from F:\src\os2\uniaud32t\lib\Release.ACP\hda.lib (hda_intel.c)
	at offset 00008C34 00826H bytes from F:\src\os2\uniaud32t\lib\Release.ACP\hda.lib (hda_codec.c)
	at offset 0000945C 0000DH bytes from F:\src\os2\uniaud32t\lib\Release.ACP\hda.lib (hda_hwdep.c)
	at offset 0000946C 001CAH bytes from F:\src\os2\uniaud32t\lib\Release.ACP\hda.lib (hda_generic.c)
	at offset 00009638 006EBH bytes from F:\src\os2\uniaud32t\lib\Release.ACP\hda.lib (hda_proc.c)
	at offset 00009D24 00163H bytes from F:\src\os2\uniaud32t\lib\Release.ACP\sequencer.lib (seq_device.c)
	at offset 00009E88 00015H bytes from F:\src\os2\uniaud32t\lib\Release.ACP\sequencer.lib (seq_info.c)
	at offset 00009EA0 00016H bytes from F:\src\os2\uniaud32t\lib\Release.ACP\sequencer.lib (seq_system.c)
	at offset 00009EB8 00156H bytes from F:\src\os2\uniaud32t\lib\Release.ACP\sequencer.lib (seq_queue.c)
	at offset 0000A010 0011AH bytes from F:\src\os2\uniaud32t\lib\Release.ACP\sequencer.lib (seq_memory.c)
	at offset 0000A12C 001FAH bytes from F:\src\os2\uniaud32t\lib\Release.ACP\sequencer.lib (seq_clientmgr.c)
	at offset 0000A328 00060H bytes from F:\src\os2\uniaud32t\lib\Release.ACP\sequencer.lib (seq_ports.c)
	at offset 0000A388 00127H bytes from F:\src\os2\uniaud32t\lib\Release.ACP\sequencer.lib (seq_timer.c)
	at offset 0000A4B0 000C3H bytes from F:\src\os2\uniaud32t\lib\Release.ACP\sequencer.lib (seq_prioq.c)
	at offset 0000A574 00027H bytes from F:\src\os2\uniaud32t\lib\Release.ACP\sequencer.lib (seq_fifo.c)
	at offset 0000A59C 00028H bytes from F:\src\os2\uniaud32t\lib\Release.ACP\opl3.lib (opl3_seq.c)
	at offset 0000A5C4 0014DH bytes from F:\src\os2\uniaud32t\lib\Release.ACP\opl3.lib (opl3_lib.c)
	at offset 0000A714 0000FH bytes from F:\src\os2\uniaud32t\lib\Release.ACP\opl3.lib (opl3_synth.c)
	at offset 0000A724 000E6H bytes from F:\src\os2\uniaud32t\lib\Release.ACP\mpu401.lib (mpu401_uart.c)
	at offset 0000A80C 00035H bytes from F:\src\os2\uniaud32t\lib\Release.ACP\cs46xx.lib (cs46xx.c)
	at offset 0000A844 00474H bytes from F:\src\os2\uniaud32t\lib\Release.ACP\cs46xx.lib (cs46xx_lib.c)
	at offset 0000ACB8 00129H bytes from F:\src\os2\uniaud32t\lib\Release.ACP\cs5535audio.lib (cs5535audio.c)
	at offset 0000ADE4 000C2H bytes from F:\src\os2\uniaud32t\lib\Release.ACP\cs5535audio.lib (cs5535audio_pm.c)
	at offset 0000AEA8 0005CH bytes from F:\src\os2\uniaud32t\lib\Release.ACP\cs5535audio.lib (cs5535audio_pcm.c)
	at offset 0000AF04 000BBH bytes from F:\src\os2\uniaud32t\lib\Release.ACP\emu10k1.lib (emu10k1.c)
	at offset 0000AFC0 00189H bytes from F:\src\os2\uniaud32t\lib\Release.ACP\emu10k1.lib (p16v.c)
	at offset 0000B14C 00016H bytes from F:\src\os2\uniaud32t\lib\Release.ACP\emu10k1.lib (timer.c)
	at offset 0000B164 00B47H bytes from F:\src\os2\uniaud32t\lib\Release.ACP\emu10k1.lib (emufx.c)
	at offset 0000BCAC 01089H bytes from F:\src\os2\uniaud32t\lib\Release.ACP\emu10k1.lib (emumixer.c)
	at offset 0000CD38 0009DH bytes from F:\src\os2\uniaud32t\lib\Release.ACP\emu10k1.lib (emupcm.c)
	at offset 0000CDD8 00082H bytes from F:\src\os2\uniaud32t\lib\Release.ACP\emu10k1.lib (emumpu401.c)
	at offset 0000CE5C 006A2H bytes from F:\src\os2\uniaud32t\lib\Release.ACP\emu10k1.lib (emu10k1_main.c)
	at offset 0000D500 00831H bytes from F:\src\os2\uniaud32t\lib\Release.ACP\emu10k1.lib (emuproc.c)
	at offset 0000DD34 0009CH bytes from F:\src\os2\uniaud32t\lib\Release.ACP\emu10k1.lib (io.c)
	at offset 0000DDD0 0008CH bytes from F:\src\os2\uniaud32t\lib\Release.ACP\emu10k1.lib (memory.c)
	at offset 0000DE5C 000C9H bytes from F:\src\os2\uniaud32t\lib\Release.ACP\emu10k1.lib (irq.c)
	at offset 0000DF28 00128H bytes from F:\src\os2\uniaud32t\lib\Release.ACP\ymfpci.lib (ymfpci.c)
	at offset 0000E050 00374H bytes from F:\src\os2\uniaud32t\lib\Release.ACP\ymfpci.lib (ymfpci_main.c)
	at offset 0000E3C4 00425H bytes from F:\src\os2\uniaud32t\lib\Release.ACP\ali5451.lib (ali5451.c)
	at offset 0000E7EC 00068H bytes from F:\src\os2\uniaud32t\lib\Release.ACP\trident.lib (trident.c)
	at offset 0000E854 00442H bytes from F:\src\os2\uniaud32t\lib\Release.ACP\trident.lib (trident_main.c)
	at offset 0000EC98 00035H bytes from F:\src\os2\uniaud32t\lib\Release.ACP\trident.lib (trident_memory.c)
	at offset 0000ECD0 003AFH bytes from F:\src\os2\uniaud32t\lib\Release.ACP\nm256.lib (nm256.c)
	at offset 0000F080 00374H bytes from F:\src\os2\uniaud32t\lib\Release.ACP\sb.lib (sb_mixer.c)
	at offset 0000F3F4 00127H bytes from F:\src\os2\uniaud32t\lib\Release.ACP\sb.lib (sb_common.c)
	at offset 0000F51C 00227H bytes from F:\src\os2\uniaud32t\lib\Release.ACP\core_oss.lib (pcm_oss.c)
	at offset 0000F744 00025H bytes from E:\watcom\lib386\os2\clib3r.lib (alphabet.c)
	at offset 0000F76C 0001AH bytes from F:\src\os2\uniaud32t\lib\Release.ACP\core.lib (vmaster.c)
	at offset 0000F788 0008CH bytes from F:\src\os2\uniaud32t\lib\Release.ACP\ac97.lib (ac97_pcm.c)
	at offset 0000F814 01DF2H bytes from F:\src\os2\uniaud32t\lib\Release.ACP\ac97.lib (ac97_codec.c)
	at offset 00011608 00BFFH bytes from F:\src\os2\uniaud32t\lib\Release.ACP\ac97.lib (ac97_proc.c)
	at offset 00012208 0004DH bytes from F:\src\os2\uniaud32t\lib\Release.ACP\sequencer.lib (seq_midi_emul.c)

 0005:00071D90 0000055D6H CONST2                 DATA 32-bit
	at offset 00000000 0017BH bytes from F:\src\os2\uniaud32t\drv32\bin\Release.ACP\init.obj (F:\src\os2\uniaud32t\drv32\init.c)
	at offset 0000017C 00040H bytes from F:\src\os2\uniaud32t\lib\Release.ACP\core.lib (info.c)
	at offset 000001BC 00004H bytes from F:\src\os2\uniaud32t\lib\Release.ACP\core.lib (pcm_memory.c)
	at offset 000001C0 0000CH bytes from F:\src\os2\uniaud32t\lib\Release.ACP\core.lib (pcm_native.c)
	at offset 000001CC 00028H bytes from F:\src\os2\uniaud32t\lib\Release.ACP\pci.lib (als4000.c)
	at offset 000001F4 00020H bytes from F:\src\os2\uniaud32t\lib\Release.ACP\pci.lib (cmipci.c)
	at offset 00000214 00010H bytes from F:\src\os2\uniaud32t\lib\Release.ACP\pci.lib (fm801.c)
	at offset 00000224 00010H bytes from F:\src\os2\uniaud32t\lib\Release.ACP\pci.lib (via82xx.c)
	at offset 00000234 000BCH bytes from F:\src\os2\uniaud32t\lib\Release.ACP\pci.lib (maestro3.c)
	at offset 000002F0 00010H bytes from F:\src\os2\uniaud32t\lib\Release.ACP\pci.lib (es1938.c)
	at offset 00000300 00010H bytes from F:\src\os2\uniaud32t\lib\Release.ACP\pci.lib (cs4281.c)
	at offset 00000310 00010H bytes from F:\src\os2\uniaud32t\lib\Release.ACP\pci.lib (ens1371.c)
	at offset 00000320 00020H bytes from F:\src\os2\uniaud32t\lib\Release.ACP\ca0106.lib (ca0106_main.c)
	at offset 00000340 00020H bytes from F:\src\os2\uniaud32t\lib\Release.ACP\ca0106.lib (ca0106_mixer.c)
	at offset 00000360 00084H bytes from F:\src\os2\uniaud32t\lib\Release.ACP\hda.lib (patch_conexant.c)
	at offset 000003E4 00010H bytes from F:\src\os2\uniaud32t\lib\Release.ACP\emu10k1.lib (p16v.c)
	at offset 000003F4 00814H bytes from F:\src\os2\uniaud32t\lib\Release.ACP\emu10k1.lib (emufx.c)
	at offset 00000C08 00010H bytes from F:\src\os2\uniaud32t\lib\Release.ACP\emu10k1.lib (emumixer.c)
	at offset 00000C18 00010H bytes from F:\src\os2\uniaud32t\lib\Release.ACP\ymfpci.lib (ymfpci_main.c)
	at offset 00000C28 00020H bytes from F:\src\os2\uniaud32t\lib\Release.ACP\trident.lib (trident_main.c)
	at offset 00000C48 00018H bytes from F:\src\os2\uniaud32t\lib\Release.ACP\ac97.lib (ac97_pcm.c)
	at offset 00000C60 04976H bytes from F:\src\os2\uniaud32t\lib\Release.ACP\ac97.lib (ac97_codec.c)

 0005:00077368 000000004H LASTDATA32             DATA 32-bit
	at offset 00000000 00004H bytes from F:\src\os2\uniaud32t\drv32\bin\Release.ACP\end.obj (end.asm)

 0005:0007736C 000000000H XIB                    DATA 32-bit

 0005:0007736C 000000006H XI                     DATA 32-bit
	at offset 00000000 00006H bytes from E:\watcom\lib386\os2\clib3r.lib (mbislead.c)

 0005:00077372 000000000H XIE                    DATA 32-bit

 0005:00077372 000000000H TIB                    DATA 32-bit

 0005:00077372 000000000H TI                     DATA 32-bit

 0005:00077372 000000000H TIE                    DATA 32-bit

 0005:00077372 000000000H YIB                    DATA 32-bit

 0005:00077372 000000000H YI                     DATA 32-bit

 0005:00077372 000000000H YIE                    DATA 32-bit

 0005:00077372 000000000H DATA                   DATA 32-bit

 0005:00077374 000000000H CONST32                CONST 32-bit

 0005:00077374 000000045H CONST32_RO             CONST 32-bit
	at offset 00000000 00045H bytes from F:\acpi\lib\acpidrv.lib (acpi)

 0005:000773C0 000000004H _NULL                  BEGDATA 32-bit
	at offset 00000000 00004H bytes from E:\watcom\lib386\os2\clib3r.lib (segdefns)

 0005:000773C4 000000000H _AFTERNULL             BEGDATA 32-bit

 0005:000773D0 000010000H STACK                  STACK 32-bit
	at offset 00000000 10000H bytes from E:\watcom\lib386\os2\clib3r.lib (segdefns)


 Origin   Group
 0000:0   FLAT
 0003:0   CGROUP
 0005:0   DGROUP


 Address         Publics by Name
 0003:0007E020       ACPIFindPCIDevice
 0003:00008F0B       AddBaseAddress_
 0003:00005343       add_timer_
 0003:0000CF3A       add_wait_queue_
 0003:0000CF3B       add_wait_queue_exclusive_
 0003:000097B5       alloc_pages_
 0003:00007421       ALSAToOSSDataType_
 0003:0000749F       ALSAToOSSRateFlags_
 0003:00004D0D       ALSA_FreeIrq_
 0003:00003652       ALSA_IDC
 0003:00004D2B       ALSA_Interrupt
 0003:00004C78       ALSA_SetIrq_
 0003:00000557       ALSA_STRATEGY
 0003:0000527F       ALSA_TIMER_
 0005:00001758       BootCode
 0003:000356A5       ca_midi_init_
 0003:00008B6F       CharOut_
 0003:0005374A       client_init_data_
 0003:00006191       ConvertVolume_
 0003:000098B4       copy_from_user_
 0003:0007EA5A       copy_from_user_toio_
 0003:00009854       copy_to_user_
 0003:0007E9EC       copy_to_user_fromio_
 0003:000054D7       create_proc_entry_
 0003:00005649       create_workqueue_
 0003:00008ECA       DbgPrintIrq_
 0003:000089AF       DecLongToASCII_
 0003:00005344       del_timer_
 0003:00005695       destroy_workqueue_
 0005:000017F4       DevHelp32
 0001:0000003C       DevHelpInit
 0003:00000010       DevHlp
 0003:00000030       DevHlp_ModifiedDS
 0003:00005524       disable_dma_
 0003:0000AEAB       disable_irq_
 0000:00000000  Imp  DOS32FLATDS          (DOSCALLS.370)
 0000:00000000  Imp  DOSCLOSE             (DOSCALLS.59)
 0000:00000000  Imp  DosExit              (DOSCALLS.234)
 0000:00000000  Imp  DOSIODELAYCNT        (DOSCALLS.427)
 0000:00000000  Imp  DOSOPEN              (DOSCALLS.70)
 0000:00000000  Imp  DosQueryCp           (DOSCALLS.291)
 0000:00000000  Imp  DosQueryDBCSEnv      (NLS.6)
 0000:00000000  Imp  DosQuerySysInfo      (DOSCALLS.348)
 0000:00000000  Imp  DosWrite             (DOSCALLS.282)
 0000:00000000  Imp  DOSWRITE             (DOSCALLS.138)
 0003:0007E41E       down_
 0003:0007E420       down_interruptible_
 0003:00005307       do_gettimeofday_
 0003:00019E19       dummy_get_unmapped_area_
 0003:00005523       enable_dma_
 0003:0000ADD7       eoi_irq_
 0003:0000551B       fasync_helper_
 0001:00000465       FileName
 0003:0000A120       FillCaps_
 0003:0007E1B0       FindAddress
 0003:000055FA       flush_workqueue_
 0001:00000040       fOpen
 0003:00005522       free_dma_
 0003:0000AD3E       free_irq_
 0003:00009695       free_pages_
 0003:00008F3F       GetBaseAddress_
 0003:00009DAB       GetMaxChannels_
 0003:00009CF6       GetNumberOfCards_
 0003:00009CFC       GetNumberOfPcm_
 0003:0000281A       GetParms_
 0003:00009D20       GetPcmForChannels_
 0003:00003510       GetTKSSBase
 0003:0000A343       GetUniaudCardInfo_
 0003:0000A6BA       GetUniaudControlInfo_
 0003:0000A41F       GetUniaudControlNum_
 0003:0000A552       GetUniaudControls_
 0003:0000A79B       GetUniaudControlValueGet_
 0003:0000A880       GetUniaudControlValuePut_
 0003:00009E27       GetUniaudPcmCaps1_
 0003:0000A172       GetUniaudPcmCaps_
 0001:00000000       help_header
 0002:00000000       help_stub_strategy
 0003:00008A91       HexLongToASCII_
 0003:0000547B       hweight32_
 0003:000000E0       IDC_
 0003:0007E0C2       InitACPICall
 0001:00000046       InitPktOff
 0001:00000044       InitPktSeg
 0003:0007E41C       init_MUTEX_
 0003:0007E41D       init_MUTEX_LOCKED_
 0003:0000CF45       init_waitqueue_entry_
 0003:0000CF39       init_waitqueue_head_
 0003:0000CF43       interruptible_sleep_on_
 0003:0000CF3D       interruptible_sleep_on_timeout_
 0005:000017F8       intSwitchStack
 0003:0000AEA5       in_interrupt_
 0003:00003550       iodelay32_
 0003:0003372E       ioport_map_
 0003:0003373E       ioport_unmap_
 0003:000336C0       ioread16_
 0003:000336DD       ioread32_
 0003:000336A5       ioread8_
 0003:00009812       iounmap_
 0003:00033706       iowrite16_
 0003:0003371B       iowrite32_
 0003:000336F3       iowrite8_
 0003:00009825       is_access_ok_
 0003:0008A550       itoa_
 0003:00009B2E       kcalloc_
 0000:00000000  Imp  KernLinToPageList    (KEE.64)
 0000:00000000  Imp  KernSelToFlat        (KEE.66)
 0000:00000000  Imp  KernThunkStackTo16   (KEE.40)
 0000:00000000  Imp  KernThunkStackTo32   (KEE.41)
 0000:00000000  Imp  KernVMAlloc          (KEE.60)
 0000:00000000  Imp  KernVMFree           (KEE.61)
 0000:00000000  Imp  KernVMLock           (KEE.62)
 0003:0000551E       kill_fasync_
 0003:0000569A       kstrdup_
 0003:00009A3A       kzalloc_
 0003:0008A4D0       lltoa_
 0003:0008A430       ltoa_
 0003:0008A300       mbtowc_
 0003:000052DE       mdelay_
 0003:000057A9       memdup_user_
 0003:00088530       memmove_
 0003:00088510       memset_
 0003:000056D5       mod_firmware_load_
 0003:00005347       mod_timer_
 0003:00005348       msleep_
 0003:00005B08       MyDevBlock_
 0002:000003DA       MY_DEVHELP_ATTACHDD
 0003:00004D93       os2gettimemsec_
 0003:00004D8D       os2gettimesec_
 0003:0000C812       OSS32_APMResume_
 0003:0000C861       OSS32_APMSuspend_
 0003:00005ACD       OSS32_CloseUNI16_
 0003:00005B37       OSS32_DebugString_
 0003:00005821       OSS32_Initialize_
 0003:00005ECB       OSS32_MidiClose_
 0003:0000606A       OSS32_MidiCommand_
 0003:00005B5E       OSS32_MidiOpen_
 0003:00006046       OSS32_MidiQueryCaps_
 0003:00005FF7       OSS32_MidiRead_
 0003:00005FF1       OSS32_MidiWrite_
 0003:000066B0       OSS32_MixClose_
 0003:00006DA2       OSS32_MixGetProperty_
 0003:00006706       OSS32_MixGetVolume_
 0003:000061B5       OSS32_MixOpen_
 0003:00006EA5       OSS32_MixQueryCaps_
 0003:00006F3A       OSS32_MixQueryName_
 0003:00006A75       OSS32_MixSetProperty_
 0003:00006761       OSS32_MixSetVolume_
 0003:00005A58       OSS32_ProcessIRQ_
 0003:00005A93       OSS32_ProcessMIDIIRQ_
 0003:00007575       OSS32_QueryDevCaps_
 0003:0000702C       OSS32_QueryNames_
 0003:000053EF       OSS32_SetFileId_
 0003:000059C5       OSS32_Shutdown_
 0003:000085A0       OSS32_WaveAddBuffer_
 0003:00007AAC       OSS32_WaveClose_
 0003:0000888D       OSS32_WaveGetHwPtr_
 0003:000087C1       OSS32_WaveGetPosition_
 0003:00008827       OSS32_WaveGetSpace_
 0003:000088F3       OSS32_WaveGetStatus_
 0003:000078E6       OSS32_WaveOpen_
 0003:00007C89       OSS32_WavePause_
 0003:00007B7A       OSS32_WavePrepare_
 0003:00007CDF       OSS32_WaveResume_
 0003:00007D38       OSS32_WaveSetHwParams_
 0003:0000894E       OSS32_WaveSetVolume_
 0003:00007BDD       OSS32_WaveStart_
 0003:00007C33       OSS32_WaveStop_
 0003:00006DC1       OSSToALSAVolume_
 0003:0000C8B7       PciAdjustInterrupts_
 0003:0000B5B7       pcibios_present_
 0003:0000B021       pcidev_activate_
 0003:0000B027       pcidev_deactivate_
 0003:0000B01B       pcidev_prepare_
 0003:0000BA5F       pci_alloc_consistent_
 0003:0000BC90       pci_disable_device_
 0003:0000B5E2       pci_dma_supported_
 0003:0000B7FA       pci_enable_device_
 0003:0000B5F7       pci_find_capability_
 0003:0000B455       pci_find_device_
 0003:0000B5CE       pci_find_slot_
 0003:0000BB1B       pci_free_consistent_
 0003:0000BB41       pci_get_dma_mask_
 0003:0000BB36       pci_get_driver_data_
 0003:0000B591       pci_get_flags_
 0003:0003373F       pci_iomap_
 0003:000338CA       pci_iounmap_
 0003:0000C706       pci_match_device_
 0003:0000B96B       pci_module_init_
 0003:0000BB8E       pci_orig_restore_state_
 0003:0000BB62       pci_orig_save_state_
 0003:0000AEAC       pci_read_config_byte_
 0003:0000AF2E       pci_read_config_dword_
 0003:0000AEEC       pci_read_config_word_
 0003:0000B838       pci_register_driver_
 0003:0000C6EC       pci_release_regions_
 0003:0000C382       pci_release_region_
 0003:0000C6B1       pci_request_regions_
 0003:0000BCCC       pci_request_region_
 0003:0000BC3C       pci_restore_state_
 0003:0000BBF1       pci_save_state_
 0003:0000BB2B       pci_set_driver_data_
 0003:0000BB4F       pci_set_latency_time_
 0003:0000BA0A       pci_set_master_
 0003:0000B686       pci_set_power_state_
 0003:0000B97A       pci_unregister_driver_
 0003:0000AF65       pci_write_config_byte_
 0003:0000AFE6       pci_write_config_dword_
 0003:0000AFA5       pci_write_config_word_
 0003:00014F8B       pcm_info_
 0003:00015027       pcm_instances_
 0005:00001778       PDDName
 0001:0000045E       pddname16
 0003:0000903E       phys_to_virt_
 0003:0000BA46       pm_register_
 0003:0000BA49       pm_unregister_
 0003:00005477       poll_wait_
 0003:0000ADE4       process_interrupt_
 0003:00005515       proc_register_
 0003:00005518       proc_unregister_
 0003:0004C7C3       query_amp_caps_
 0003:00052600       queueptr_
 0003:00005566       queue_work_
 0003:000071A1       register_chrdev_
 0003:00005525       register_reboot_notifier_
 0003:00007271       register_sound_dsp_
 0003:0000723C       register_sound_midi_
 0003:00007207       register_sound_mixer_
 0003:000071D2       register_sound_special_
 0003:000072A3       register_sound_synth_
 0003:0007E997       release_and_free_resource_
 0003:00005791       release_firmware_
 0003:0000BB4C       release_resource_
 0003:000097B8       remap_page_range_
 0003:00005514       remove_proc_entry_
 0003:0000CF3C       remove_wait_queue_
 0003:0000551F       request_dma_
 0003:00005712       request_firmware_
 0003:0000AC1A       request_irq_
 0005:0000177C       RMAllocResource1632
 0005:0000179C       RMCreateAdapter1632
 0005:00001794       RMCreateDevice1632
 0005:000017A4       RMCreateDriver1632
 0003:00004887       RMDeallocateIRQ_
 0005:0000178C       RMDeallocResource1632
 0005:000017AC       RMDestroyDriver1632
 0005:000017BC       RMDevIDToHandleList1632
 0003:000048AE       RMDone_
 0005:000017B4       RMGetNodeInfo1632
 0005:000017C4       RMHandleToResourceHandleList1632
 0003:00004510       RMInit_
 0005:00001784       RMModifyResources1632
 0003:00004687       RMRequestIO_
 0003:000047C0       RMRequestIRQ_
 0003:0000472B       RMRequestMem_
 0003:00004C6C       RMSetHandles_
 0003:00005476       schedule_
 0003:000052BB       schedule_timeout_
 0003:00009D01       SetPCMInstance_
 0003:000850F4       snd_ac97_bus_
 0003:0008756B       snd_ac97_bus_proc_done_
 0003:00087510       snd_ac97_bus_proc_init_
 0003:00084E7E       snd_ac97_get_name_
 0003:00085011       snd_ac97_get_short_name_
 0003:00085177       snd_ac97_mixer_
 0003:0007F08E       snd_ac97_pcm_assign_
 0003:0007F695       snd_ac97_pcm_close_
 0003:0007F75D       snd_ac97_pcm_double_rate_rules_
 0003:0007F409       snd_ac97_pcm_open_
 0003:000874ED       snd_ac97_proc_done_
 0003:00087409       snd_ac97_proc_init_
 0003:00082D27       snd_ac97_read_
 0003:00085CF8       snd_ac97_resume_
 0003:0007ECD0       snd_ac97_set_rate_
 0003:00085BF5       snd_ac97_suspend_
 0003:00086463       snd_ac97_tune_hardware_
 0003:00082DF7       snd_ac97_update_
 0003:00082E77       snd_ac97_update_bits_
 0003:00082EC1       snd_ac97_update_bits_nolock_
 0003:00082CCA       snd_ac97_write_
 0003:00082DA1       snd_ac97_write_cache_
 0003:000152AB       snd_add_device_sysfs_file_
 0003:0004F320       snd_array_free_
 0003:0004F2A2       snd_array_new_
 0003:00033A34       snd_ca0106_i2c_write_
 0003:0003609E       snd_ca0106_mixer_
 0003:00036276       snd_ca0106_mixer_resume_
 0003:0003623D       snd_ca0106_mixer_suspend_
 0003:00036AC9       snd_ca0106_proc_init_
 0003:000338EE       snd_ca0106_ptr_read_
 0003:00033928       snd_ca0106_ptr_write_
 0003:00033962       snd_ca0106_spi_write_
 0003:0001C542       snd_card_create_
 0003:0001C87E       snd_card_disconnect_
 0003:0001CF4F       snd_card_file_add_
 0003:0001CFC3       snd_card_file_remove_
 0003:0001CA7D       snd_card_free_
 0003:0001CA2D       snd_card_free_when_closed_
 0003:0001CE72       snd_card_info_done_
 0003:0001CDF4       snd_card_info_init_
 0003:0001CD6B       snd_card_info_read_oss_
 0003:0001C7A7       snd_card_locked_
 0003:00015F97       snd_card_proc_new_
 0003:0001CC8D       snd_card_register_
 0003:0001CC67       snd_card_set_id_
 0003:0001CE89       snd_component_add_
 0003:0005C6D3       snd_cs46xx_create_
 0003:0005A998       snd_cs46xx_download_
 0003:0005A9D1       snd_cs46xx_download_image_
 0003:0005BE8C       snd_cs46xx_gameport_
 0003:0005BDD5       snd_cs46xx_midi_
 0003:0005B9CE       snd_cs46xx_mixer_
 0003:0005B75B       snd_cs46xx_pcm_
 0003:0005C5CE       snd_cs46xx_resume_
 0003:0005C27C       snd_cs46xx_start_dsp_
 0003:0005C50F       snd_cs46xx_suspend_
 0003:0005D679       snd_cs5535audio_pcm_
 0003:0005D13B       snd_cs5535audio_resume_
 0003:0005D097       snd_cs5535audio_suspend_
 0003:0001AAED       snd_ctl_add_
 0003:0001C0C4       snd_ctl_boolean_mono_info_
 0003:0001C0E3       snd_ctl_boolean_stereo_info_
 0003:0001C0AC       snd_ctl_create_
 0003:0001ADB1       snd_ctl_find_id_
 0003:0001AD84       snd_ctl_find_numid_
 0003:0001AA24       snd_ctl_free_one_
 0003:0007E8D5       snd_ctl_make_virtual_master_
 0003:0001A953       snd_ctl_new1_
 0003:0001A7EA       snd_ctl_notify_
 0003:0001BF46       snd_ctl_register_ioctl_
 0003:0001AC00       snd_ctl_remove_
 0003:0001AC6B       snd_ctl_remove_id_
 0003:0001AD28       snd_ctl_rename_id_
 0003:0001BFA0       snd_ctl_unregister_ioctl_
 0003:0001A443       snd_device_disconnect_
 0003:0001A545       snd_device_disconnect_all_
 0003:0001A3AC       snd_device_free_
 0003:0001A57D       snd_device_free_all_
 0003:0001A359       snd_device_new_
 0003:0001A4AD       snd_device_register_
 0003:0001A507       snd_device_register_all_
 0003:0001C1EA       snd_dma_alloc_pages_
 0003:0001C279       snd_dma_alloc_pages_fallback_
 0003:0001C2D9       snd_dma_free_pages_
 0003:0001C32C       snd_dma_get_reserved_buf_
 0003:0001C3DD       snd_dma_reserve_buf_
 0003:0006DAB7       snd_emu1010_fpga_link_dst_src_write_
 0003:0006DA40       snd_emu1010_fpga_read_
 0003:0006D9B5       snd_emu1010_fpga_write_
 0003:0006DEFE       snd_emu10k1_ac97_read_
 0003:0006DF40       snd_emu10k1_ac97_write_
 0003:0006E5B3       snd_emu10k1_alloc_pages_
 0003:0006AB7A       snd_emu10k1_audigy_midi_
 0003:0006C2CB       snd_emu10k1_create_
 0003:0006B384       snd_emu10k1_done_
 0003:00065B3E       snd_emu10k1_efx_alloc_pm_buffer_
 0003:00065BE5       snd_emu10k1_efx_free_pm_buffer_
 0003:0005EE2C       snd_emu10k1_efx_read_
 0003:00065D39       snd_emu10k1_efx_resume_
 0003:00065C16       snd_emu10k1_efx_suspend_
 0003:000652C9       snd_emu10k1_free_efx_
 0003:0006E6A4       snd_emu10k1_free_pages_
 0003:00065A8D       snd_emu10k1_fx8010_new_
 0003:0005EC32       snd_emu10k1_fx8010_register_irq_handler_
 0003:00065303       snd_emu10k1_fx8010_tram_setup_
 0003:0005ECD3       snd_emu10k1_fx8010_unregister_irq_handler_
 0003:0006D8AA       snd_emu10k1_i2c_write_
 0003:00065291       snd_emu10k1_init_efx_
 0003:0006EA50       snd_emu10k1_interrupt_
 0003:0006DB44       snd_emu10k1_intr_disable_
 0003:0006DB0B       snd_emu10k1_intr_enable_
 0003:0006E513       snd_emu10k1_memblk_map_
 0003:0006AB2D       snd_emu10k1_midi_
 0003:000674D8       snd_emu10k1_mixer_
 0003:00069A85       snd_emu10k1_pcm_
 0003:0006A41E       snd_emu10k1_pcm_efx_
 0003:00069C82       snd_emu10k1_pcm_mic_
 0003:00069BA5       snd_emu10k1_pcm_multi_
 0003:0006D37D       snd_emu10k1_proc_init_
 0003:0006D734       snd_emu10k1_ptr20_read_
 0003:0006D774       snd_emu10k1_ptr20_write_
 0003:0006D5A4       snd_emu10k1_ptr_read_
 0003:0006D660       snd_emu10k1_ptr_write_
 0003:0006DF82       snd_emu10k1_rate_to_pitch_
 0003:0006C956       snd_emu10k1_resume_init_
 0003:0006C9BA       snd_emu10k1_resume_regs_
 0003:0006D7B4       snd_emu10k1_spi_write_
 0003:0006C8C7       snd_emu10k1_suspend_regs_
 0003:0006E6A9       snd_emu10k1_synth_alloc_
 0003:0006E94E       snd_emu10k1_synth_bzero_
 0003:0006E9C2       snd_emu10k1_synth_copy_from_user_
 0003:0006E709       snd_emu10k1_synth_free_
 0003:0005E8B1       snd_emu10k1_timer_
 0003:0006E15E       snd_emu10k1_voice_alloc_
 0003:0006DE3C       snd_emu10k1_voice_clear_loop_stop_
 0003:0006E1F1       snd_emu10k1_voice_free_
 0003:0006DD77       snd_emu10k1_voice_half_loop_intr_ack_
 0003:0006DD10       snd_emu10k1_voice_half_loop_intr_disable_
 0003:0006DCAB       snd_emu10k1_voice_half_loop_intr_enable_
 0003:0006AC12       snd_emu10k1_voice_init_
 0003:0006DC4B       snd_emu10k1_voice_intr_ack_
 0003:0006DBE4       snd_emu10k1_voice_intr_disable_
 0003:0006DB7F       snd_emu10k1_voice_intr_enable_
 0003:0006DDD7       snd_emu10k1_voice_set_loop_stop_
 0003:0006DEA3       snd_emu10k1_wait_
 0003:0001C1B5       snd_free_dev_pages_
 0003:0001C14E       snd_free_pages_
 0003:0001D136       snd_free_sgbuf_pages_
 0003:0004B78D       snd_hda_add_codec_preset_
 0003:0004E58F       snd_hda_add_new_ctls_
 0003:0004C1B3       snd_hda_add_pincfg_
 0003:0004D143       snd_hda_add_vmaster_
 0003:0004DD70       snd_hda_build_controls_
 0003:0004E4A7       snd_hda_build_pcms_
 0003:0004BD28       snd_hda_bus_new_
 0003:0004DE01       snd_hda_calc_stream_format_
 0003:0004E549       snd_hda_check_board_codec_sid_config_
 0003:0004E4CE       snd_hda_check_board_config_
 0003:0004E623       snd_hda_ch_mode_get_
 0003:0004E5EC       snd_hda_ch_mode_info_
 0003:0004E647       snd_hda_ch_mode_put_
 0003:0004C9AB       snd_hda_codec_amp_read_
 0003:0004CA92       snd_hda_codec_amp_stereo_
 0003:0004C9EB       snd_hda_codec_amp_update_
 0003:0004DDCD       snd_hda_codec_build_controls_
 0003:0004E3F4       snd_hda_codec_build_pcms_
 0003:0004C6EE       snd_hda_codec_cleanup_stream_
 0003:0004C5E3       snd_hda_codec_configure_
 0003:0004C237       snd_hda_codec_get_pincfg_
 0003:0004C36E       snd_hda_codec_new_
 0003:00051988       snd_hda_codec_proc_new_
 0003:0004B95B       snd_hda_codec_read_
 0003:0004CFEA       snd_hda_codec_reset_
 0003:0004CADD       snd_hda_codec_resume_amp_
 0003:0004DB2A       snd_hda_codec_resume_cache_
 0003:0004C6A8       snd_hda_codec_setup_stream_
 0003:0004C222       snd_hda_codec_set_pincfg_
 0003:0004B988       snd_hda_codec_write_
 0003:0004DAB4       snd_hda_codec_write_cache_
 0003:0004F57A       snd_hda_create_hwdep_
 0003:0004DA13       snd_hda_create_spdif_in_ctls_
 0003:0004D856       snd_hda_create_spdif_out_ctls_
 0003:0004D930       snd_hda_create_spdif_share_sw_
 0003:0004CF55       snd_hda_ctls_clear_
 0003:0004CF27       snd_hda_ctl_add_
 0003:0004B7BD       snd_hda_delete_codec_preset_
 0003:0004CF1D       snd_hda_find_mixer_ctl_
 0003:0004BA26       snd_hda_get_connections_
 0003:0004B82E       snd_hda_get_jack_connectivity_
 0003:0004B7E5       snd_hda_get_jack_location_
 0003:0004B83C       snd_hda_get_jack_type_
 0003:0004B9EE       snd_hda_get_sub_nodes_
 0003:0004E690       snd_hda_input_mux_info_
 0003:0004E6DF       snd_hda_input_mux_put_
 0003:0004E154       snd_hda_is_supported_format_
 0003:0004D1FD       snd_hda_mixer_amp_switch_get_
 0003:0004D1CD       snd_hda_mixer_amp_switch_info_
 0003:0004D294       snd_hda_mixer_amp_switch_put_
 0003:0004CDBE       snd_hda_mixer_amp_tlv_
 0003:0004CC75       snd_hda_mixer_amp_volume_get_
 0003:0004CB90       snd_hda_mixer_amp_volume_info_
 0003:0004CD0F       snd_hda_mixer_amp_volume_put_
 0003:0004D463       snd_hda_mixer_bind_ctls_get_
 0003:0004D42B       snd_hda_mixer_bind_ctls_info_
 0003:0004D49C       snd_hda_mixer_bind_ctls_put_
 0003:0004D34F       snd_hda_mixer_bind_switch_get_
 0003:0004D38A       snd_hda_mixer_bind_switch_put_
 0003:0004D50A       snd_hda_mixer_bind_tlv_
 0003:0004EB85       snd_hda_multi_out_analog_cleanup_
 0003:0004E8D5       snd_hda_multi_out_analog_open_
 0003:0004E9E9       snd_hda_multi_out_analog_prepare_
 0003:0004E885       snd_hda_multi_out_dig_cleanup_
 0003:0004E8B3       snd_hda_multi_out_dig_close_
 0003:0004E81B       snd_hda_multi_out_dig_open_
 0003:0004E855       snd_hda_multi_out_dig_prepare_
 0003:0004C834       snd_hda_override_amp_caps_
 0003:00050862       snd_hda_parse_generic_codec_
 0003:0004ECC8       snd_hda_parse_pin_def_config_
 0003:0004C8B1       snd_hda_query_pin_caps_
 0003:0004BC45       snd_hda_queue_unsol_event_
 0003:0004F27F       snd_hda_resume_
 0003:0004B9C1       snd_hda_sequence_write_
 0003:0004DB77       snd_hda_sequence_write_cache_
 0003:0004CE81       snd_hda_set_vmaster_tlv_
 0003:0004F25C       snd_hda_suspend_
 0003:0000D524       snd_hwdep_new_
 0003:00015C54       snd_info_card_create_
 0003:00015D0E       snd_info_card_disconnect_
 0003:00015D62       snd_info_card_free_
 0003:00015CCF       snd_info_card_id_change_
 0003:00015CB6       snd_info_card_register_
 0003:000154A5       snd_info_check_reserved_words_
 0003:00015F06       snd_info_create_card_entry_
 0003:00015EEC       snd_info_create_module_entry_
 0003:00015C06       snd_info_done_
 0003:00015FEF       snd_info_free_entry_
 0003:00015D82       snd_info_get_line_
 0003:00015E0D       snd_info_get_str_
 0003:00015B6A       snd_info_init_
 0003:00019FC4       snd_info_minor_register_
 0003:0001A018       snd_info_minor_unregister_
 0003:00016032       snd_info_register_
 0003:00012A7A       snd_interval_div_
 0003:000130C6       snd_interval_list_
 0003:00012B33       snd_interval_muldivk_
 0003:00012BE2       snd_interval_mulkdiv_
 0003:000129DC       snd_interval_mul_
 0003:00012CA4       snd_interval_ratnum_
 0003:00012886       snd_interval_refine_
 0003:00008CF8       snd_iprintf_
 0003:0001508D       snd_lookup_minor_data_
 0003:0001A02A       snd_lookup_oss_minor_data_
 0003:0001C178       snd_malloc_dev_pages_
 0003:0001C122       snd_malloc_pages_
 0003:0001D17C       snd_malloc_sgbuf_pages_
 0003:0008800F       snd_midi_channel_alloc_set_
 0003:00088066       snd_midi_channel_free_set_
 0003:00087B67       snd_midi_channel_set_clear_
 0003:0008757F       snd_midi_process_event_
 0003:000153E6       snd_minor_info_done_
 0003:000153A5       snd_minor_info_init_
 0003:0001A341       snd_minor_info_oss_done_
 0003:0001A2FE       snd_minor_info_oss_init_
 0003:00059AC8       snd_mpu401_uart_interrupt_
 0003:00059ADA       snd_mpu401_uart_interrupt_tx_
 0003:0005A05C       snd_mpu401_uart_new_
 0003:00058608       snd_opl3_calc_volume_
 0003:000595D6       snd_opl3_clear_patches_
 0003:0005918B       snd_opl3_control_
 0003:00057FDE       snd_opl3_create_
 0003:0005855B       snd_opl3_drum_switch_
 0003:00059561       snd_opl3_find_patch_
 0003:00058164       snd_opl3_hwdep_new_
 0003:00057F6D       snd_opl3_init_
 0003:00057E77       snd_opl3_interrupt_
 0003:000591F7       snd_opl3_ioctl_
 0003:0005905C       snd_opl3_key_press_
 0003:000584EA       snd_opl3_load_drums_
 0003:00059477       snd_opl3_load_patch_
 0003:00057EEA       snd_opl3_new_
 0003:00058FBC       snd_opl3_note_off_
 0003:00058941       snd_opl3_note_on_
 0003:000591F0       snd_opl3_nrpn_
 0003:000591F4       snd_opl3_open_
 0003:00059373       snd_opl3_release_
 0003:00059614       snd_opl3_reset_
 0003:00057751       snd_opl3_synth_cleanup_
 0003:000576A7       snd_opl3_synth_setup_
 0003:000576A6       snd_opl3_synth_use_dec_
 0003:0005768A       snd_opl3_synth_use_inc_
 0003:000591F1       snd_opl3_sysex_
 0003:0005905D       snd_opl3_terminate_note_
 0003:00058851       snd_opl3_timer_func_
 0003:00058127       snd_opl3_timer_new_
 0003:00059381       snd_opl3_write_
 0003:00019E1E       snd_oss_info_register_
 0003:0005E775       snd_p16v_alloc_pm_buffer_
 0003:0005E350       snd_p16v_free_
 0003:0005E797       snd_p16v_free_pm_buffer_
 0003:0005E736       snd_p16v_mixer_
 0003:0005E361       snd_p16v_pcm_
 0003:0005E7D4       snd_p16v_resume_
 0003:0005E7A2       snd_p16v_suspend_
 0003:0000C805       snd_pci_compat_get_pci_driver_
 0003:0000C7AA       snd_pci_dev_present_
 0003:0007E9AC       snd_pci_quirk_lookup_
 0003:00014988       snd_pcm_attach_substream_
 0003:00014BE0       snd_pcm_detach_substream_
 0003:00017901       snd_pcm_drain_done_
 0003:00011A80       snd_pcm_format_big_endian_
 0003:00011A48       snd_pcm_format_linear_
 0003:00011A58       snd_pcm_format_little_endian_
 0003:00011ABB       snd_pcm_format_physical_width_
 0003:00011B24       snd_pcm_format_set_silence_
 0003:00011A0D       snd_pcm_format_signed_
 0003:00011AF9       snd_pcm_format_silence_64_
 0003:00011AE3       snd_pcm_format_size_
 0003:00011A35       snd_pcm_format_unsigned_
 0003:00011A93       snd_pcm_format_width_
 0003:00018AA9       snd_pcm_hw_constraints_complete_
 0003:00018766       snd_pcm_hw_constraints_init_
 0003:0001334E       snd_pcm_hw_constraint_integer_
 0003:000133D9       snd_pcm_hw_constraint_list_
 0003:00013301       snd_pcm_hw_constraint_mask64_
 0003:000132D4       snd_pcm_hw_constraint_mask_
 0003:0001336D       snd_pcm_hw_constraint_minmax_
 0003:00013538       snd_pcm_hw_constraint_msbits_
 0003:000135C4       snd_pcm_hw_constraint_pow2_
 0003:000134EB       snd_pcm_hw_constraint_ratdens_
 0003:00013462       snd_pcm_hw_constraint_ratnums_
 0003:0001357D       snd_pcm_hw_constraint_step_
 0003:00013898       snd_pcm_hw_params_choose_
 0003:000137C4       snd_pcm_hw_param_first_
 0003:00013861       snd_pcm_hw_param_last_
 0003:00013686       snd_pcm_hw_param_value_
 0003:00016A26       snd_pcm_hw_refine_
 0003:000131BC       snd_pcm_hw_rule_add_
 0003:00016909       snd_pcm_info_
 0003:000169CA       snd_pcm_info_user_
 0003:00019BE9       snd_pcm_kernel_ioctl_
 0003:000163E1       snd_pcm_lib_free_pages_
 0003:00013A15       snd_pcm_lib_ioctl_
 0003:00016316       snd_pcm_lib_malloc_pages_
 0003:000161C0       snd_pcm_lib_preallocate_free_
 0003:000161C8       snd_pcm_lib_preallocate_free_for_all_
 0003:0001622A       snd_pcm_lib_preallocate_pages_
 0003:00016242       snd_pcm_lib_preallocate_pages_for_all_
 0003:00014417       snd_pcm_lib_readv_
 0003:000142E9       snd_pcm_lib_read_
 0003:00014026       snd_pcm_lib_writev_
 0003:00013EBB       snd_pcm_lib_write_
 0003:00011C5D       snd_pcm_limit_hw_rates_
 0003:00014817       snd_pcm_new_
 0003:000146E9       snd_pcm_new_stream_
 0003:00014E30       snd_pcm_notify_
 0003:00018CA9       snd_pcm_open_substream_
 0003:0007C20C       snd_pcm_oss_read3_
 0003:0007C2FD       snd_pcm_oss_readv3_
 0003:0007C1AD       snd_pcm_oss_write3_
 0003:0007C29E       snd_pcm_oss_writev3_
 0003:00013A53       snd_pcm_period_elapsed_
 0003:0001212D       snd_pcm_playback_silence_
 0003:00011CC5       snd_pcm_rate_to_rate_bit_
 0003:00018C40       snd_pcm_release_substream_
 0003:0001275F       snd_pcm_set_ops_
 0003:00012784       snd_pcm_set_sync_
 0003:000162C0       snd_pcm_sgbuf_get_chunk_size_
 0003:000162A2       snd_pcm_sgbuf_ops_page_
 0003:00017848       snd_pcm_start_
 0003:00017264       snd_pcm_status_
 0003:000178F0       snd_pcm_stop_
 0003:00017AAF       snd_pcm_suspend_
 0003:00017B00       snd_pcm_suspend_all_
 0003:00016628       snd_pcm_timer_done_
 0003:0001652F       snd_pcm_timer_init_
 0003:0001643A       snd_pcm_timer_resolution_change_
 0003:00012669       snd_pcm_update_hw_ptr_
 0003:0001D076       snd_power_wait_
 0003:0004F39C       snd_print_pcm_bits_
 0003:0004F341       snd_print_pcm_rates_
 0003:0000FFC3       snd_rawmidi_drain_input_
 0003:0000FF4F       snd_rawmidi_drain_output_
 0003:0000FF0D       snd_rawmidi_drop_output_
 0003:000106D9       snd_rawmidi_info_select_
 0003:0001087F       snd_rawmidi_input_params_
 0003:000101BA       snd_rawmidi_kernel_open_
 0003:00010C67       snd_rawmidi_kernel_read_
 0003:000105C9       snd_rawmidi_kernel_release_
 0003:000110CC       snd_rawmidi_kernel_write_
 0003:00011470       snd_rawmidi_new_
 0003:000107DB       snd_rawmidi_output_params_
 0003:000109C9       snd_rawmidi_receive_
 0003:00011959       snd_rawmidi_set_ops_
 0003:00010F4F       snd_rawmidi_transmit_
 0003:00010ED4       snd_rawmidi_transmit_ack_
 0003:00010DAD       snd_rawmidi_transmit_empty_
 0003:00010DF6       snd_rawmidi_transmit_peek_
 0003:0001516E       snd_register_device_for_dev_
 0003:0001A0FC       snd_register_oss_device_
 0003:0007A446       snd_sbdsp_command_
 0003:0007A6CA       snd_sbdsp_create_
 0003:0007A499       snd_sbdsp_get_byte_
 0003:0007A4E1       snd_sbdsp_reset_
 0003:0007A0AC       snd_sbmixer_add_ctl_
 0003:0007A1D1       snd_sbmixer_new_
 0003:000797D0       snd_sbmixer_read_
 0003:0007A3D2       snd_sbmixer_resume_
 0003:0007A35E       snd_sbmixer_suspend_
 0003:000797A5       snd_sbmixer_write_
 0003:00055B3F       snd_sequencer_device_done_
 0003:00055AE6       snd_sequencer_device_init_
 0003:000535EA       snd_sequencer_memory_done_
 0003:000535E7       snd_sequencer_memory_init_
 0003:00053094       snd_seq_cell_free_
 0003:00052676       snd_seq_check_queue_
 0003:00054855       snd_seq_client_notify_subscription_
 0003:000536D7       snd_seq_client_use_ptr_
 0003:00052D42       snd_seq_control_queue_
 0003:000555B6       snd_seq_create_kernel_client_
 0003:00055C7F       snd_seq_create_port_
 0003:00055F6B       snd_seq_delete_all_ports_
 0003:00055690       snd_seq_delete_kernel_client_
 0003:00055EE4       snd_seq_delete_port_
 0003:00051AB4       snd_seq_device_load_drivers_
 0003:00051AB5       snd_seq_device_new_
 0003:00051C86       snd_seq_device_register_driver_
 0003:00051DC2       snd_seq_device_unregister_driver_
 0003:00053FBA       snd_seq_dispatch_event_
 0003:00052EFA       snd_seq_dump_var_event_
 0003:00052756       snd_seq_enqueue_event_
 0003:00053207       snd_seq_event_dup_
 0003:0005665C       snd_seq_event_port_attach_
 0003:000566EA       snd_seq_event_port_detach_
 0003:00052FEB       snd_seq_expand_var_event_
 0003:00057527       snd_seq_fifo_cell_out_
 0003:000575B2       snd_seq_fifo_cell_putback_
 0003:0005743E       snd_seq_fifo_clear_
 0003:000573F5       snd_seq_fifo_delete_
 0003:00057476       snd_seq_fifo_event_in_
 0003:00057371       snd_seq_fifo_new_
 0003:000575E6       snd_seq_fifo_poll_wait_
 0003:00057601       snd_seq_fifo_resize_
 0003:000560A9       snd_seq_get_port_info_
 0003:000559C4       snd_seq_info_clients_read_
 0003:00052138       snd_seq_info_done_
 0003:000520F7       snd_seq_info_init_
 0003:000535EB       snd_seq_info_pool_
 0003:00052D97       snd_seq_info_queues_read_
 0003:00056E02       snd_seq_info_timer_read_
 0003:00055770       snd_seq_kernel_client_ctl_
 0003:0005572D       snd_seq_kernel_client_dispatch_
 0003:0005570C       snd_seq_kernel_client_enqueue_
 0003:00055718       snd_seq_kernel_client_enqueue_blocking_
 0003:00055783       snd_seq_kernel_client_write_poll_
 0003:000535C8       snd_seq_pool_delete_
 0003:000534A1       snd_seq_pool_done_
 0003:00053403       snd_seq_pool_init_
 0003:0005355C       snd_seq_pool_new_
 0003:000533E3       snd_seq_pool_poll_wait_
 0003:00056294       snd_seq_port_connect_
 0003:000564F8       snd_seq_port_disconnect_
 0003:00056618       snd_seq_port_get_subscription_
 0003:00055BE2       snd_seq_port_query_nearest_
 0003:00055B84       snd_seq_port_use_ptr_
 0003:000570CC       snd_seq_prioq_avail_
 0003:00056FA9       snd_seq_prioq_cell_in_
 0003:00057075       snd_seq_prioq_cell_out_
 0003:000570EA       snd_seq_prioq_cell_peek_
 0003:00056EFE       snd_seq_prioq_delete_
 0003:0005714A       snd_seq_prioq_leave_
 0003:00056EB4       snd_seq_prioq_new_
 0003:000572C2       snd_seq_prioq_remove_events_
 0003:00052578       snd_seq_queues_delete_
 0003:00052575       snd_seq_queues_init_
 0003:00052598       snd_seq_queue_alloc_
 0003:0005284F       snd_seq_queue_check_access_
 0003:00052AC3       snd_seq_queue_client_leave_
 0003:00052B52       snd_seq_queue_client_leave_cells_
 0003:00052A60       snd_seq_queue_client_termination_
 0003:000525D7       snd_seq_queue_delete_
 0003:00052639       snd_seq_queue_find_name_
 0003:000523BB       snd_seq_queue_get_cur_queues_
 0003:00052A2C       snd_seq_queue_is_used_
 0003:00052B90       snd_seq_queue_remove_cells_
 0003:00052889       snd_seq_queue_set_owner_
 0003:00052913       snd_seq_queue_timer_close_
 0003:000528D8       snd_seq_queue_timer_open_
 0003:0005292A       snd_seq_queue_timer_set_tempo_
 0003:00052998       snd_seq_queue_use_
 0003:0005601E       snd_seq_set_port_info_
 0003:00054DF8       snd_seq_set_queue_tempo_
 0003:000521B1       snd_seq_system_broadcast_
 0003:00052349       snd_seq_system_client_done_
 0003:0005221F       snd_seq_system_client_init_
 0003:000521DE       snd_seq_system_notify_
 0003:00056C06       snd_seq_timer_close_
 0003:00056D1D       snd_seq_timer_continue_
 0003:00056882       snd_seq_timer_defaults_
 0003:00056849       snd_seq_timer_delete_
 0003:00056DFE       snd_seq_timer_get_cur_tick_
 0003:00056D6E       snd_seq_timer_get_cur_time_
 0003:00056805       snd_seq_timer_new_
 0003:00056B0A       snd_seq_timer_open_
 0003:000568EE       snd_seq_timer_reset_
 0003:00056A5A       snd_seq_timer_set_position_tick_
 0003:00056A8A       snd_seq_timer_set_position_time_
 0003:000569F3       snd_seq_timer_set_ppq_
 0003:00056AC4       snd_seq_timer_set_skew_
 0003:000569AF       snd_seq_timer_set_tempo_
 0003:00056CD4       snd_seq_timer_start_
 0003:00056C29       snd_seq_timer_stop_
 0003:0000DC05       snd_timer_close_
 0003:0000E0DB       snd_timer_continue_
 0003:0000E890       snd_timer_global_free_
 0003:0000E85B       snd_timer_global_new_
 0003:0000E895       snd_timer_global_register_
 0003:0000E269       snd_timer_interrupt_
 0003:0000E4B1       snd_timer_new_
 0003:0000E765       snd_timer_notify_
 0003:0000DAAF       snd_timer_open_
 0003:0000E155       snd_timer_pause_
 0003:0000DD5D       snd_timer_resolution_
 0003:0000DF39       snd_timer_start_
 0003:0000E095       snd_timer_stop_
 0003:000781B7       snd_trident_alloc_pages_
 0003:00077BE6       snd_trident_alloc_voice_
 0003:000776B1       snd_trident_create_
 0003:0007707F       snd_trident_create_gameport_
 0003:0007612C       snd_trident_foldback_pcm_
 0003:000781C6       snd_trident_free_pages_
 0003:00077C96       snd_trident_free_voice_
 0003:00075FD6       snd_trident_pcm_
 0003:00077E55       snd_trident_resume_
 0003:000762CF       snd_trident_spdif_pcm_
 0003:00074892       snd_trident_start_voice_
 0003:000748BD       snd_trident_stop_voice_
 0003:00077DD3       snd_trident_suspend_
 0003:000749CE       snd_trident_write_voice_regs_
 0003:0001525C       snd_unregister_device_
 0003:0001A187       snd_unregister_oss_device_
 0003:000880C0       snd_util_memhdr_free_
 0003:0008808D       snd_util_memhdr_new_
 0003:0008819E       snd_util_mem_alloc_
 0003:00088203       snd_util_mem_avail_
 0003:000881E2       snd_util_mem_free_
 0003:00071FA4       snd_ymfpci_create_
 0003:0006EE6D       snd_ymfpci_free_gameport_
 0003:00071427       snd_ymfpci_mixer_
 0003:00070A0B       snd_ymfpci_pcm2_
 0003:0007093A       snd_ymfpci_pcm_
 0003:00070B84       snd_ymfpci_pcm_4ch_
 0003:00070AC5       snd_ymfpci_pcm_spdif_
 0003:00071EBA       snd_ymfpci_resume_
 0003:00071DF1       snd_ymfpci_suspend_
 0003:000716E2       snd_ymfpci_timer_
 0003:000884E0       snprintf_
 0003:0000CF50       spin_lock_
 0003:0000CF5A       spin_lock_flag_
 0003:0000CF49       spin_lock_init_
 0003:0000CF64       spin_trylock_
 0003:0000CF67       spin_unlock_
 0003:00005259       sprintf_
 0003:00088410       sscanf_
 0005:00001768       stackbase
 0005:0000176C       stacksel
 0003:00000080       STRATEGY_
 0003:0000537A       strcmp_
 0003:00008BB1       StringOut_
 0003:00088350       strlcpy_
 0003:0007E160       StrLen
 0003:0007E180       StrNCmp
 0003:0000539D       strncmp_
 0003:0000CF14       strncpy_
 0003:000882A0       strstr_
 0003:0008AB90       strtol_
 0003:0008AB80       strtoul_
 0003:0008A250       strupr_
 0003:000053C6       tasklet_hi_schedule_
 0003:000053DB       tasklet_init_
 0003:00000024       thunk1632_devhelp
 0003:00000044       thunk1632_devhelp_modified_ds
 0002:000001A0       thunk3216_devhelp
 0002:000001B2       thunk3216_devhelp_modified_ds
 0003:00000140       TIMER_
 0003:0008A580       tolower_
 0003:0008A460       ulltoa_
 0003:0008A3E0       ultoa_
 0003:0000AB8F       UniaudCloseAll_
 0003:0000A1BB       UniaudCtlGetPowerState_
 0003:0000A27F       UniaudCtlSetPowerState_
 0003:0000A9A6       UniaudIoctlHWParamSet_
 0003:0000A965       UniaudIoctlHWRefine_
 0003:0000AB5E       UniaudIoctlPCMDrop_
 0003:0000AAC9       UniaudIoctlPCMPrepare_
 0003:0000AA99       UniaudIoctlPCMRead_
 0003:0000AAFA       UniaudIoctlPCMResume_
 0003:0000AB2D       UniaudIoctlPCMStart_
 0003:0000AA28       UniaudIoctlPCMStatus_
 0003:0000AA69       UniaudIoctlPCMWrite_
 0003:0000A9E7       UniaudIoctlSWParamSet_
 0001:0000001E       uniaud_header
 0003:00009BC2       uniaud_set_interrupted_substream_
 0002:0000010A       uniaud_stub_idc
 0002:00000096       uniaud_stub_strategy
 0002:00000128       uniaud_stub_timer
 0003:00007346       UNIXToOSSError_
 0003:000071BA       unregister_chrdev_
 0003:00005528       unregister_reboot_notifier_
 0003:0000731A       unregister_sound_dsp_
 0003:00007304       unregister_sound_midi_
 0003:000072EE       unregister_sound_mixer_
 0003:000072D8       unregister_sound_special_
 0003:00007330       unregister_sound_synth_
 0003:0007E41F       up_
 0003:0008A500       utoa_
 0003:00009784       vfree_
 0003:00009010       virt_to_phys_
 0003:000096C2       vmalloc_
 0003:0000907A       VMAlloc_
 0003:000090E0       VMFree_
 0003:00088480       vsnprintf_
 0003:00004FAA       vsprintf_
 0003:000883E0       vsscanf_
 0003:00004D81       W?$dln(pnv)v
 0003:00004D7C       W?$nwn(ui)pnv
 0003:00004D86       W?$nwn(uipnv)pnv
 0005:00000554       W?acHeap$npnuc
 0003:000057EC       W?CallOSS16$n(ululul)ul
 0003:000016DB       W?CheckCardName$n(pfa)v
 0003:0000CC31       W?compact$n()v
 0005:00000030       W?deviceOwner$nul
 0003:000006B0       W?DevSaveMessage$n(pfai)v
 0003:000007D2       W?DiscardableInit$n(pf$RPInit$$)ul
 0003:00001912       W?DoParm$n(apfa)i
 0003:0000C9B4       W?dumpheap$n()v
 0005:000000B0       W?fnCardExitCall$n[]pn()v
 0005:00001894       W?ForceCard$ni
 0003:0000CCD5       W?free$n(pnv)v
 0003:0000CA2A       W?HeapCheck$n(pna)v
 0003:0000CEB4       W?HeapInit$n(ul)ul
 0003:0000CE94       W?IsHeapAddr$n(ul)ul
 0003:00001682       W?IsWhitespace$n(a)i
 0003:00000730       W?LockSegments$n()i
 0003:0000CB00       W?malloc$n(ul)pnv
 0003:000015B2       W?mymemchr$n(pfaaus)pfa
 0003:0000CA83       W?npvAllocateBlock$n(pn$_MEMBLOCK$$ulpn$1$)pnv
 0005:00000034       W?numOS2Opens$nul
 0003:00003ABA       W?OSS32IDC$n(ulpn$__6ikc0pIDC32_PACKET$$)ul
 0003:00001BEF       W?ParseParm$n(pfai)i
 0005:0000054C       W?pmbFree$npn$_MEMBLOCK$$
 0005:00000548       W?pmbUsed$npn$_MEMBLOCK$$
 0003:0000CE21       W?realloc$n(pnvul)pnv
 0003:0000CC03       W?remove$n(pn$_MEMBLOCK$$)v
 0005:00000060       W?RMFlags$nul
 0005:00000054       W?RM_Help$npn()i
 0005:00000058       W?RM_Help0$npn()i
 0005:0000005C       W?RM_Help3$npn()i
 0003:0000C9E5       W?SignatureCheck$n(pn$_MEMBLOCK$$pna)s
 0003:0000169B       W?SkipWhite$n(pfa)pfa
 0003:000044E1       W?StratClose$n(pf$RP$$)ul
 0005:00001800       W?StratDispatch$n[]pn(pf$RP$$)ul
 0003:000004E6       W?StratInit$n(pf$RP$$)ul
 0003:00000523       W?StratInitComplete$n(pf$RP$$)ul
 0003:00003DD0       W?StratIOCtl$n(pf$RP$$)ul
 0003:000004C1       W?StratOpen$n(pf$RP$$)ul
 0003:000005AA       W?StratRead$n(pf$RP$$)ul
 0003:0000053D       W?StratShutdown$n(pf$RP$$)ul
 0003:000015EA       W?sz2us$n(pfai)us
 0003:000015A4       W?toupper$n(i)i
 0005:0000055C       W?ulcAlloc$nul
 0005:00000568       W?ulcFree$nul
 0005:0000E9E0       W?ulcTotalHeap$nul
 0005:00000558       W?ulnAlloc$nul
 0005:00000560       W?ulnAllocCalls$nul
 0005:00000570       W?ulnCompact$nul
 0005:00000564       W?ulnFree$nul
 0005:0000056C       W?ulnFreeCalls$nul
 0005:00000550       W?uMemFree$nui
 0003:0000CE0F       W?_memfree$n()ui
 0003:0000CE15       W?_msize$n(pnv)ui
 0003:00009BF5       WaitForControlChange_
 0003:00009C52       WaitForPCMInterrupt_
 0003:0000CF46       waitqueue_active_
 0003:0008A2D0       wctomb_
 0005:00002144       _alsa_fops
 0005:0003FE1F       _auto_pin_cfg_labels
 0003:00000050       _CallPDD16
 0002:0000049A       _CallRM
 0005:00001D04       _cardcalls
 0005:0000A214       _card_id_changed
 0005:0000A210       _control_id_changed
 0005:000081D4       _CountWv
 0005:000018EC       _current
 0005:000018C8       _current_task
 0005:000000D8       _DbgInt
 0005:000000FC       _DebugLevel
 0005:000873D0       _edata
 0005:000873D0       _end
 0005:00000048       _fDebug
 0005:0000A21C       _fInInterrupt
 0005:0000D5DC       _fRewired
 0005:000000D4       _fStrategyInit
 0005:00000044       _fVerbose
 0005:000081DC       _hextab
 0005:0000004C       _idc16_PddHandler
 0005:00001CB4       _iLastError
 0005:00001A92       _iomem_resource
 0005:00001A76       _ioport_resource
 0003:0008A3C0       _ismbblead_
 0005:000017D2       _ISR00
 0005:000017D6       _ISR01
 0005:000017DA       _ISR02
 0005:000017DE       _ISR03
 0005:000017E2       _ISR04
 0005:000017E6       _ISR05
 0005:000017EA       _ISR06
 0005:000017EE       _ISR07
 0005:000018C4       _jiffies
 0000:00000000  Imp  _KernSISData         (KEE.90)
 0005:000081D8       _LockAdd
 0005:000081ED       _MAGIC_COMM_PORT
 0005:00001AAE       _mem_map
 0001:00000058       _MESSAGE_STR
 0005:00001E0C       _midi_port
 0001:00000458       _MSG_TABLE16
 0005:00001774       _MSG_TABLE32
 0005:000000D0       _nrCardsDetected
 0005:00002158       _opened_handles
 0005:000401BC       _opl3_ops
 0005:00002004       _oss_devices
 0005:0000AA9C       _pci_devices
 0005:000081F0       _pcmcaps
 0005:00002150       _pcm_device
 0005:00002148       _per_bytes
 0005:0000214C       _prev_size
 0003:0000541E       _printk
 0005:00001CB8       _proc_root
 0003:0000990A       _put_user_
 0005:00000038       _rdOffset
 0003:00000230       _RMAllocResource
 0002:00000204       _RMAllocResource16
 0002:000001C8       _RMAllocResourceOrg
 0003:0000033C       _RMCreateAdapter
 0002:000002B6       _RMCreateAdapter16
 0002:0000027A       _RMCreateAdapterOrg
 0003:000002F4       _RMCreateDevice
 0002:0000031E       _RMCreateDevice16
 0002:000002E2       _RMCreateDeviceOrg
 0003:00000384       _RMCreateDriver
 0002:0000047A       _RMCreateDriver16
 0002:00000400       _RMCreateDriverOrg
 0003:000002B4       _RMDeallocResource
 0002:000003BA       _RMDeallocResource16
 0002:00000390       _RMDeallocResourceOrg
 0002:00000374       _RMDestroyDevice16
 0002:0000034A       _RMDestroyDeviceOrg
 0003:000003C4       _RMDestroyDriver
 0002:000004F8       _RMDestroyDriver16
 0002:000004CE       _RMDestroyDriverOrg
 0003:00000430       _RMDevIDToHandleList
 0002:000005A8       _RMDevIDToHandleList16
 0001:00000054       _RMFlags
 0003:000003F0       _RMGetNodeInfo
 0002:0000054C       _RMGetNodeInfo16
 0003:00000484       _RMHandleToResourceHandleList
 0002:0000061C       _RMHandleToResourceHandleList16
 0003:00000270       _RMModifyResources
 0002:00000252       _RMModifyResources16
 0002:00000228       _RMModifyResourcesOrg
 0001:00000048       _RM_Help0
 0001:0000004C       _RM_Help1
 0001:00000050       _RM_Help3
 0005:0003FFE8       _seq_client_load
 0005:0004002C       _seq_default_timer_card
 0005:00040024       _seq_default_timer_class
 0005:00040030       _seq_default_timer_device
 0005:00040038       _seq_default_timer_resolution
 0005:00040028       _seq_default_timer_sclass
 0005:00040034       _seq_default_timer_subdevice
 0005:00000DA8       _snd_cards
 0003:0007E70B       _snd_ctl_add_slave_
 0005:00000AA4       _snd_ecards_limit
 0005:0003FB93       _snd_hda_bind_sw
 0005:0003FB83       _snd_hda_bind_vol
 0005:00000AA8       _snd_major
 0005:000403EC       _snd_opl3_regmap
 0005:00000AB8       _snd_oss_root
 0005:0000059C       _snd_pcm_devices_os2
 0005:0000F008       _snd_pcm_f_ops
 0003:00013640       _snd_pcm_hw_params_any_
 0003:000136FD       _snd_pcm_hw_param_setempty_
 0003:0007B387       _snd_pcm_hw_param_set_
 0005:00071F50       _snd_pcm_known_rates
 0005:0000EF44       _snd_pcm_link_rwlock
 0005:00000AB4       _snd_seq_root
 0005:00008210       _substream_int
 0005:000018F0       _system_utsname
 0005:00001BB2       _szLastALSAError1
 0005:00001C33       _szLastALSAError2
 0005:00001C32       _szOverrunTest1
 0005:00001CB3       _szOverrunTest2
 0005:00000040       _szprintBuf
 0005:00001F78       _szRecSources
 0005:00001AB2       _this_module
 0005:000017CC       _TimerHandler16
 0005:000017FC       _TKSSBase
 0005:00002154       _total
 0005:00000104       _ulget_free_pagesMemUsed
 0005:0000A218       _unlock_all
 0005:000401B8       _use_internal_drums
 0005:0000003C       _wrOffset
 0005:0005F098       __AccessFHeap
 0005:0005F084       __AccessFileH
 0005:0005F08C       __AccessIOB
 0005:0005F094       __AccessNHeap
 0005:0005F0A4       __AccessTDList
 0005:0005F10C       __amblksiz
 0005:0005F0EC       __ASTACKPTR
 0005:0005F0E8       __ASTACKSIZ
 0003:0008A270       __Bits
 0005:0005F0F0       __cbyte
 0005:0005F0F4       __cbyte2
 0003:00005478       __check_region_
 0005:0005F0F8       __child
 0003:0008A950       __CommonInit_
 0003:0000BA4A       __compat_get_order_
 0003:0000982B       __copy_user_
 0003:0000987F       __copy_user_zeroing_
 0005:0005F0C4       __curbrk
 0000:00001234  Abs  __DOSseg__
 0005:0005F0C0       __dynend
 0005:00077372       __End_XI
 0005:00077372       __End_YI
 0003:0008A860       __EnterWVIDEO_
 0005:0005F0FE       __Envptr
 0005:0005F102       __Envseg
 0003:0008A816       __exit_
 0003:0008A590       __exit_with_msg_
 0003:0008A5E0       __fatal_runtime_error_
 0003:0008A204       __FDFS
 0003:0008A8F0       __FiniRtns
 0003:00000000       __GETDS
 0003:000090EE       __get_free_dma_pages_
 0003:000092D9       __get_free_pages_
 0003:000098DF       __get_user_
 0003:00088265       __I8LS
 0003:00088280       __I8M
 0003:0008824A       __I8RS
 0003:0008A8A0       __InitRtns
 0003:000097BB       __ioremap_
 0003:00088590       __IsTable
 0003:000099F5       __kfree_
 0003:0000991A       __kmalloc_
 0005:0005F0C8       __LpCmdLine
 0005:0005F0D0       __LpDllName
 0005:0005F0CC       __LpPgmName
 0005:0005F0D4       __LpwCmdLine
 0005:0005F0DC       __LpwDllName
 0005:0005F0D8       __LpwPgmName
 0003:0008A63A       __mbinit_
 0005:0005F0FC       __no87
 0005:000773C0       __nullarea
 0003:00000000       __OffBeginCS32
 0005:00000000       __OffBeginDS32
 0002:000006DB       __OffFinalCS16
 0003:0008ABE8       __OffFinalCS32
 0001:00000483       __OffFinalDS16
 0005:00077368       __OffFinalDS32
 0005:00001770       __OffsetFinalCS16
 0005:00001772       __OffsetFinalDS16
 0003:0008A7F9       __OS2Fini_
 0003:0008A7BB       __OS2Init_
 0003:0008A74C       __OS2MainInit_
 0005:0005F104       __osmajor
 0005:0005F105       __osminor
 0003:00089520       __prtf_
 0005:0005F0A0       __ReleaseFHeap
 0005:0005F088       __ReleaseFileH
 0005:0005F090       __ReleaseIOB
 0005:0005F09C       __ReleaseNHeap
 0005:0005F0A8       __ReleaseTDList
 0003:0000B566       __release_region_
 0003:0000B4EC       __request_region_
 0003:000892B0       __scnf_
 0003:0008ABDA       __set_doserrno_
 0003:0008ABAB       __set_EDOM_
 0003:0008ABC7       __set_EINVAL_
 0003:0008ABB9       __set_ERANGE_
 0003:0008AB9D       __set_errno_
 0003:0008A801       __shutdown_stack_checking_
 0003:00088148       __snd_util_memblk_new_
 0003:000880F4       __snd_util_mem_alloc_
 0003:000881C1       __snd_util_mem_free_
 0005:0005F0E0       __STACKLOW
 0005:0005F0E4       __STACKTOP
 0005:0007736C       __Start_XI
 0005:00077372       __Start_YI
 0003:000886A0       __STOSB
 0003:000886D7       __STOSD
 0003:0008A743       __threadid_
 0003:0008A73C       __threadstack_
 0005:0005F0B4       __threadstksize
 0003:00088265       __U8LS
 0003:00088280       __U8M
 0003:00088230       __U8RS
 0003:000052CA       __udelay_
 0003:0000CF44       __wake_up_
 0003:00004D70       __wcpp_2_pure_error__
 0003:00004D6C       __wcpp_2_undefed_cdtor__
 0003:00004D6E       __wcpp_2_undefined_member_function__
 0003:00004D72       __wcpp_2_undef_vfun__
 0003:00004D78       __wcpp_4_pure_error__
 0003:00004D74       __wcpp_4_undefed_cdtor__
 0003:00004D76       __wcpp_4_undefined_member_function__
 0003:00004D7A       __wcpp_4_undef_vfun__
 0005:0006F278       ___Alphabet
 0004:00000003       ___begtext
 0005:0005F070       ___EFG_printf
 0005:0005F074       ___EFG_scanf
 0005:0005F972       ___exitcall_alsa_ac97_exit
 0005:00051BF8       ___exitcall_alsa_card_ali_exit
 0005:0000F714       ___exitcall_alsa_card_als4000_exit
 0005:00010918       ___exitcall_alsa_card_atiixp_exit
 0005:0003FA30       ___exitcall_alsa_card_azx_exit
 0005:0000F578       ___exitcall_alsa_card_bt87x_exit
 0005:0001410C       ___exitcall_alsa_card_ca0106_exit
 0005:00010575       ___exitcall_alsa_card_cmipci_exit
 0005:000137A4       ___exitcall_alsa_card_cs4281_exit
 0005:00040550       ___exitcall_alsa_card_cs46xx_exit
 0005:0004E230       ___exitcall_alsa_card_cs5535audio_exit
 0005:0004E49C       ___exitcall_alsa_card_emu10k1_exit
 0005:00013C20       ___exitcall_alsa_card_ens137x_exit
 0005:000134D1       ___exitcall_alsa_card_es1938_exit
 0005:00012C38       ___exitcall_alsa_card_es1968_exit
 0005:00010DD8       ___exitcall_alsa_card_fm801_exit
 0005:00012984       ___exitcall_alsa_card_intel8x0_exit
 0005:00011A10       ___exitcall_alsa_card_m3_exit
 0005:0005EA28       ___exitcall_alsa_card_nm256_exit
 0005:00051D34       ___exitcall_alsa_card_trident_exit
 0005:000113EC       ___exitcall_alsa_card_via82xx_exit
 0005:00051238       ___exitcall_alsa_card_ymfpci_exit
 0005:0000EA48       ___exitcall_alsa_hwdep_exit
 0005:00040434       ___exitcall_alsa_mpu401_uart_exit
 0005:00040258       ___exitcall_alsa_opl3_exit
 0005:000401E4       ___exitcall_alsa_opl3_seq_exit
 0005:0000EE64       ___exitcall_alsa_pcm_exit
 0005:0005F06C       ___exitcall_alsa_pcm_oss_exit
 0005:0000EB84       ___exitcall_alsa_rawmidi_exit
 0005:0005EFEC       ___exitcall_alsa_sb_common_exit
 0005:00040068       ___exitcall_alsa_seq_device_exit
 0005:00040040       ___exitcall_alsa_seq_exit
 0005:0005FA9C       ___exitcall_alsa_seq_midi_emul_exit
 0005:0000EEC0       ___exitcall_alsa_sound_exit
 0005:0000EAF4       ___exitcall_alsa_timer_exit
 0005:0005FAA4       ___exitcall_alsa_util_mem_exit
 0005:00022144       ___exitcall_patch_analog_exit
 0005:00017D9C       ___exitcall_patch_atihdmi_exit
 0005:000228D4       ___exitcall_patch_cmedia_exit
 0005:00017C40       ___exitcall_patch_conexant_exit
 0005:0003F401       ___exitcall_patch_realtek_exit
 0005:0001AC32       ___exitcall_patch_sigmatel_exit
 0005:00015E20       ___exitcall_patch_via_exit
 0005:0000F118       ___exitcall_snd_mem_exit
 0005:0005F07C       ___FirstThreadData
 0005:0005F106       ___FPE_handler
 0005:0005F080       ___GetThreadPtr
 0005:00001734       ___hmodule
 0005:0005F96E       ___initcall_alsa_ac97_init
 0005:00051BF4       ___initcall_alsa_card_ali_init
 0005:0000F710       ___initcall_alsa_card_als4000_init
 0005:00010914       ___initcall_alsa_card_atiixp_init
 0005:0003FA2C       ___initcall_alsa_card_azx_init
 0005:0000F574       ___initcall_alsa_card_bt87x_init
 0005:00014108       ___initcall_alsa_card_ca0106_init
 0005:00010571       ___initcall_alsa_card_cmipci_init
 0005:000137A0       ___initcall_alsa_card_cs4281_init
 0005:0004054C       ___initcall_alsa_card_cs46xx_init
 0005:0004E22C       ___initcall_alsa_card_cs5535audio_init
 0005:0004E498       ___initcall_alsa_card_emu10k1_init
 0005:00013C1C       ___initcall_alsa_card_ens137x_init
 0005:000134CD       ___initcall_alsa_card_es1938_init
 0005:00012C34       ___initcall_alsa_card_es1968_init
 0005:00010DD4       ___initcall_alsa_card_fm801_init
 0005:00012980       ___initcall_alsa_card_intel8x0_init
 0005:00011A0C       ___initcall_alsa_card_m3_init
 0005:0005EA24       ___initcall_alsa_card_nm256_init
 0005:00051D30       ___initcall_alsa_card_trident_init
 0005:000113E8       ___initcall_alsa_card_via82xx_init
 0005:00051234       ___initcall_alsa_card_ymfpci_init
 0005:0000EA44       ___initcall_alsa_hwdep_init
 0005:00040430       ___initcall_alsa_mpu401_uart_init
 0005:00040254       ___initcall_alsa_opl3_init
 0005:000401E0       ___initcall_alsa_opl3_seq_init
 0005:0000EE60       ___initcall_alsa_pcm_init
 0005:0005F068       ___initcall_alsa_pcm_oss_init
 0005:0000EB80       ___initcall_alsa_rawmidi_init
 0005:0005EFE8       ___initcall_alsa_sb_common_init
 0005:00040064       ___initcall_alsa_seq_device_init
 0005:0004003C       ___initcall_alsa_seq_init
 0005:0005FA98       ___initcall_alsa_seq_midi_emul_init
 0005:0000EEBC       ___initcall_alsa_sound_init
 0005:0000EAF0       ___initcall_alsa_timer_init
 0005:0005FAA0       ___initcall_alsa_util_mem_init
 0005:00022140       ___initcall_patch_analog_init
 0005:00017D98       ___initcall_patch_atihdmi_init
 0005:000228D0       ___initcall_patch_cmedia_init
 0005:00017C3C       ___initcall_patch_conexant_init
 0005:0003F3FD       ___initcall_patch_realtek_init
 0005:0001AC2E       ___initcall_patch_sigmatel_init
 0005:00015E1C       ___initcall_patch_via_init
 0005:0000F114       ___initcall_snd_mem_init
 0005:00001628       ___IsDBCS
 0005:0000162C       ___Is_DLL
 0005:0005F078       ___MBCodePage
 0005:00001524       ___MBCSIsTable
 0005:0005F0B8       ___process_fini
 0005:00001630       ___saved_CS
 0005:0005F0B0       ___sig_fini_rtn
 0005:0005F0AC       ___sig_init_rtn
 0005:0005F0BC       ___WD_Present


 Address         Publics by Value
 0000:00000000  Imp  DOSCLOSE             (DOSCALLS.59)
 0000:00000000  Imp  DOSIODELAYCNT        (DOSCALLS.427)
 0000:00000000  Imp  DosQuerySysInfo      (DOSCALLS.348)
 0000:00000000  Imp  KernSelToFlat        (KEE.66)
 0000:00000000  Imp  KernVMFree           (KEE.61)
 0000:00000000  Imp  KernVMLock           (KEE.62)
 0000:00000000  Imp  DosWrite             (DOSCALLS.282)
 0000:00000000  Imp  _KernSISData         (KEE.90)
 0000:00000000  Imp  DOSOPEN              (DOSCALLS.70)
 0000:00000000  Imp  DosQueryCp           (DOSCALLS.291)
 0000:00000000  Imp  KernLinToPageList    (KEE.64)
 0000:00000000  Imp  KernThunkStackTo32   (KEE.41)
 0000:00000000  Imp  DOS32FLATDS          (DOSCALLS.370)
 0000:00000000  Imp  KernVMAlloc          (KEE.60)
 0000:00000000  Imp  DOSWRITE             (DOSCALLS.138)
 0000:00000000  Imp  KernThunkStackTo16   (KEE.40)
 0000:00000000  Imp  DosExit              (DOSCALLS.234)
 0000:00000000  Imp  DosQueryDBCSEnv      (NLS.6)
 0000:00001234  Abs  __DOSseg__
 0001:00000000       help_header
 0001:0000001E       uniaud_header
 0001:0000003C       DevHelpInit
 0001:00000040       fOpen
 0001:00000044       InitPktSeg
 0001:00000046       InitPktOff
 0001:00000048       _RM_Help0
 0001:0000004C       _RM_Help1
 0001:00000050       _RM_Help3
 0001:00000054       _RMFlags
 0001:00000058       _MESSAGE_STR
 0001:00000458       _MSG_TABLE16
 0001:0000045E       pddname16
 0001:00000465       FileName
 0001:00000483       __OffFinalDS16
 0002:00000000       help_stub_strategy
 0002:00000096       uniaud_stub_strategy
 0002:0000010A       uniaud_stub_idc
 0002:00000128       uniaud_stub_timer
 0002:000001A0       thunk3216_devhelp
 0002:000001B2       thunk3216_devhelp_modified_ds
 0002:000001C8       _RMAllocResourceOrg
 0002:00000204       _RMAllocResource16
 0002:00000228       _RMModifyResourcesOrg
 0002:00000252       _RMModifyResources16
 0002:0000027A       _RMCreateAdapterOrg
 0002:000002B6       _RMCreateAdapter16
 0002:000002E2       _RMCreateDeviceOrg
 0002:0000031E       _RMCreateDevice16
 0002:0000034A       _RMDestroyDeviceOrg
 0002:00000374       _RMDestroyDevice16
 0002:00000390       _RMDeallocResourceOrg
 0002:000003BA       _RMDeallocResource16
 0002:000003DA       MY_DEVHELP_ATTACHDD
 0002:00000400       _RMCreateDriverOrg
 0002:0000047A       _RMCreateDriver16
 0002:0000049A       _CallRM
 0002:000004CE       _RMDestroyDriverOrg
 0002:000004F8       _RMDestroyDriver16
 0002:0000054C       _RMGetNodeInfo16
 0002:000005A8       _RMDevIDToHandleList16
 0002:0000061C       _RMHandleToResourceHandleList16
 0002:000006DB       __OffFinalCS16
 0003:00000000       __OffBeginCS32
 0003:00000000       __GETDS
 0003:00000010       DevHlp
 0003:00000024       thunk1632_devhelp
 0003:00000030       DevHlp_ModifiedDS
 0003:00000044       thunk1632_devhelp_modified_ds
 0003:00000050       _CallPDD16
 0003:00000080       STRATEGY_
 0003:000000E0       IDC_
 0003:00000140       TIMER_
 0003:00000230       _RMAllocResource
 0003:00000270       _RMModifyResources
 0003:000002B4       _RMDeallocResource
 0003:000002F4       _RMCreateDevice
 0003:0000033C       _RMCreateAdapter
 0003:00000384       _RMCreateDriver
 0003:000003C4       _RMDestroyDriver
 0003:000003F0       _RMGetNodeInfo
 0003:00000430       _RMDevIDToHandleList
 0003:00000484       _RMHandleToResourceHandleList
 0003:000004C1       W?StratOpen$n(pf$RP$$)ul
 0003:000004E6       W?StratInit$n(pf$RP$$)ul
 0003:00000523       W?StratInitComplete$n(pf$RP$$)ul
 0003:0000053D       W?StratShutdown$n(pf$RP$$)ul
 0003:00000557       ALSA_STRATEGY
 0003:000005AA       W?StratRead$n(pf$RP$$)ul
 0003:000006B0       W?DevSaveMessage$n(pfai)v
 0003:00000730       W?LockSegments$n()i
 0003:000007D2       W?DiscardableInit$n(pf$RPInit$$)ul
 0003:000015A4       W?toupper$n(i)i
 0003:000015B2       W?mymemchr$n(pfaaus)pfa
 0003:000015EA       W?sz2us$n(pfai)us
 0003:00001682       W?IsWhitespace$n(a)i
 0003:0000169B       W?SkipWhite$n(pfa)pfa
 0003:000016DB       W?CheckCardName$n(pfa)v
 0003:00001912       W?DoParm$n(apfa)i
 0003:00001BEF       W?ParseParm$n(pfai)i
 0003:0000281A       GetParms_
 0003:00003510       GetTKSSBase
 0003:00003550       iodelay32_
 0003:00003652       ALSA_IDC
 0003:00003ABA       W?OSS32IDC$n(ulpn$__6ikc0pIDC32_PACKET$$)ul
 0003:00003DD0       W?StratIOCtl$n(pf$RP$$)ul
 0003:000044E1       W?StratClose$n(pf$RP$$)ul
 0003:00004510       RMInit_
 0003:00004687       RMRequestIO_
 0003:0000472B       RMRequestMem_
 0003:000047C0       RMRequestIRQ_
 0003:00004887       RMDeallocateIRQ_
 0003:000048AE       RMDone_
 0003:00004C6C       RMSetHandles_
 0003:00004C78       ALSA_SetIrq_
 0003:00004D0D       ALSA_FreeIrq_
 0003:00004D2B       ALSA_Interrupt
 0003:00004D6C       __wcpp_2_undefed_cdtor__
 0003:00004D6E       __wcpp_2_undefined_member_function__
 0003:00004D70       __wcpp_2_pure_error__
 0003:00004D72       __wcpp_2_undef_vfun__
 0003:00004D74       __wcpp_4_undefed_cdtor__
 0003:00004D76       __wcpp_4_undefined_member_function__
 0003:00004D78       __wcpp_4_pure_error__
 0003:00004D7A       __wcpp_4_undef_vfun__
 0003:00004D7C       W?$nwn(ui)pnv
 0003:00004D81       W?$dln(pnv)v
 0003:00004D86       W?$nwn(uipnv)pnv
 0003:00004D8D       os2gettimesec_
 0003:00004D93       os2gettimemsec_
 0003:00004FAA       vsprintf_
 0003:00005259       sprintf_
 0003:0000527F       ALSA_TIMER_
 0003:000052BB       schedule_timeout_
 0003:000052CA       __udelay_
 0003:000052DE       mdelay_
 0003:00005307       do_gettimeofday_
 0003:00005343       add_timer_
 0003:00005344       del_timer_
 0003:00005347       mod_timer_
 0003:00005348       msleep_
 0003:0000537A       strcmp_
 0003:0000539D       strncmp_
 0003:000053C6       tasklet_hi_schedule_
 0003:000053DB       tasklet_init_
 0003:000053EF       OSS32_SetFileId_
 0003:0000541E       _printk
 0003:00005476       schedule_
 0003:00005477       poll_wait_
 0003:00005478       __check_region_
 0003:0000547B       hweight32_
 0003:000054D7       create_proc_entry_
 0003:00005514       remove_proc_entry_
 0003:00005515       proc_register_
 0003:00005518       proc_unregister_
 0003:0000551B       fasync_helper_
 0003:0000551E       kill_fasync_
 0003:0000551F       request_dma_
 0003:00005522       free_dma_
 0003:00005523       enable_dma_
 0003:00005524       disable_dma_
 0003:00005525       register_reboot_notifier_
 0003:00005528       unregister_reboot_notifier_
 0003:00005566       queue_work_
 0003:000055FA       flush_workqueue_
 0003:00005649       create_workqueue_
 0003:00005695       destroy_workqueue_
 0003:0000569A       kstrdup_
 0003:000056D5       mod_firmware_load_
 0003:00005712       request_firmware_
 0003:00005791       release_firmware_
 0003:000057A9       memdup_user_
 0003:000057EC       W?CallOSS16$n(ululul)ul
 0003:00005821       OSS32_Initialize_
 0003:000059C5       OSS32_Shutdown_
 0003:00005A58       OSS32_ProcessIRQ_
 0003:00005A93       OSS32_ProcessMIDIIRQ_
 0003:00005ACD       OSS32_CloseUNI16_
 0003:00005B08       MyDevBlock_
 0003:00005B37       OSS32_DebugString_
 0003:00005B5E       OSS32_MidiOpen_
 0003:00005ECB       OSS32_MidiClose_
 0003:00005FF1       OSS32_MidiWrite_
 0003:00005FF7       OSS32_MidiRead_
 0003:00006046       OSS32_MidiQueryCaps_
 0003:0000606A       OSS32_MidiCommand_
 0003:00006191       ConvertVolume_
 0003:000061B5       OSS32_MixOpen_
 0003:000066B0       OSS32_MixClose_
 0003:00006706       OSS32_MixGetVolume_
 0003:00006761       OSS32_MixSetVolume_
 0003:00006A75       OSS32_MixSetProperty_
 0003:00006DA2       OSS32_MixGetProperty_
 0003:00006DC1       OSSToALSAVolume_
 0003:00006EA5       OSS32_MixQueryCaps_
 0003:00006F3A       OSS32_MixQueryName_
 0003:0000702C       OSS32_QueryNames_
 0003:000071A1       register_chrdev_
 0003:000071BA       unregister_chrdev_
 0003:000071D2       register_sound_special_
 0003:00007207       register_sound_mixer_
 0003:0000723C       register_sound_midi_
 0003:00007271       register_sound_dsp_
 0003:000072A3       register_sound_synth_
 0003:000072D8       unregister_sound_special_
 0003:000072EE       unregister_sound_mixer_
 0003:00007304       unregister_sound_midi_
 0003:0000731A       unregister_sound_dsp_
 0003:00007330       unregister_sound_synth_
 0003:00007346       UNIXToOSSError_
 0003:00007421       ALSAToOSSDataType_
 0003:0000749F       ALSAToOSSRateFlags_
 0003:00007575       OSS32_QueryDevCaps_
 0003:000078E6       OSS32_WaveOpen_
 0003:00007AAC       OSS32_WaveClose_
 0003:00007B7A       OSS32_WavePrepare_
 0003:00007BDD       OSS32_WaveStart_
 0003:00007C33       OSS32_WaveStop_
 0003:00007C89       OSS32_WavePause_
 0003:00007CDF       OSS32_WaveResume_
 0003:00007D38       OSS32_WaveSetHwParams_
 0003:000085A0       OSS32_WaveAddBuffer_
 0003:000087C1       OSS32_WaveGetPosition_
 0003:00008827       OSS32_WaveGetSpace_
 0003:0000888D       OSS32_WaveGetHwPtr_
 0003:000088F3       OSS32_WaveGetStatus_
 0003:0000894E       OSS32_WaveSetVolume_
 0003:000089AF       DecLongToASCII_
 0003:00008A91       HexLongToASCII_
 0003:00008B6F       CharOut_
 0003:00008BB1       StringOut_
 0003:00008CF8       snd_iprintf_
 0003:00008ECA       DbgPrintIrq_
 0003:00008F0B       AddBaseAddress_
 0003:00008F3F       GetBaseAddress_
 0003:00009010       virt_to_phys_
 0003:0000903E       phys_to_virt_
 0003:0000907A       VMAlloc_
 0003:000090E0       VMFree_
 0003:000090EE       __get_free_dma_pages_
 0003:000092D9       __get_free_pages_
 0003:00009695       free_pages_
 0003:000096C2       vmalloc_
 0003:00009784       vfree_
 0003:000097B5       alloc_pages_
 0003:000097B8       remap_page_range_
 0003:000097BB       __ioremap_
 0003:00009812       iounmap_
 0003:00009825       is_access_ok_
 0003:0000982B       __copy_user_
 0003:00009854       copy_to_user_
 0003:0000987F       __copy_user_zeroing_
 0003:000098B4       copy_from_user_
 0003:000098DF       __get_user_
 0003:0000990A       _put_user_
 0003:0000991A       __kmalloc_
 0003:000099F5       __kfree_
 0003:00009A3A       kzalloc_
 0003:00009B2E       kcalloc_
 0003:00009BC2       uniaud_set_interrupted_substream_
 0003:00009BF5       WaitForControlChange_
 0003:00009C52       WaitForPCMInterrupt_
 0003:00009CF6       GetNumberOfCards_
 0003:00009CFC       GetNumberOfPcm_
 0003:00009D01       SetPCMInstance_
 0003:00009D20       GetPcmForChannels_
 0003:00009DAB       GetMaxChannels_
 0003:00009E27       GetUniaudPcmCaps1_
 0003:0000A120       FillCaps_
 0003:0000A172       GetUniaudPcmCaps_
 0003:0000A1BB       UniaudCtlGetPowerState_
 0003:0000A27F       UniaudCtlSetPowerState_
 0003:0000A343       GetUniaudCardInfo_
 0003:0000A41F       GetUniaudControlNum_
 0003:0000A552       GetUniaudControls_
 0003:0000A6BA       GetUniaudControlInfo_
 0003:0000A79B       GetUniaudControlValueGet_
 0003:0000A880       GetUniaudControlValuePut_
 0003:0000A965       UniaudIoctlHWRefine_
 0003:0000A9A6       UniaudIoctlHWParamSet_
 0003:0000A9E7       UniaudIoctlSWParamSet_
 0003:0000AA28       UniaudIoctlPCMStatus_
 0003:0000AA69       UniaudIoctlPCMWrite_
 0003:0000AA99       UniaudIoctlPCMRead_
 0003:0000AAC9       UniaudIoctlPCMPrepare_
 0003:0000AAFA       UniaudIoctlPCMResume_
 0003:0000AB2D       UniaudIoctlPCMStart_
 0003:0000AB5E       UniaudIoctlPCMDrop_
 0003:0000AB8F       UniaudCloseAll_
 0003:0000AC1A       request_irq_
 0003:0000AD3E       free_irq_
 0003:0000ADD7       eoi_irq_
 0003:0000ADE4       process_interrupt_
 0003:0000AEA5       in_interrupt_
 0003:0000AEAB       disable_irq_
 0003:0000AEAC       pci_read_config_byte_
 0003:0000AEEC       pci_read_config_word_
 0003:0000AF2E       pci_read_config_dword_
 0003:0000AF65       pci_write_config_byte_
 0003:0000AFA5       pci_write_config_word_
 0003:0000AFE6       pci_write_config_dword_
 0003:0000B01B       pcidev_prepare_
 0003:0000B021       pcidev_activate_
 0003:0000B027       pcidev_deactivate_
 0003:0000B455       pci_find_device_
 0003:0000B4EC       __request_region_
 0003:0000B566       __release_region_
 0003:0000B591       pci_get_flags_
 0003:0000B5B7       pcibios_present_
 0003:0000B5CE       pci_find_slot_
 0003:0000B5E2       pci_dma_supported_
 0003:0000B5F7       pci_find_capability_
 0003:0000B686       pci_set_power_state_
 0003:0000B7FA       pci_enable_device_
 0003:0000B838       pci_register_driver_
 0003:0000B96B       pci_module_init_
 0003:0000B97A       pci_unregister_driver_
 0003:0000BA0A       pci_set_master_
 0003:0000BA46       pm_register_
 0003:0000BA49       pm_unregister_
 0003:0000BA4A       __compat_get_order_
 0003:0000BA5F       pci_alloc_consistent_
 0003:0000BB1B       pci_free_consistent_
 0003:0000BB2B       pci_set_driver_data_
 0003:0000BB36       pci_get_driver_data_
 0003:0000BB41       pci_get_dma_mask_
 0003:0000BB4C       release_resource_
 0003:0000BB4F       pci_set_latency_time_
 0003:0000BB62       pci_orig_save_state_
 0003:0000BB8E       pci_orig_restore_state_
 0003:0000BBF1       pci_save_state_
 0003:0000BC3C       pci_restore_state_
 0003:0000BC90       pci_disable_device_
 0003:0000BCCC       pci_request_region_
 0003:0000C382       pci_release_region_
 0003:0000C6B1       pci_request_regions_
 0003:0000C6EC       pci_release_regions_
 0003:0000C706       pci_match_device_
 0003:0000C7AA       snd_pci_dev_present_
 0003:0000C805       snd_pci_compat_get_pci_driver_
 0003:0000C812       OSS32_APMResume_
 0003:0000C861       OSS32_APMSuspend_
 0003:0000C8B7       PciAdjustInterrupts_
 0003:0000C9B4       W?dumpheap$n()v
 0003:0000C9E5       W?SignatureCheck$n(pn$_MEMBLOCK$$pna)s
 0003:0000CA2A       W?HeapCheck$n(pna)v
 0003:0000CA83       W?npvAllocateBlock$n(pn$_MEMBLOCK$$ulpn$1$)pnv
 0003:0000CB00       W?malloc$n(ul)pnv
 0003:0000CC03       W?remove$n(pn$_MEMBLOCK$$)v
 0003:0000CC31       W?compact$n()v
 0003:0000CCD5       W?free$n(pnv)v
 0003:0000CE0F       W?_memfree$n()ui
 0003:0000CE15       W?_msize$n(pnv)ui
 0003:0000CE21       W?realloc$n(pnvul)pnv
 0003:0000CE94       W?IsHeapAddr$n(ul)ul
 0003:0000CEB4       W?HeapInit$n(ul)ul
 0003:0000CF14       strncpy_
 0003:0000CF39       init_waitqueue_head_
 0003:0000CF3A       add_wait_queue_
 0003:0000CF3B       add_wait_queue_exclusive_
 0003:0000CF3C       remove_wait_queue_
 0003:0000CF3D       interruptible_sleep_on_timeout_
 0003:0000CF43       interruptible_sleep_on_
 0003:0000CF44       __wake_up_
 0003:0000CF45       init_waitqueue_entry_
 0003:0000CF46       waitqueue_active_
 0003:0000CF49       spin_lock_init_
 0003:0000CF50       spin_lock_
 0003:0000CF5A       spin_lock_flag_
 0003:0000CF64       spin_trylock_
 0003:0000CF67       spin_unlock_
 0003:0000D524       snd_hwdep_new_
 0003:0000DAAF       snd_timer_open_
 0003:0000DC05       snd_timer_close_
 0003:0000DD5D       snd_timer_resolution_
 0003:0000DF39       snd_timer_start_
 0003:0000E095       snd_timer_stop_
 0003:0000E0DB       snd_timer_continue_
 0003:0000E155       snd_timer_pause_
 0003:0000E269       snd_timer_interrupt_
 0003:0000E4B1       snd_timer_new_
 0003:0000E765       snd_timer_notify_
 0003:0000E85B       snd_timer_global_new_
 0003:0000E890       snd_timer_global_free_
 0003:0000E895       snd_timer_global_register_
 0003:0000FF0D       snd_rawmidi_drop_output_
 0003:0000FF4F       snd_rawmidi_drain_output_
 0003:0000FFC3       snd_rawmidi_drain_input_
 0003:000101BA       snd_rawmidi_kernel_open_
 0003:000105C9       snd_rawmidi_kernel_release_
 0003:000106D9       snd_rawmidi_info_select_
 0003:000107DB       snd_rawmidi_output_params_
 0003:0001087F       snd_rawmidi_input_params_
 0003:000109C9       snd_rawmidi_receive_
 0003:00010C67       snd_rawmidi_kernel_read_
 0003:00010DAD       snd_rawmidi_transmit_empty_
 0003:00010DF6       snd_rawmidi_transmit_peek_
 0003:00010ED4       snd_rawmidi_transmit_ack_
 0003:00010F4F       snd_rawmidi_transmit_
 0003:000110CC       snd_rawmidi_kernel_write_
 0003:00011470       snd_rawmidi_new_
 0003:00011959       snd_rawmidi_set_ops_
 0003:00011A0D       snd_pcm_format_signed_
 0003:00011A35       snd_pcm_format_unsigned_
 0003:00011A48       snd_pcm_format_linear_
 0003:00011A58       snd_pcm_format_little_endian_
 0003:00011A80       snd_pcm_format_big_endian_
 0003:00011A93       snd_pcm_format_width_
 0003:00011ABB       snd_pcm_format_physical_width_
 0003:00011AE3       snd_pcm_format_size_
 0003:00011AF9       snd_pcm_format_silence_64_
 0003:00011B24       snd_pcm_format_set_silence_
 0003:00011C5D       snd_pcm_limit_hw_rates_
 0003:00011CC5       snd_pcm_rate_to_rate_bit_
 0003:0001212D       snd_pcm_playback_silence_
 0003:00012669       snd_pcm_update_hw_ptr_
 0003:0001275F       snd_pcm_set_ops_
 0003:00012784       snd_pcm_set_sync_
 0003:00012886       snd_interval_refine_
 0003:000129DC       snd_interval_mul_
 0003:00012A7A       snd_interval_div_
 0003:00012B33       snd_interval_muldivk_
 0003:00012BE2       snd_interval_mulkdiv_
 0003:00012CA4       snd_interval_ratnum_
 0003:000130C6       snd_interval_list_
 0003:000131BC       snd_pcm_hw_rule_add_
 0003:000132D4       snd_pcm_hw_constraint_mask_
 0003:00013301       snd_pcm_hw_constraint_mask64_
 0003:0001334E       snd_pcm_hw_constraint_integer_
 0003:0001336D       snd_pcm_hw_constraint_minmax_
 0003:000133D9       snd_pcm_hw_constraint_list_
 0003:00013462       snd_pcm_hw_constraint_ratnums_
 0003:000134EB       snd_pcm_hw_constraint_ratdens_
 0003:00013538       snd_pcm_hw_constraint_msbits_
 0003:0001357D       snd_pcm_hw_constraint_step_
 0003:000135C4       snd_pcm_hw_constraint_pow2_
 0003:00013640       _snd_pcm_hw_params_any_
 0003:00013686       snd_pcm_hw_param_value_
 0003:000136FD       _snd_pcm_hw_param_setempty_
 0003:000137C4       snd_pcm_hw_param_first_
 0003:00013861       snd_pcm_hw_param_last_
 0003:00013898       snd_pcm_hw_params_choose_
 0003:00013A15       snd_pcm_lib_ioctl_
 0003:00013A53       snd_pcm_period_elapsed_
 0003:00013EBB       snd_pcm_lib_write_
 0003:00014026       snd_pcm_lib_writev_
 0003:000142E9       snd_pcm_lib_read_
 0003:00014417       snd_pcm_lib_readv_
 0003:000146E9       snd_pcm_new_stream_
 0003:00014817       snd_pcm_new_
 0003:00014988       snd_pcm_attach_substream_
 0003:00014BE0       snd_pcm_detach_substream_
 0003:00014E30       snd_pcm_notify_
 0003:00014F8B       pcm_info_
 0003:00015027       pcm_instances_
 0003:0001508D       snd_lookup_minor_data_
 0003:0001516E       snd_register_device_for_dev_
 0003:0001525C       snd_unregister_device_
 0003:000152AB       snd_add_device_sysfs_file_
 0003:000153A5       snd_minor_info_init_
 0003:000153E6       snd_minor_info_done_
 0003:000154A5       snd_info_check_reserved_words_
 0003:00015B6A       snd_info_init_
 0003:00015C06       snd_info_done_
 0003:00015C54       snd_info_card_create_
 0003:00015CB6       snd_info_card_register_
 0003:00015CCF       snd_info_card_id_change_
 0003:00015D0E       snd_info_card_disconnect_
 0003:00015D62       snd_info_card_free_
 0003:00015D82       snd_info_get_line_
 0003:00015E0D       snd_info_get_str_
 0003:00015EEC       snd_info_create_module_entry_
 0003:00015F06       snd_info_create_card_entry_
 0003:00015F97       snd_card_proc_new_
 0003:00015FEF       snd_info_free_entry_
 0003:00016032       snd_info_register_
 0003:000161C0       snd_pcm_lib_preallocate_free_
 0003:000161C8       snd_pcm_lib_preallocate_free_for_all_
 0003:0001622A       snd_pcm_lib_preallocate_pages_
 0003:00016242       snd_pcm_lib_preallocate_pages_for_all_
 0003:000162A2       snd_pcm_sgbuf_ops_page_
 0003:000162C0       snd_pcm_sgbuf_get_chunk_size_
 0003:00016316       snd_pcm_lib_malloc_pages_
 0003:000163E1       snd_pcm_lib_free_pages_
 0003:0001643A       snd_pcm_timer_resolution_change_
 0003:0001652F       snd_pcm_timer_init_
 0003:00016628       snd_pcm_timer_done_
 0003:00016909       snd_pcm_info_
 0003:000169CA       snd_pcm_info_user_
 0003:00016A26       snd_pcm_hw_refine_
 0003:00017264       snd_pcm_status_
 0003:00017848       snd_pcm_start_
 0003:000178F0       snd_pcm_stop_
 0003:00017901       snd_pcm_drain_done_
 0003:00017AAF       snd_pcm_suspend_
 0003:00017B00       snd_pcm_suspend_all_
 0003:00018766       snd_pcm_hw_constraints_init_
 0003:00018AA9       snd_pcm_hw_constraints_complete_
 0003:00018C40       snd_pcm_release_substream_
 0003:00018CA9       snd_pcm_open_substream_
 0003:00019BE9       snd_pcm_kernel_ioctl_
 0003:00019E19       dummy_get_unmapped_area_
 0003:00019E1E       snd_oss_info_register_
 0003:00019FC4       snd_info_minor_register_
 0003:0001A018       snd_info_minor_unregister_
 0003:0001A02A       snd_lookup_oss_minor_data_
 0003:0001A0FC       snd_register_oss_device_
 0003:0001A187       snd_unregister_oss_device_
 0003:0001A2FE       snd_minor_info_oss_init_
 0003:0001A341       snd_minor_info_oss_done_
 0003:0001A359       snd_device_new_
 0003:0001A3AC       snd_device_free_
 0003:0001A443       snd_device_disconnect_
 0003:0001A4AD       snd_device_register_
 0003:0001A507       snd_device_register_all_
 0003:0001A545       snd_device_disconnect_all_
 0003:0001A57D       snd_device_free_all_
 0003:0001A7EA       snd_ctl_notify_
 0003:0001A953       snd_ctl_new1_
 0003:0001AA24       snd_ctl_free_one_
 0003:0001AAED       snd_ctl_add_
 0003:0001AC00       snd_ctl_remove_
 0003:0001AC6B       snd_ctl_remove_id_
 0003:0001AD28       snd_ctl_rename_id_
 0003:0001AD84       snd_ctl_find_numid_
 0003:0001ADB1       snd_ctl_find_id_
 0003:0001BF46       snd_ctl_register_ioctl_
 0003:0001BFA0       snd_ctl_unregister_ioctl_
 0003:0001C0AC       snd_ctl_create_
 0003:0001C0C4       snd_ctl_boolean_mono_info_
 0003:0001C0E3       snd_ctl_boolean_stereo_info_
 0003:0001C122       snd_malloc_pages_
 0003:0001C14E       snd_free_pages_
 0003:0001C178       snd_malloc_dev_pages_
 0003:0001C1B5       snd_free_dev_pages_
 0003:0001C1EA       snd_dma_alloc_pages_
 0003:0001C279       snd_dma_alloc_pages_fallback_
 0003:0001C2D9       snd_dma_free_pages_
 0003:0001C32C       snd_dma_get_reserved_buf_
 0003:0001C3DD       snd_dma_reserve_buf_
 0003:0001C542       snd_card_create_
 0003:0001C7A7       snd_card_locked_
 0003:0001C87E       snd_card_disconnect_
 0003:0001CA2D       snd_card_free_when_closed_
 0003:0001CA7D       snd_card_free_
 0003:0001CC67       snd_card_set_id_
 0003:0001CC8D       snd_card_register_
 0003:0001CD6B       snd_card_info_read_oss_
 0003:0001CDF4       snd_card_info_init_
 0003:0001CE72       snd_card_info_done_
 0003:0001CE89       snd_component_add_
 0003:0001CF4F       snd_card_file_add_
 0003:0001CFC3       snd_card_file_remove_
 0003:0001D076       snd_power_wait_
 0003:0001D136       snd_free_sgbuf_pages_
 0003:0001D17C       snd_malloc_sgbuf_pages_
 0003:000336A5       ioread8_
 0003:000336C0       ioread16_
 0003:000336DD       ioread32_
 0003:000336F3       iowrite8_
 0003:00033706       iowrite16_
 0003:0003371B       iowrite32_
 0003:0003372E       ioport_map_
 0003:0003373E       ioport_unmap_
 0003:0003373F       pci_iomap_
 0003:000338CA       pci_iounmap_
 0003:000338EE       snd_ca0106_ptr_read_
 0003:00033928       snd_ca0106_ptr_write_
 0003:00033962       snd_ca0106_spi_write_
 0003:00033A34       snd_ca0106_i2c_write_
 0003:000356A5       ca_midi_init_
 0003:0003609E       snd_ca0106_mixer_
 0003:0003623D       snd_ca0106_mixer_suspend_
 0003:00036276       snd_ca0106_mixer_resume_
 0003:00036AC9       snd_ca0106_proc_init_
 0003:0004B78D       snd_hda_add_codec_preset_
 0003:0004B7BD       snd_hda_delete_codec_preset_
 0003:0004B7E5       snd_hda_get_jack_location_
 0003:0004B82E       snd_hda_get_jack_connectivity_
 0003:0004B83C       snd_hda_get_jack_type_
 0003:0004B95B       snd_hda_codec_read_
 0003:0004B988       snd_hda_codec_write_
 0003:0004B9C1       snd_hda_sequence_write_
 0003:0004B9EE       snd_hda_get_sub_nodes_
 0003:0004BA26       snd_hda_get_connections_
 0003:0004BC45       snd_hda_queue_unsol_event_
 0003:0004BD28       snd_hda_bus_new_
 0003:0004C1B3       snd_hda_add_pincfg_
 0003:0004C222       snd_hda_codec_set_pincfg_
 0003:0004C237       snd_hda_codec_get_pincfg_
 0003:0004C36E       snd_hda_codec_new_
 0003:0004C5E3       snd_hda_codec_configure_
 0003:0004C6A8       snd_hda_codec_setup_stream_
 0003:0004C6EE       snd_hda_codec_cleanup_stream_
 0003:0004C7C3       query_amp_caps_
 0003:0004C834       snd_hda_override_amp_caps_
 0003:0004C8B1       snd_hda_query_pin_caps_
 0003:0004C9AB       snd_hda_codec_amp_read_
 0003:0004C9EB       snd_hda_codec_amp_update_
 0003:0004CA92       snd_hda_codec_amp_stereo_
 0003:0004CADD       snd_hda_codec_resume_amp_
 0003:0004CB90       snd_hda_mixer_amp_volume_info_
 0003:0004CC75       snd_hda_mixer_amp_volume_get_
 0003:0004CD0F       snd_hda_mixer_amp_volume_put_
 0003:0004CDBE       snd_hda_mixer_amp_tlv_
 0003:0004CE81       snd_hda_set_vmaster_tlv_
 0003:0004CF1D       snd_hda_find_mixer_ctl_
 0003:0004CF27       snd_hda_ctl_add_
 0003:0004CF55       snd_hda_ctls_clear_
 0003:0004CFEA       snd_hda_codec_reset_
 0003:0004D143       snd_hda_add_vmaster_
 0003:0004D1CD       snd_hda_mixer_amp_switch_info_
 0003:0004D1FD       snd_hda_mixer_amp_switch_get_
 0003:0004D294       snd_hda_mixer_amp_switch_put_
 0003:0004D34F       snd_hda_mixer_bind_switch_get_
 0003:0004D38A       snd_hda_mixer_bind_switch_put_
 0003:0004D42B       snd_hda_mixer_bind_ctls_info_
 0003:0004D463       snd_hda_mixer_bind_ctls_get_
 0003:0004D49C       snd_hda_mixer_bind_ctls_put_
 0003:0004D50A       snd_hda_mixer_bind_tlv_
 0003:0004D856       snd_hda_create_spdif_out_ctls_
 0003:0004D930       snd_hda_create_spdif_share_sw_
 0003:0004DA13       snd_hda_create_spdif_in_ctls_
 0003:0004DAB4       snd_hda_codec_write_cache_
 0003:0004DB2A       snd_hda_codec_resume_cache_
 0003:0004DB77       snd_hda_sequence_write_cache_
 0003:0004DD70       snd_hda_build_controls_
 0003:0004DDCD       snd_hda_codec_build_controls_
 0003:0004DE01       snd_hda_calc_stream_format_
 0003:0004E154       snd_hda_is_supported_format_
 0003:0004E3F4       snd_hda_codec_build_pcms_
 0003:0004E4A7       snd_hda_build_pcms_
 0003:0004E4CE       snd_hda_check_board_config_
 0003:0004E549       snd_hda_check_board_codec_sid_config_
 0003:0004E58F       snd_hda_add_new_ctls_
 0003:0004E5EC       snd_hda_ch_mode_info_
 0003:0004E623       snd_hda_ch_mode_get_
 0003:0004E647       snd_hda_ch_mode_put_
 0003:0004E690       snd_hda_input_mux_info_
 0003:0004E6DF       snd_hda_input_mux_put_
 0003:0004E81B       snd_hda_multi_out_dig_open_
 0003:0004E855       snd_hda_multi_out_dig_prepare_
 0003:0004E885       snd_hda_multi_out_dig_cleanup_
 0003:0004E8B3       snd_hda_multi_out_dig_close_
 0003:0004E8D5       snd_hda_multi_out_analog_open_
 0003:0004E9E9       snd_hda_multi_out_analog_prepare_
 0003:0004EB85       snd_hda_multi_out_analog_cleanup_
 0003:0004ECC8       snd_hda_parse_pin_def_config_
 0003:0004F25C       snd_hda_suspend_
 0003:0004F27F       snd_hda_resume_
 0003:0004F2A2       snd_array_new_
 0003:0004F320       snd_array_free_
 0003:0004F341       snd_print_pcm_rates_
 0003:0004F39C       snd_print_pcm_bits_
 0003:0004F57A       snd_hda_create_hwdep_
 0003:00050862       snd_hda_parse_generic_codec_
 0003:00051988       snd_hda_codec_proc_new_
 0003:00051AB4       snd_seq_device_load_drivers_
 0003:00051AB5       snd_seq_device_new_
 0003:00051C86       snd_seq_device_register_driver_
 0003:00051DC2       snd_seq_device_unregister_driver_
 0003:000520F7       snd_seq_info_init_
 0003:00052138       snd_seq_info_done_
 0003:000521B1       snd_seq_system_broadcast_
 0003:000521DE       snd_seq_system_notify_
 0003:0005221F       snd_seq_system_client_init_
 0003:00052349       snd_seq_system_client_done_
 0003:000523BB       snd_seq_queue_get_cur_queues_
 0003:00052575       snd_seq_queues_init_
 0003:00052578       snd_seq_queues_delete_
 0003:00052598       snd_seq_queue_alloc_
 0003:000525D7       snd_seq_queue_delete_
 0003:00052600       queueptr_
 0003:00052639       snd_seq_queue_find_name_
 0003:00052676       snd_seq_check_queue_
 0003:00052756       snd_seq_enqueue_event_
 0003:0005284F       snd_seq_queue_check_access_
 0003:00052889       snd_seq_queue_set_owner_
 0003:000528D8       snd_seq_queue_timer_open_
 0003:00052913       snd_seq_queue_timer_close_
 0003:0005292A       snd_seq_queue_timer_set_tempo_
 0003:00052998       snd_seq_queue_use_
 0003:00052A2C       snd_seq_queue_is_used_
 0003:00052A60       snd_seq_queue_client_termination_
 0003:00052AC3       snd_seq_queue_client_leave_
 0003:00052B52       snd_seq_queue_client_leave_cells_
 0003:00052B90       snd_seq_queue_remove_cells_
 0003:00052D42       snd_seq_control_queue_
 0003:00052D97       snd_seq_info_queues_read_
 0003:00052EFA       snd_seq_dump_var_event_
 0003:00052FEB       snd_seq_expand_var_event_
 0003:00053094       snd_seq_cell_free_
 0003:00053207       snd_seq_event_dup_
 0003:000533E3       snd_seq_pool_poll_wait_
 0003:00053403       snd_seq_pool_init_
 0003:000534A1       snd_seq_pool_done_
 0003:0005355C       snd_seq_pool_new_
 0003:000535C8       snd_seq_pool_delete_
 0003:000535E7       snd_sequencer_memory_init_
 0003:000535EA       snd_sequencer_memory_done_
 0003:000535EB       snd_seq_info_pool_
 0003:000536D7       snd_seq_client_use_ptr_
 0003:0005374A       client_init_data_
 0003:00053FBA       snd_seq_dispatch_event_
 0003:00054855       snd_seq_client_notify_subscription_
 0003:00054DF8       snd_seq_set_queue_tempo_
 0003:000555B6       snd_seq_create_kernel_client_
 0003:00055690       snd_seq_delete_kernel_client_
 0003:0005570C       snd_seq_kernel_client_enqueue_
 0003:00055718       snd_seq_kernel_client_enqueue_blocking_
 0003:0005572D       snd_seq_kernel_client_dispatch_
 0003:00055770       snd_seq_kernel_client_ctl_
 0003:00055783       snd_seq_kernel_client_write_poll_
 0003:000559C4       snd_seq_info_clients_read_
 0003:00055AE6       snd_sequencer_device_init_
 0003:00055B3F       snd_sequencer_device_done_
 0003:00055B84       snd_seq_port_use_ptr_
 0003:00055BE2       snd_seq_port_query_nearest_
 0003:00055C7F       snd_seq_create_port_
 0003:00055EE4       snd_seq_delete_port_
 0003:00055F6B       snd_seq_delete_all_ports_
 0003:0005601E       snd_seq_set_port_info_
 0003:000560A9       snd_seq_get_port_info_
 0003:00056294       snd_seq_port_connect_
 0003:000564F8       snd_seq_port_disconnect_
 0003:00056618       snd_seq_port_get_subscription_
 0003:0005665C       snd_seq_event_port_attach_
 0003:000566EA       snd_seq_event_port_detach_
 0003:00056805       snd_seq_timer_new_
 0003:00056849       snd_seq_timer_delete_
 0003:00056882       snd_seq_timer_defaults_
 0003:000568EE       snd_seq_timer_reset_
 0003:000569AF       snd_seq_timer_set_tempo_
 0003:000569F3       snd_seq_timer_set_ppq_
 0003:00056A5A       snd_seq_timer_set_position_tick_
 0003:00056A8A       snd_seq_timer_set_position_time_
 0003:00056AC4       snd_seq_timer_set_skew_
 0003:00056B0A       snd_seq_timer_open_
 0003:00056C06       snd_seq_timer_close_
 0003:00056C29       snd_seq_timer_stop_
 0003:00056CD4       snd_seq_timer_start_
 0003:00056D1D       snd_seq_timer_continue_
 0003:00056D6E       snd_seq_timer_get_cur_time_
 0003:00056DFE       snd_seq_timer_get_cur_tick_
 0003:00056E02       snd_seq_info_timer_read_
 0003:00056EB4       snd_seq_prioq_new_
 0003:00056EFE       snd_seq_prioq_delete_
 0003:00056FA9       snd_seq_prioq_cell_in_
 0003:00057075       snd_seq_prioq_cell_out_
 0003:000570CC       snd_seq_prioq_avail_
 0003:000570EA       snd_seq_prioq_cell_peek_
 0003:0005714A       snd_seq_prioq_leave_
 0003:000572C2       snd_seq_prioq_remove_events_
 0003:00057371       snd_seq_fifo_new_
 0003:000573F5       snd_seq_fifo_delete_
 0003:0005743E       snd_seq_fifo_clear_
 0003:00057476       snd_seq_fifo_event_in_
 0003:00057527       snd_seq_fifo_cell_out_
 0003:000575B2       snd_seq_fifo_cell_putback_
 0003:000575E6       snd_seq_fifo_poll_wait_
 0003:00057601       snd_seq_fifo_resize_
 0003:0005768A       snd_opl3_synth_use_inc_
 0003:000576A6       snd_opl3_synth_use_dec_
 0003:000576A7       snd_opl3_synth_setup_
 0003:00057751       snd_opl3_synth_cleanup_
 0003:00057E77       snd_opl3_interrupt_
 0003:00057EEA       snd_opl3_new_
 0003:00057F6D       snd_opl3_init_
 0003:00057FDE       snd_opl3_create_
 0003:00058127       snd_opl3_timer_new_
 0003:00058164       snd_opl3_hwdep_new_
 0003:000584EA       snd_opl3_load_drums_
 0003:0005855B       snd_opl3_drum_switch_
 0003:00058608       snd_opl3_calc_volume_
 0003:00058851       snd_opl3_timer_func_
 0003:00058941       snd_opl3_note_on_
 0003:00058FBC       snd_opl3_note_off_
 0003:0005905C       snd_opl3_key_press_
 0003:0005905D       snd_opl3_terminate_note_
 0003:0005918B       snd_opl3_control_
 0003:000591F0       snd_opl3_nrpn_
 0003:000591F1       snd_opl3_sysex_
 0003:000591F4       snd_opl3_open_
 0003:000591F7       snd_opl3_ioctl_
 0003:00059373       snd_opl3_release_
 0003:00059381       snd_opl3_write_
 0003:00059477       snd_opl3_load_patch_
 0003:00059561       snd_opl3_find_patch_
 0003:000595D6       snd_opl3_clear_patches_
 0003:00059614       snd_opl3_reset_
 0003:00059AC8       snd_mpu401_uart_interrupt_
 0003:00059ADA       snd_mpu401_uart_interrupt_tx_
 0003:0005A05C       snd_mpu401_uart_new_
 0003:0005A998       snd_cs46xx_download_
 0003:0005A9D1       snd_cs46xx_download_image_
 0003:0005B75B       snd_cs46xx_pcm_
 0003:0005B9CE       snd_cs46xx_mixer_
 0003:0005BDD5       snd_cs46xx_midi_
 0003:0005BE8C       snd_cs46xx_gameport_
 0003:0005C27C       snd_cs46xx_start_dsp_
 0003:0005C50F       snd_cs46xx_suspend_
 0003:0005C5CE       snd_cs46xx_resume_
 0003:0005C6D3       snd_cs46xx_create_
 0003:0005D097       snd_cs5535audio_suspend_
 0003:0005D13B       snd_cs5535audio_resume_
 0003:0005D679       snd_cs5535audio_pcm_
 0003:0005E350       snd_p16v_free_
 0003:0005E361       snd_p16v_pcm_
 0003:0005E736       snd_p16v_mixer_
 0003:0005E775       snd_p16v_alloc_pm_buffer_
 0003:0005E797       snd_p16v_free_pm_buffer_
 0003:0005E7A2       snd_p16v_suspend_
 0003:0005E7D4       snd_p16v_resume_
 0003:0005E8B1       snd_emu10k1_timer_
 0003:0005EC32       snd_emu10k1_fx8010_register_irq_handler_
 0003:0005ECD3       snd_emu10k1_fx8010_unregister_irq_handler_
 0003:0005EE2C       snd_emu10k1_efx_read_
 0003:00065291       snd_emu10k1_init_efx_
 0003:000652C9       snd_emu10k1_free_efx_
 0003:00065303       snd_emu10k1_fx8010_tram_setup_
 0003:00065A8D       snd_emu10k1_fx8010_new_
 0003:00065B3E       snd_emu10k1_efx_alloc_pm_buffer_
 0003:00065BE5       snd_emu10k1_efx_free_pm_buffer_
 0003:00065C16       snd_emu10k1_efx_suspend_
 0003:00065D39       snd_emu10k1_efx_resume_
 0003:000674D8       snd_emu10k1_mixer_
 0003:00069A85       snd_emu10k1_pcm_
 0003:00069BA5       snd_emu10k1_pcm_multi_
 0003:00069C82       snd_emu10k1_pcm_mic_
 0003:0006A41E       snd_emu10k1_pcm_efx_
 0003:0006AB2D       snd_emu10k1_midi_
 0003:0006AB7A       snd_emu10k1_audigy_midi_
 0003:0006AC12       snd_emu10k1_voice_init_
 0003:0006B384       snd_emu10k1_done_
 0003:0006C2CB       snd_emu10k1_create_
 0003:0006C8C7       snd_emu10k1_suspend_regs_
 0003:0006C956       snd_emu10k1_resume_init_
 0003:0006C9BA       snd_emu10k1_resume_regs_
 0003:0006D37D       snd_emu10k1_proc_init_
 0003:0006D5A4       snd_emu10k1_ptr_read_
 0003:0006D660       snd_emu10k1_ptr_write_
 0003:0006D734       snd_emu10k1_ptr20_read_
 0003:0006D774       snd_emu10k1_ptr20_write_
 0003:0006D7B4       snd_emu10k1_spi_write_
 0003:0006D8AA       snd_emu10k1_i2c_write_
 0003:0006D9B5       snd_emu1010_fpga_write_
 0003:0006DA40       snd_emu1010_fpga_read_
 0003:0006DAB7       snd_emu1010_fpga_link_dst_src_write_
 0003:0006DB0B       snd_emu10k1_intr_enable_
 0003:0006DB44       snd_emu10k1_intr_disable_
 0003:0006DB7F       snd_emu10k1_voice_intr_enable_
 0003:0006DBE4       snd_emu10k1_voice_intr_disable_
 0003:0006DC4B       snd_emu10k1_voice_intr_ack_
 0003:0006DCAB       snd_emu10k1_voice_half_loop_intr_enable_
 0003:0006DD10       snd_emu10k1_voice_half_loop_intr_disable_
 0003:0006DD77       snd_emu10k1_voice_half_loop_intr_ack_
 0003:0006DDD7       snd_emu10k1_voice_set_loop_stop_
 0003:0006DE3C       snd_emu10k1_voice_clear_loop_stop_
 0003:0006DEA3       snd_emu10k1_wait_
 0003:0006DEFE       snd_emu10k1_ac97_read_
 0003:0006DF40       snd_emu10k1_ac97_write_
 0003:0006DF82       snd_emu10k1_rate_to_pitch_
 0003:0006E15E       snd_emu10k1_voice_alloc_
 0003:0006E1F1       snd_emu10k1_voice_free_
 0003:0006E513       snd_emu10k1_memblk_map_
 0003:0006E5B3       snd_emu10k1_alloc_pages_
 0003:0006E6A4       snd_emu10k1_free_pages_
 0003:0006E6A9       snd_emu10k1_synth_alloc_
 0003:0006E709       snd_emu10k1_synth_free_
 0003:0006E94E       snd_emu10k1_synth_bzero_
 0003:0006E9C2       snd_emu10k1_synth_copy_from_user_
 0003:0006EA50       snd_emu10k1_interrupt_
 0003:0006EE6D       snd_ymfpci_free_gameport_
 0003:0007093A       snd_ymfpci_pcm_
 0003:00070A0B       snd_ymfpci_pcm2_
 0003:00070AC5       snd_ymfpci_pcm_spdif_
 0003:00070B84       snd_ymfpci_pcm_4ch_
 0003:00071427       snd_ymfpci_mixer_
 0003:000716E2       snd_ymfpci_timer_
 0003:00071DF1       snd_ymfpci_suspend_
 0003:00071EBA       snd_ymfpci_resume_
 0003:00071FA4       snd_ymfpci_create_
 0003:00074892       snd_trident_start_voice_
 0003:000748BD       snd_trident_stop_voice_
 0003:000749CE       snd_trident_write_voice_regs_
 0003:00075FD6       snd_trident_pcm_
 0003:0007612C       snd_trident_foldback_pcm_
 0003:000762CF       snd_trident_spdif_pcm_
 0003:0007707F       snd_trident_create_gameport_
 0003:000776B1       snd_trident_create_
 0003:00077BE6       snd_trident_alloc_voice_
 0003:00077C96       snd_trident_free_voice_
 0003:00077DD3       snd_trident_suspend_
 0003:00077E55       snd_trident_resume_
 0003:000781B7       snd_trident_alloc_pages_
 0003:000781C6       snd_trident_free_pages_
 0003:000797A5       snd_sbmixer_write_
 0003:000797D0       snd_sbmixer_read_
 0003:0007A0AC       snd_sbmixer_add_ctl_
 0003:0007A1D1       snd_sbmixer_new_
 0003:0007A35E       snd_sbmixer_suspend_
 0003:0007A3D2       snd_sbmixer_resume_
 0003:0007A446       snd_sbdsp_command_
 0003:0007A499       snd_sbdsp_get_byte_
 0003:0007A4E1       snd_sbdsp_reset_
 0003:0007A6CA       snd_sbdsp_create_
 0003:0007B387       _snd_pcm_hw_param_set_
 0003:0007C1AD       snd_pcm_oss_write3_
 0003:0007C20C       snd_pcm_oss_read3_
 0003:0007C29E       snd_pcm_oss_writev3_
 0003:0007C2FD       snd_pcm_oss_readv3_
 0003:0007E020       ACPIFindPCIDevice
 0003:0007E0C2       InitACPICall
 0003:0007E160       StrLen
 0003:0007E180       StrNCmp
 0003:0007E1B0       FindAddress
 0003:0007E41C       init_MUTEX_
 0003:0007E41D       init_MUTEX_LOCKED_
 0003:0007E41E       down_
 0003:0007E41F       up_
 0003:0007E420       down_interruptible_
 0003:0007E70B       _snd_ctl_add_slave_
 0003:0007E8D5       snd_ctl_make_virtual_master_
 0003:0007E997       release_and_free_resource_
 0003:0007E9AC       snd_pci_quirk_lookup_
 0003:0007E9EC       copy_to_user_fromio_
 0003:0007EA5A       copy_from_user_toio_
 0003:0007ECD0       snd_ac97_set_rate_
 0003:0007F08E       snd_ac97_pcm_assign_
 0003:0007F409       snd_ac97_pcm_open_
 0003:0007F695       snd_ac97_pcm_close_
 0003:0007F75D       snd_ac97_pcm_double_rate_rules_
 0003:00082CCA       snd_ac97_write_
 0003:00082D27       snd_ac97_read_
 0003:00082DA1       snd_ac97_write_cache_
 0003:00082DF7       snd_ac97_update_
 0003:00082E77       snd_ac97_update_bits_
 0003:00082EC1       snd_ac97_update_bits_nolock_
 0003:00084E7E       snd_ac97_get_name_
 0003:00085011       snd_ac97_get_short_name_
 0003:000850F4       snd_ac97_bus_
 0003:00085177       snd_ac97_mixer_
 0003:00085BF5       snd_ac97_suspend_
 0003:00085CF8       snd_ac97_resume_
 0003:00086463       snd_ac97_tune_hardware_
 0003:00087409       snd_ac97_proc_init_
 0003:000874ED       snd_ac97_proc_done_
 0003:00087510       snd_ac97_bus_proc_init_
 0003:0008756B       snd_ac97_bus_proc_done_
 0003:0008757F       snd_midi_process_event_
 0003:00087B67       snd_midi_channel_set_clear_
 0003:0008800F       snd_midi_channel_alloc_set_
 0003:00088066       snd_midi_channel_free_set_
 0003:0008808D       snd_util_memhdr_new_
 0003:000880C0       snd_util_memhdr_free_
 0003:000880F4       __snd_util_mem_alloc_
 0003:00088148       __snd_util_memblk_new_
 0003:0008819E       snd_util_mem_alloc_
 0003:000881C1       __snd_util_mem_free_
 0003:000881E2       snd_util_mem_free_
 0003:00088203       snd_util_mem_avail_
 0003:00088230       __U8RS
 0003:0008824A       __I8RS
 0003:00088265       __U8LS
 0003:00088265       __I8LS
 0003:00088280       __I8M
 0003:00088280       __U8M
 0003:000882A0       strstr_
 0003:00088350       strlcpy_
 0003:000883E0       vsscanf_
 0003:00088410       sscanf_
 0003:00088480       vsnprintf_
 0003:000884E0       snprintf_
 0003:00088510       memset_
 0003:00088530       memmove_
 0003:00088590       __IsTable
 0003:000886A0       __STOSB
 0003:000886D7       __STOSD
 0003:000892B0       __scnf_
 0003:00089520       __prtf_
 0003:0008A204       __FDFS
 0003:0008A250       strupr_
 0003:0008A270       __Bits
 0003:0008A2D0       wctomb_
 0003:0008A300       mbtowc_
 0003:0008A3C0       _ismbblead_
 0003:0008A3E0       ultoa_
 0003:0008A430       ltoa_
 0003:0008A460       ulltoa_
 0003:0008A4D0       lltoa_
 0003:0008A500       utoa_
 0003:0008A550       itoa_
 0003:0008A580       tolower_
 0003:0008A590       __exit_with_msg_
 0003:0008A5E0       __fatal_runtime_error_
 0003:0008A63A       __mbinit_
 0003:0008A73C       __threadstack_
 0003:0008A743       __threadid_
 0003:0008A74C       __OS2MainInit_
 0003:0008A7BB       __OS2Init_
 0003:0008A7F9       __OS2Fini_
 0003:0008A801       __shutdown_stack_checking_
 0003:0008A816       __exit_
 0003:0008A860       __EnterWVIDEO_
 0003:0008A8A0       __InitRtns
 0003:0008A8F0       __FiniRtns
 0003:0008A950       __CommonInit_
 0003:0008AB80       strtoul_
 0003:0008AB90       strtol_
 0003:0008AB9D       __set_errno_
 0003:0008ABAB       __set_EDOM_
 0003:0008ABB9       __set_ERANGE_
 0003:0008ABC7       __set_EINVAL_
 0003:0008ABDA       __set_doserrno_
 0003:0008ABE8       __OffFinalCS32
 0004:00000003       ___begtext
 0005:00000000       __OffBeginDS32
 0005:00000030       W?deviceOwner$nul
 0005:00000034       W?numOS2Opens$nul
 0005:00000038       _rdOffset
 0005:0000003C       _wrOffset
 0005:00000040       _szprintBuf
 0005:00000044       _fVerbose
 0005:00000048       _fDebug
 0005:0000004C       _idc16_PddHandler
 0005:00000054       W?RM_Help$npn()i
 0005:00000058       W?RM_Help0$npn()i
 0005:0000005C       W?RM_Help3$npn()i
 0005:00000060       W?RMFlags$nul
 0005:000000B0       W?fnCardExitCall$n[]pn()v
 0005:000000D0       _nrCardsDetected
 0005:000000D4       _fStrategyInit
 0005:000000D8       _DbgInt
 0005:000000FC       _DebugLevel
 0005:00000104       _ulget_free_pagesMemUsed
 0005:00000548       W?pmbUsed$npn$_MEMBLOCK$$
 0005:0000054C       W?pmbFree$npn$_MEMBLOCK$$
 0005:00000550       W?uMemFree$nui
 0005:00000554       W?acHeap$npnuc
 0005:00000558       W?ulnAlloc$nul
 0005:0000055C       W?ulcAlloc$nul
 0005:00000560       W?ulnAllocCalls$nul
 0005:00000564       W?ulnFree$nul
 0005:00000568       W?ulcFree$nul
 0005:0000056C       W?ulnFreeCalls$nul
 0005:00000570       W?ulnCompact$nul
 0005:0000059C       _snd_pcm_devices_os2
 0005:00000AA4       _snd_ecards_limit
 0005:00000AA8       _snd_major
 0005:00000AB4       _snd_seq_root
 0005:00000AB8       _snd_oss_root
 0005:00000DA8       _snd_cards
 0005:00001524       ___MBCSIsTable
 0005:00001628       ___IsDBCS
 0005:0000162C       ___Is_DLL
 0005:00001630       ___saved_CS
 0005:00001734       ___hmodule
 0005:00001758       BootCode
 0005:00001768       stackbase
 0005:0000176C       stacksel
 0005:00001770       __OffsetFinalCS16
 0005:00001772       __OffsetFinalDS16
 0005:00001774       _MSG_TABLE32
 0005:00001778       PDDName
 0005:0000177C       RMAllocResource1632
 0005:00001784       RMModifyResources1632
 0005:0000178C       RMDeallocResource1632
 0005:00001794       RMCreateDevice1632
 0005:0000179C       RMCreateAdapter1632
 0005:000017A4       RMCreateDriver1632
 0005:000017AC       RMDestroyDriver1632
 0005:000017B4       RMGetNodeInfo1632
 0005:000017BC       RMDevIDToHandleList1632
 0005:000017C4       RMHandleToResourceHandleList1632
 0005:000017CC       _TimerHandler16
 0005:000017D2       _ISR00
 0005:000017D6       _ISR01
 0005:000017DA       _ISR02
 0005:000017DE       _ISR03
 0005:000017E2       _ISR04
 0005:000017E6       _ISR05
 0005:000017EA       _ISR06
 0005:000017EE       _ISR07
 0005:000017F4       DevHelp32
 0005:000017F8       intSwitchStack
 0005:000017FC       _TKSSBase
 0005:00001800       W?StratDispatch$n[]pn(pf$RP$$)ul
 0005:00001894       W?ForceCard$ni
 0005:000018C4       _jiffies
 0005:000018C8       _current_task
 0005:000018EC       _current
 0005:000018F0       _system_utsname
 0005:00001A76       _ioport_resource
 0005:00001A92       _iomem_resource
 0005:00001AAE       _mem_map
 0005:00001AB2       _this_module
 0005:00001BB2       _szLastALSAError1
 0005:00001C32       _szOverrunTest1
 0005:00001C33       _szLastALSAError2
 0005:00001CB3       _szOverrunTest2
 0005:00001CB4       _iLastError
 0005:00001CB8       _proc_root
 0005:00001D04       _cardcalls
 0005:00001E0C       _midi_port
 0005:00001F78       _szRecSources
 0005:00002004       _oss_devices
 0005:00002144       _alsa_fops
 0005:00002148       _per_bytes
 0005:0000214C       _prev_size
 0005:00002150       _pcm_device
 0005:00002154       _total
 0005:00002158       _opened_handles
 0005:000081D4       _CountWv
 0005:000081D8       _LockAdd
 0005:000081DC       _hextab
 0005:000081ED       _MAGIC_COMM_PORT
 0005:000081F0       _pcmcaps
 0005:00008210       _substream_int
 0005:0000A210       _control_id_changed
 0005:0000A214       _card_id_changed
 0005:0000A218       _unlock_all
 0005:0000A21C       _fInInterrupt
 0005:0000AA9C       _pci_devices
 0005:0000D5DC       _fRewired
 0005:0000E9E0       W?ulcTotalHeap$nul
 0005:0000EA44       ___initcall_alsa_hwdep_init
 0005:0000EA48       ___exitcall_alsa_hwdep_exit
 0005:0000EAF0       ___initcall_alsa_timer_init
 0005:0000EAF4       ___exitcall_alsa_timer_exit
 0005:0000EB80       ___initcall_alsa_rawmidi_init
 0005:0000EB84       ___exitcall_alsa_rawmidi_exit
 0005:0000EE60       ___initcall_alsa_pcm_init
 0005:0000EE64       ___exitcall_alsa_pcm_exit
 0005:0000EEBC       ___initcall_alsa_sound_init
 0005:0000EEC0       ___exitcall_alsa_sound_exit
 0005:0000EF44       _snd_pcm_link_rwlock
 0005:0000F008       _snd_pcm_f_ops
 0005:0000F114       ___initcall_snd_mem_init
 0005:0000F118       ___exitcall_snd_mem_exit
 0005:0000F574       ___initcall_alsa_card_bt87x_init
 0005:0000F578       ___exitcall_alsa_card_bt87x_exit
 0005:0000F710       ___initcall_alsa_card_als4000_init
 0005:0000F714       ___exitcall_alsa_card_als4000_exit
 0005:00010571       ___initcall_alsa_card_cmipci_init
 0005:00010575       ___exitcall_alsa_card_cmipci_exit
 0005:00010914       ___initcall_alsa_card_atiixp_init
 0005:00010918       ___exitcall_alsa_card_atiixp_exit
 0005:00010DD4       ___initcall_alsa_card_fm801_init
 0005:00010DD8       ___exitcall_alsa_card_fm801_exit
 0005:000113E8       ___initcall_alsa_card_via82xx_init
 0005:000113EC       ___exitcall_alsa_card_via82xx_exit
 0005:00011A0C       ___initcall_alsa_card_m3_init
 0005:00011A10       ___exitcall_alsa_card_m3_exit
 0005:00012980       ___initcall_alsa_card_intel8x0_init
 0005:00012984       ___exitcall_alsa_card_intel8x0_exit
 0005:00012C34       ___initcall_alsa_card_es1968_init
 0005:00012C38       ___exitcall_alsa_card_es1968_exit
 0005:000134CD       ___initcall_alsa_card_es1938_init
 0005:000134D1       ___exitcall_alsa_card_es1938_exit
 0005:000137A0       ___initcall_alsa_card_cs4281_init
 0005:000137A4       ___exitcall_alsa_card_cs4281_exit
 0005:00013C1C       ___initcall_alsa_card_ens137x_init
 0005:00013C20       ___exitcall_alsa_card_ens137x_exit
 0005:00014108       ___initcall_alsa_card_ca0106_init
 0005:0001410C       ___exitcall_alsa_card_ca0106_exit
 0005:00015E1C       ___initcall_patch_via_init
 0005:00015E20       ___exitcall_patch_via_exit
 0005:00017C3C       ___initcall_patch_conexant_init
 0005:00017C40       ___exitcall_patch_conexant_exit
 0005:00017D98       ___initcall_patch_atihdmi_init
 0005:00017D9C       ___exitcall_patch_atihdmi_exit
 0005:0001AC2E       ___initcall_patch_sigmatel_init
 0005:0001AC32       ___exitcall_patch_sigmatel_exit
 0005:00022140       ___initcall_patch_analog_init
 0005:00022144       ___exitcall_patch_analog_exit
 0005:000228D0       ___initcall_patch_cmedia_init
 0005:000228D4       ___exitcall_patch_cmedia_exit
 0005:0003F3FD       ___initcall_patch_realtek_init
 0005:0003F401       ___exitcall_patch_realtek_exit
 0005:0003FA2C       ___initcall_alsa_card_azx_init
 0005:0003FA30       ___exitcall_alsa_card_azx_exit
 0005:0003FB83       _snd_hda_bind_vol
 0005:0003FB93       _snd_hda_bind_sw
 0005:0003FE1F       _auto_pin_cfg_labels
 0005:0003FFE8       _seq_client_load
 0005:00040024       _seq_default_timer_class
 0005:00040028       _seq_default_timer_sclass
 0005:0004002C       _seq_default_timer_card
 0005:00040030       _seq_default_timer_device
 0005:00040034       _seq_default_timer_subdevice
 0005:00040038       _seq_default_timer_resolution
 0005:0004003C       ___initcall_alsa_seq_init
 0005:00040040       ___exitcall_alsa_seq_exit
 0005:00040064       ___initcall_alsa_seq_device_init
 0005:00040068       ___exitcall_alsa_seq_device_exit
 0005:000401B8       _use_internal_drums
 0005:000401BC       _opl3_ops
 0005:000401E0       ___initcall_alsa_opl3_seq_init
 0005:000401E4       ___exitcall_alsa_opl3_seq_exit
 0005:00040254       ___initcall_alsa_opl3_init
 0005:00040258       ___exitcall_alsa_opl3_exit
 0005:000403EC       _snd_opl3_regmap
 0005:00040430       ___initcall_alsa_mpu401_uart_init
 0005:00040434       ___exitcall_alsa_mpu401_uart_exit
 0005:0004054C       ___initcall_alsa_card_cs46xx_init
 0005:00040550       ___exitcall_alsa_card_cs46xx_exit
 0005:0004E22C       ___initcall_alsa_card_cs5535audio_init
 0005:0004E230       ___exitcall_alsa_card_cs5535audio_exit
 0005:0004E498       ___initcall_alsa_card_emu10k1_init
 0005:0004E49C       ___exitcall_alsa_card_emu10k1_exit
 0005:00051234       ___initcall_alsa_card_ymfpci_init
 0005:00051238       ___exitcall_alsa_card_ymfpci_exit
 0005:00051BF4       ___initcall_alsa_card_ali_init
 0005:00051BF8       ___exitcall_alsa_card_ali_exit
 0005:00051D30       ___initcall_alsa_card_trident_init
 0005:00051D34       ___exitcall_alsa_card_trident_exit
 0005:0005EA24       ___initcall_alsa_card_nm256_init
 0005:0005EA28       ___exitcall_alsa_card_nm256_exit
 0005:0005EFE8       ___initcall_alsa_sb_common_init
 0005:0005EFEC       ___exitcall_alsa_sb_common_exit
 0005:0005F068       ___initcall_alsa_pcm_oss_init
 0005:0005F06C       ___exitcall_alsa_pcm_oss_exit
 0005:0005F070       ___EFG_printf
 0005:0005F074       ___EFG_scanf
 0005:0005F078       ___MBCodePage
 0005:0005F07C       ___FirstThreadData
 0005:0005F080       ___GetThreadPtr
 0005:0005F084       __AccessFileH
 0005:0005F088       __ReleaseFileH
 0005:0005F08C       __AccessIOB
 0005:0005F090       __ReleaseIOB
 0005:0005F094       __AccessNHeap
 0005:0005F098       __AccessFHeap
 0005:0005F09C       __ReleaseNHeap
 0005:0005F0A0       __ReleaseFHeap
 0005:0005F0A4       __AccessTDList
 0005:0005F0A8       __ReleaseTDList
 0005:0005F0AC       ___sig_init_rtn
 0005:0005F0B0       ___sig_fini_rtn
 0005:0005F0B4       __threadstksize
 0005:0005F0B8       ___process_fini
 0005:0005F0BC       ___WD_Present
 0005:0005F0C0       __dynend
 0005:0005F0C4       __curbrk
 0005:0005F0C8       __LpCmdLine
 0005:0005F0CC       __LpPgmName
 0005:0005F0D0       __LpDllName
 0005:0005F0D4       __LpwCmdLine
 0005:0005F0D8       __LpwPgmName
 0005:0005F0DC       __LpwDllName
 0005:0005F0E0       __STACKLOW
 0005:0005F0E4       __STACKTOP
 0005:0005F0E8       __ASTACKSIZ
 0005:0005F0EC       __ASTACKPTR
 0005:0005F0F0       __cbyte
 0005:0005F0F4       __cbyte2
 0005:0005F0F8       __child
 0005:0005F0FC       __no87
 0005:0005F0FE       __Envptr
 0005:0005F102       __Envseg
 0005:0005F104       __osmajor
 0005:0005F105       __osminor
 0005:0005F106       ___FPE_handler
 0005:0005F10C       __amblksiz
 0005:0005F96E       ___initcall_alsa_ac97_init
 0005:0005F972       ___exitcall_alsa_ac97_exit
 0005:0005FA98       ___initcall_alsa_seq_midi_emul_init
 0005:0005FA9C       ___exitcall_alsa_seq_midi_emul_exit
 0005:0005FAA0       ___initcall_alsa_util_mem_init
 0005:0005FAA4       ___exitcall_alsa_util_mem_exit
 0005:0006F278       ___Alphabet
 0005:00071F50       _snd_pcm_known_rates
 0005:00077368       __OffFinalDS32
 0005:0007736C       __Start_XI
 0005:00077372       __Start_YI
 0005:00077372       __End_XI
 0005:00077372       __End_YI
 0005:000773C0       __nullarea
 0005:000873D0       _end
 0005:000873D0       _edata
